:100000000C9470170C949A170C949A170C949A17D6
:100010000C949A170C949A170C949A170C949A179C
:100020000C949A170C9481640C949A170C949A1758
:100030000C949A170C9448480C949A170C949A179D
:100040000C949A170C94BACD0C9424400C949A17E3
:100050000C94A3860C949A170C949A170C949A17E4
:100060000C949A170C949A170C949A170C949A174C
:100070000C949A170C949A170C949A170C949A173C
:100080000C949A170C949A170C949A17153F183FD2
:100090000B3F0F3F2F3F2F3F1C3F203F263F2A3F64
:1000A000933F983F9D3FA73FD53FD53FB13FB93FD5
:1000B000C13FCB3F084AD73B3BCE016E84BCBFFD5E
:1000C000C12F3D6C74319ABD56833DDA3D00C77F28
:1000D00011BED9E4BB4C3E916BAAAABE00000080C1
:1000E0003F05A84CCDB2D44EB93836A9020C50B950
:1000F000918688083CA6AAAA2ABE000000803F007C
:100100004E414E494E495459494E46CDCCCC3D0AFC
:10011000D7233C17B7D13877CC2B329595E6241FDF
:10012000B14F0A000020410000C84200401C462098
:10013000BCBE4CCA1B0E5AAEC59D74434F4D4D55A7
:100140004E49434154494F4E0044525952554E0076
:100150004552524F525300494E464F004543484F77
:100160000020746F6F206C6F6E67206578747275F5
:1001700073696F6E2070726576656E7465640A00CF
:1001800020636F6C6420657874727573696F6E207C
:1001900070726576656E7465640A0047322F473366
:1001A0002062616420706172616D65746572730AAA
:1001B00000536C6565702E2E2E004E6F206D6F768D
:1001C000652E00456E642066696C65206C697374E9
:1001D0000A00426567696E2066696C65206C697308
:1001E000740A00286E6F2066696C652900534420EC
:1001F0007072696E74696E67206279746520004E52
:100200006F74205344207072696E74696E670A00BF
:1002100043757272656E742066696C653A2000469B
:10022000696C652064656C657465643A0044656C4E
:100230006574696F6E206661696C65642C2046691F
:100240006C653A20002569730025696D2025697366
:10025000002569682025696D20256973002569647A
:10026000202569682025696D202569730025697935
:1002700020256964202569682025696D202569731A
:10028000005072696E742074696D653A20005C01DB
:100290005701500149013B016F66660044454255D4
:1002A000473A004B494C4C45442E20004D313133E8
:1002B0002053006F6B0020573A0042656420636F43
:1002C0006F6C696E672E2E2E004265642068656132
:1002D00074696E672E2E2E002C20002C20005448AE
:1002E00045524D414C5F50524F54454354494F4E37
:1002F000004155544F5245504F52545F53445F5341
:10030000544154555300454D455247454E43595F5E
:1003100050415253455200434153455F4C49474871
:10032000545F4252494748544E45535300544F4737
:10033000474C455F4C494748545300534F46545728
:100340004152455F504F574552004255494C445F1A
:1003500050455243454E54004C4556454C494E4736
:100360005F44415441005A5F50524F42450041554D
:10037000544F4C4556454C005052494E545F4A4FDD
:10038000420050524F4752455353004155544F522B
:1003900045504F52545F54454D5000564F4C554DAB
:1003A000455452494300454550524F4D0053455224
:1003B00049414C5F584F4E5F584F464600464952A0
:1003C0004D574152455F4E414D453A4D61726C6902
:1003D0006E20312E312E39202847697468756229C4
:1003E00020534F555243455F434F44455F55524C50
:1003F0003A68747470733A2F2F6769746875622E47
:10040000636F6D2F4D61726C696E4669726D7761B5
:1004100072652F4D61726C696E2050524F544F437C
:100420004F4C5F56455253494F4E3A312E30204D76
:10043000414348494E455F545950453A456E6465BD
:100440007220332050726F20455854525544455203
:100450005F434F554E543A3120555549443A6365F0
:100460006465326132662D343161322D343734386F
:100470002D396231322D6335356336326633363786
:1004800066660A002F2F20004D31343520533C6919
:100490006E6465783E206F7574206F662072616EA1
:1004A00067652028302D31290A0020540020520091
:1004B000416363656C65726174696F6E3A205000C8
:1004C000486F6D65202573257325732066697273E7
:1004D00074002066697273740A005A00590058004B
:1004E000486F6D6520004F66667365747320617098
:1004F000706C696564004572723A20546F6F2066B3
:1005000061722100546F6F206661722066726F6D98
:10051000207265666572656E636520706F696E74C2
:100520000A00205A00205900580020204D61783AD6
:100530002000205A00205900580020204D696E3AB2
:1005400020004F6E20004F666600536F6674206572
:100550006E6473746F70733A200020466C6F773A44
:10056000200000010F150E12FFFFFFFF16170E13DC
:10057000FFFFFFFF03021A14FFFFFFFFFFFFFF0C47
:1005800004FFFFFF01000EFFFFFF0C190DFF1820F5
:10059000643A0020693A0020703A00496E76616C36
:1005A00069642065787472756465720A0043290A6B
:1005B0000061626C656420286D696E2074656D70E1
:1005C0002000436F6C6420657874727564657320D5
:1005D000617265200023646566696E652044454646
:1005E00041554C545F4B64200023646566696E6519
:1005F0002044454641554C545F4B692000236465B7
:1006000066696E652044454641554C545F4B7020E9
:1006100000504944204175746F74756E6520666999
:100620006E69736865642120507574207468652054
:100630006C617374204B702C204B6920616E6420B8
:100640004B6420636F6E7374616E74732066726F97
:100650006D2062656C6F7720696E746F20436F6EDA
:1006600066696775726174696F6E2E680A00504919
:1006700044204175746F74756E65206661696C65A0
:1006800064212074696D656F75740A0045312054CA
:100690004845524D414C2052554E41574159005406
:1006A0006865726D616C2052756E61776179004585
:1006B000312048656174696E67206661696C6564A4
:1006C0000048656174696E67206661696C656400E5
:1006D000504944204175746F74756E652066616978
:1006E0006C6564212054656D706572617475726506
:1006F00020746F6F20686967680A00204B643A2095
:1007000000204B693A2000204B703A20000A204319
:100710006C617373696320504944200A002054754A
:100720003A2000204B753A2000206D61783A200075
:10073000206D696E3A200020643A200020626961D1
:10074000733A2000504944204175746F74756E658A
:10075000206661696C65642120426164206578745B
:100760007275646572206E756D6265720A0050491B
:1007700044204175746F74756E6520737461727472
:100780000A004E6F2063617365206C696768740AA4
:10079000004163746976652045787472756465728A
:1007A0003A2000496E76616C6964206578747275D0
:1007B0006465720A00506C656173652072657365CB
:1007C00074005052494E5445522048414C544544BF
:1007D000005072696E7465722068616C7465642E75
:1007E000206B696C6C28292063616C6C6564210A3C
:1007F00000656E7175657565696E67202200000081
:10080000000000000000000000000000484200005E
:10081000484200008040000000005761726E696E1F
:10082000673A20486F6D696E672042756D7020448D
:10083000697669736F72203C20310A00020204005D
:1008400000A0400000A0400000004000005C430009
:10085000005C4300007A43FFFFFF7C3C3E5E2B3D83
:100860003F2F5B5D3B2C2A225C000000210024000E
:1008700027002A0024F4D43050C38E20C2A240178F
:10088000828B7011127A910D816CD90AA861E108EE
:10089000C7586607615143061E4B5D05C145A70455
:1008A0001A411104093D9803713931034036DB02C6
:1008B00065339102D4305402802E1D02632CEE0168
:1008C000752AC501B028A001102781018F25640178
:1008D0002B244B01E0223401AC211F018D200D019E
:1008E000801FFC00841EED00971DDF00B81CD200A5
:1008F000E61BC600201BBC00641AB200B219A80097
:100900000A19A0006A189900D117910040178B00AE
:10091000B516840031167E00B31579003A157300C0
:10092000C7146F0058146A00EE1366008813630042
:1009300025135E00C7125B006C125700151254009D
:10094000C111510070114F0021114B00D610490008
:100950008D1047004610440002104200C00F4000B6
:10096000800F3E00420F3C00060F3B00CB0E3800CC
:10097000930E37005C0E3500270E3400F30D320065
:10098000C10D3100900D3000600D2E00320D2D0094
:10099000050D2C00D90C2B00AE0C2900850C29006C
:1009A0005C0C2700350C27000E0C2600E80B2400F9
:1009B000C40B2400A00B23007D0B23005A0B210045
:1009C000390B2100180B2000F80A1F00D90A1E005D
:1009D000BB0A1E009D0A1D00800A1D00630A1C0040
:1009E000470A1B002C0A1B00110A1A00F7091A00FB
:1009F000DD091900C4091900AB0919009209170093
:100A00007B091800630917004C0916003609160007
:100A1000200916000A091500F5081500E008140061
:100A2000CC081400B8081400A4081400900813009F
:100A30007D0812006B0813005808120046081200C7
:100A400034081100230811001208110001081100D8
:100A5000F0071000E0071000D0071000C0071000DA
:100A6000B0070F00A107100091070E0083070F00C9
:100A700074070F0065070E0057070E0049070E00A8
:100A80003B070D002E070E0020070D0013070D0079
:100A900006070D00F9060C00ED060D00E0060C003F
:100AA000D4060C00C8060C00BC060C00B0060C00F6
:100AB000A4060B0099060C008D060B0082060B00A5
:100AC00077060B006C060B0061060A0057060B0048
:100AD0004C060A0042060A0038060A002E060A00E2
:100AE00024060A001A060A001006090007060A0072
:100AF000FD050900F4050900EB050900E205090000
:100B0000D9050900D0050900C7050900BE0509007F
:100B1000B5050800AD050800A50509009C050800FD
:100B2000940508008C050800840508007C05080071
:100B3000740508006C050700650508005D050700E1
:100B4000560508004E050700470507004005080048
:100B500038050700310507002A05070023050700AF
:100B60001C050600160507000F050700080506000E
:100B700002050700FB040600F5040700EE0406006A
:100B8000E8040600E2040700DB040600D5040600C2
:100B9000CF040600C9040600C3040600BD04060015
:100BA000B7040600B1040500AC040600A604060064
:100BB000A00405009B0406009504050090040600AF
:100BC0008A04050085040500800406007A040500F7
:100BD00075040500700405006B040500660405003B
:100BE000610405005C04050057040500520405007B
:100BF0004D04050048040500430405003E040400BC
:100C00003A04050035040500300404002C040500F6
:100C100027040400230405001E0404001A04040031
:100C200016040500110404000D0404000904050065
:100C30000404040000040400FC030400F80304009E
:100C4000F4030400F0030400EC030400E8030400D0
:100C5000E4030400E0030400DC030400D803040000
:100C6000D4030400D0030400CC030400C803030031
:100C7000C503030024F404D9201BC40C5C0E9804A3
:100C8000C4095F0265077101F405F900FB04B300B4
:100C900048048700C1036900580355000303450059
:100CA000BE023A008402310053022A0029022500C4
:100CB00004022000E4011C00C8011900AF01170064
:100CC00098011400840113007101100061011000EB
:100CD00051010E0043010D0036010B002B010B00EA
:100CE00020010B00150109000C0109000301080097
:100CF000FB000800F3000800EB000700E40006001A
:100D0000DE000600D8000600D2000600CC00050078
:100D1000C7000500C2000500BD000400B9000400C2
:100D2000B5000400B1000400AD000400A9000400F7
:100D3000A5000300A20003009F0004009B00030025
:100D40009800030095000200930003009000030048
:100D50008D0002008B000300880002008600020064
:100D600084000300810002007F0002007D00020079
:100D70007B0002007900020077000100760002008B
:100D80007400020072000100710002006F00020096
:100D90006D0001006C0002006A00010069000200A1
:100DA00067000100660001006500010064000200A8
:100DB0006200010061000100600001005F000200AC
:100DC0005D0001005C0001005B0001005A000100B1
:100DD00059000100580001005700010056000100B1
:100DE00055000100540001005300000053000100B1
:100DF0005200010051000100500001004F000100AD
:100E00004E0000004E0001004D0001004C000100AA
:100E10004B0000004B0001004A00010049000100A6
:100E200048000000480001004700010046000000A3
:100E3000460001004500000045000100440001009B
:100E40004300000043000100420000004200010096
:100E50004100000041000100400001003F0000008F
:100E60003F0001003E0000003E0001003D00000088
:100E70003D0001003C0000003C0000003C0001007F
:100E80003B0000003B0001003A0000003A00010076
:100E9000390000003900010038000000380000006F
:100EA0003800010037000000370001003600000064
:100EB000360000003600010035000000350000005B
:100EC000350001003400000034000000340001004F
:100ED0003300000033000000330001003200000046
:100EE000320000003200010031000000310000003B
:100EF000310001003000000030000000300001002F
:100F00002F0000002F0000002F0000002F00010024
:100F10002E0000002E0000002E0001002D00000019
:100F20002D0000002D0000002D0001002C0000000D
:100F30002C0000002C0000002C0001002B00000001
:100F40002B0000002B0000002B0001002A000000F5
:100F50002A0000002A0000002A00010029000000E9
:100F600029000000290000002900000029000100DC
:100F700028000000280000002800000028000000D1
:100F800028000100270000002700000027000000C3
:100F900027000000270001002600000026000000B6
:100FA00026000000260000002600010025000000A9
:100FB000250000002500000025000000250000009D
:100FC000250001002400000024000000240000008F
:100FD0002400000024000100230000002300000082
:100FE0002300000023000000230000002300000075
:100FF0002300010022000000220000002200000067
:101000002200000022000000220001002100000058
:10101000210000002100000021000000210000004C
:10102000210000002100010020000000200000003D
:101030002000000020000000200000002000000030
:1010400020000000200001001F0000001F00000021
:101050001F0000001F0000001F0000001F00000014
:101060001F0001001E0000001E0000001E00000006
:101070001E000000043700001E290000511B000064
:101080005810000010090000CC0400007802000095
:101090004101000000060900FE0701920321207FA4
:1010A000FF07FF07FF000000060000010707060218
:1010B0000080808080800080030202060105A0A0DD
:1010C0000507070600005050F850F8505005070774
:1010D0000600002078A07028F02005070706000011
:1010E000C0C810204098180507070600006090A0AF
:1010F00040A89068020303060104C040800307076C
:101100000601002040808080402003070706010080
:101110008040202020408005050506000120A870A1
:10112000A8200505050600012020F8202002030361
:101130000602FFC04080050101060003F80202021A
:10114000060200C0C0050505060001081020408009
:1011500005070706000070888888888870030707DD
:1011600006010040C040404040E00507070600007F
:10117000708808708080F8050707060000F81020C6
:10118000100808F005070706000010305090F8100E
:1011900010050707060000F880F0080888700507AA
:1011A00007060000708080F0888870050707060039
:1011B00000F808102020202005070706000070888E
:1011C000887088887005070706000070888878088E
:1011D0000870020505060200C0C000C0C002060675
:1011E0000602FFC0C000C0408004070706000010D0
:1011F000204080402010050303060002F800F80498
:1012000007070601008040201020408005070706E0
:1012100000007088081020002005070706000070F5
:10122000880868A8A870050707060000708888F875
:10123000888888050707060000F08888F08888F00D
:101240000507070600007088808080887005070702
:10125000060000F08888888888F0050707060000E7
:10126000F88080F08080F8050707060000F880808D
:10127000F0808080050707060000708880B88888A5
:1012800070050707060000888888F88888880107A5
:1012900007060200808080808080800507070600A6
:1012A00000381010101090600507070600008890A5
:1012B000A0C0A0908805070706000080808080807D
:1012C00080F805070706000088D8A8888888880560
:1012D00007070600008888C8A898888805070706B9
:1012E000000070888888888870050707060000F06D
:1012F0008888F0808080050707060000708888884D
:10130000A89068050707060000F08888F0A090887C
:10131000050707060000788080700808F0050707B9
:10132000060000F8202020202020050707060000E6
:10133000888888888888700507070600008888885C
:10134000888850200507070600008888888888A8B4
:101350005005070706000088885020508888050738
:10136000070600008888885020202005070706000F
:1013700000F80810204080F8030707060100E0800D
:1013800080808080E005050506000180402010086F
:10139000030707060100E02020202020E0050303CA
:1013A000060004205088050101060000F802020230
:1013B000060205804005050506000070087888785B
:1013C0000507070600008080B0C88888F00505057D
:1013D0000600007080808870050707060000080876
:1013E00068988888780505050600007088F8807080
:1013F0000507070600003048E0404040400506066B
:101400000600FF70888878087005070706000080CE
:1014100080B0C888888801070706020080008080A5
:101420008080800308080601FF200020202020A0E3
:1014300040040707060000808090A0C0A09003072A
:1014400007060100C04040404040E0050505060099
:1014500000D0A8A8A8A8050505060000B0C888887F
:101460008805050506000070888888700506060650
:1014700000FFF08888F080800506060600FF788867
:1014800088780808050505060000B0C8808080053A
:10149000050506000070807008F0040707060000CC
:1014A0004040E0404040300505050600008888883F
:1014B0009868050505060000888888502005050500
:1014C0000600008888A8A850050505060000885079
:1014D0002050880506060600FF8888887808700571
:1014E0000505060000F8102040F803070706010074
:1014F0002040408040402001070706020080808095
:101500008080808003070706010080404020404023
:101510008005020206000268900000000600002517
:10152000753A2530327500253032753A25303275DE
:101530000025756420253032753A2530327500203B
:101540002020202020005A00590020202020005870
:101550000009200000000000000000000000000062
:10156000003FFFF00000000000000000000000004D
:1015700000380070000000000000000000000000C3
:101580000030FC30000000000000000000000000FF
:101590000020FC100000000000000000000000001F
:1015A0000020781000000000000000000000000093
:1015B00000203010000000000000000000000000CB
:1015C000002C00D0F80180000C1FE00000082080F3
:1015D000002E31D048008000123FF000000410407F
:1015E000002F7BD043C38CD0023FF000000410409A
:1015F000002F7BD071249267CC3FF0000008208040
:10160000002E31D041249E40021FE0000010410016
:10161000002C00D049249040121FE00000208200DE
:1016200000203010FBB3CEE00C3FF0000020820021
:101630000020781000000000003FF0000010410082
:101640000020FC1000000000003FF0000008208097
:101650000030FC3000000000000FC000000000005F
:1016600000380070000000000007800000FFFFC08D
:10167000003FFFF0000000000003000000FFFFC07B
:10168000000000000000000000000000000000005A
:10169000003FFFF00000000000000000000000001C
:1016A0000038007000000000000000000000000092
:1016B0000033873000000000000000000000000040
:1016C00000278790000000000000000000000000DC
:1016D000002F87D000000000000000000000000084
:1016E000002F87D000000000000000000000000074
:1016F000002F03D0F80180000C1FE00000082080BC
:101700000020301048008000123FF000000410401C
:101710000020781043C38CD0023FF000000410403A
:101720000020781071249267CC3FF00000082080E0
:101730000020301041249E40021FE00000104100B4
:10174000002F03D049249040121FE00000208200A7
:10175000002F87D0FBB3CEE00C3FF00000208200CA
:10176000002F87D000000000003FF0000010410073
:101770000027879000000000003FF0000008208054
:101780000033873000000000000FC00000000000A0
:1017900000380070000000000007800000FFFFC05C
:1017A000003FFFF0000000000003000000FFFFC04A
:1017B0000000000000060900FE0000000000010912
:1017C0000008FE000005080806000040F0C88888F0
:1017D000987810050808060000C0F888888888886E
:1017E000F80505050600012030F830200508080638
:1017F00000002070F820202020E00509090600FFE5
:101800002070A8A8B8888870200509090600FFE0A4
:1018100080C0B0A8283028280509090600FFF8A8CC
:101820008888888888A8F8050A0A0600FE20505093
:10183000505088A8A8887003030306000340A04006
:1018400000002200250028002B00000020002300BB
:101850002600290002020202020202020404040419
:10186000040404040303030303030303010101014C
:101870000101010101020408102040800102040856
:101880001020408001020408102040808040201079
:1018900008040201000000010200090A0000000023
:1018A0000403080700000000000000000000000022
:1018B00000000000024B494C4C45442E2000202DD6
:1018C00020496E76616C6964206578747275646510
:1018D00072206E756D62657220210A00FFFFFFFFA6
:1018E000EFFFFFFFFFFFFFFFFFFFFFEFEFFFFFFF38
:1018F000FFFFFFFFFFFFE7DFFFFFFFFFFFFFFFFF30
:10190000FFE7DFFFFFFFFFFFFFFFFFFFE3DFFFFF5B
:10191000FFFFFFFFFFFFFFF3CFFFFFFFFFFFFFFF13
:10192000FFE1E1CFFFFFFFFFFFFFFE78000003DDD7
:10193000FFFFFFFFFEFF807E0001EEFFFFFFFFFEC7
:101940007DCFFC0000F77FFFFFFFFF8E0600000049
:101950007BBFFFFFFFFFC0000000007DDFFFFFFF38
:10196000FFFC01FE00003EE7FFFFFFFFFFFFFC0062
:10197000031F73FFFFFFFFFFFFF800018F81FFFFD1
:10198000FFFFFFFFE0000083F9FFFFFFFFFFFF0005
:10199000FC0000F0FFFFFFFFFFE00FFFC00000FFB3
:1019A000FFFFFFFE03FFFFC00000FFFFFFFFFFFF81
:1019B000FFF9000000FFFFFFFFFFFFFFFC0007C073
:1019C000FFFFFFFFFFFFFFFF0007E0FFFFFFFFFF3D
:1019D000FFFFFFE007F1FFFFFFFFFFFFFFFFFC0737
:1019E000F9FFFFFFFFFFFFFFFFFF03F9FFFFFFFF0F
:1019F000FFFFFFFFFF83F9FFFFFFFFFFFFFFFFFF79
:101A0000C3FFFFFFFFFFFFFFFFFFFFE1FFFFFFFF40
:101A1000FFFFFFFFFFFFF0BFFFFFFFFFFFFFFFFF25
:101A2000FBF83FFFFFFFFFFFFFFFFFF9F83FFFFF5E
:101A3000FFFFFFFFFFFF7EF0FFFFFFFFFFFFFFFF46
:101A4000FF8E03FFFFFFFFFFFFFFFFFFE01FFFFF12
:101A5000FFFFFFFFFFFFFFFFFFFFFFFFFFFFFFFF96
:101A6000FFFFFFFFFFFFFFFFFFFFFFFFFFFFFF7F06
:101A7000FFFFFFFF00007FFFFFF87FFFFFFFFF80FA
:101A8000007FFFFFE07FFFFFFFFFC3FCFFFFFFF8CA
:101A9000FFFFFFFFFFC3FCFFFFFFF8FFFFFFFFFF9C
:101AA00087FDFFFFFFF1FFFFFFFFFF87FFFFFFFF46
:101AB000F1FFFFFFFFFF0FE7F30FFC23FC3FFFFFEA
:101AC000FF0FEF8007F003F01E007FFE1FCF81871E
:101AD000C787C70C007FFE001FC7C78FC79F0F0CAB
:101AE000FFFE001F878F1F8F1F0F1FFFFC3F9F8F61
:101AF0008F1F8E001E3FFFFC7F3F0F1E3F1E3FFECD
:101B00003FFFF87FFF1F1C3F1C7FFC7FFFF8FFFF9C
:101B10001E1C7E1C7FFC7FFFF0FFCE3E3C7E3C7F88
:101B2000B8FFFFF0FF9E3C387C387E78FFFFE1FF76
:101B30003C7C787C783CF1FFFFE1F838787810182D
:101B400001F1FFFF000060203C007C07807FFFFF69
:101B5000FFFFFFFE1FFE1FFFFFFF1FFFFFFFFFFF37
:101B6000FF600000000001FF400000000000FF8057
:101B700000000000007F83CF00000C303F87FF8013
:101B8000000C301F867980000C000F8C30C7838CCE
:101B900030E78C30CFC7CC31F38C30DCECEC33B990
:101BA0008C30D86C6C33198C30D06C0C33198C3071
:101BB000D86C0C33198C30DC6C0E3B198C30CF7C1C
:101BC000079F198C30C77C038F194000000000006C
:101BD00002600000000000061FFFFFFFFFFFF8206B
:101BE00020506C616E6E65724275666665724279F0
:101BF0007465733A20002046726565204D656D6FEF
:101C000072793A2000436F6D70696C65643A204ABE
:101C1000616E20323820323031390A00207C204178
:101C20007574686F723A20287468697369736B659C
:101C3000697468622C20456E646572332050726F3F
:101C4000290A00323031382D30382D303100204C07
:101C500061737420557064617465643A2000312E9C
:101C6000312E390A004D61726C696E0020536F6627
:101C700074776172652052657365740A002057613C
:101C8000746368646F672052657365740A0020424C
:101C9000726F776E206F75742052657365740A00D9
:101CA0002045787465726E616C2052657365740AA4
:101CB00000506F77657255700A0073746172740A10
:101CC000006175746F25692E67006572726F7220EE
:101CD00077726974696E6720746F2066696C650A33
:101CE00000456E6473746F70732025632025632034
:101CF000256320256300205A3A0020593A002058D5
:101D00003A00656E6473746F7073206869743A206A
:101D100000446F6E6520736176696E672066696C3A
:101D2000652E0A004D3239004573746570732F6D4E
:101D30006D004573746570732F6D6D005A73746513
:101D400070732F6D6D005A73746570732F6D6D0015
:101D50005973746570732F6D6D005973746570736A
:101D60002F6D6D005873746570732F6D6D0058730F
:101D7000746570732F6D6D004D6F74696F6E0053D5
:101D8000746570732F6D6D004A65726B00416363FB
:101D9000656C65726174696F6E0056656C6F63691E
:101DA000747900436F6E74726F6C0046696C2E20FC
:101DB0004469612E0046696C2E204469612E004FF3
:101DC0006666004F6E20004520696E206D6D330001
:101DD000436F6E74726F6C0043616E6E6F7420653A
:101DE0006E746572207375626469723A2000022E07
:101DF0002E000152656672657368004D61696E0060
:101E00004D61782054656D703A20313235004D694E
:101E10006E2054656D703A203500544265643A4531
:101E200050434F53203130304B004D617820546582
:101E30006D703A20323735004D696E2054656D70F3
:101E40003A20350054303A204550434F532031302A
:101E5000304B005053553A2047656E6572696300F8
:101E600050726F746F636F6C3A20312E3000426194
:101E700075643A20313135323030004D656C7A6905
:101E80002028437265616C69747929004578747201
:101E900075646572733A203100687474703A2F2F3C
:101EA0006D61726C696E66772E6F726700456E6445
:101EB000657220332050726F00323031382D303847
:101EC0002D303100312E312E39004D61726C696E2A
:101ED00000546865726D6973746F727300426F614C
:101EE000726420496E666F005072696E746572206C
:101EF000496E666F004D61696E0070012C019001A2
:101F00002701B0012201C0011D01F00118011002DA
:101F1000130130020E016002090190020401C002A7
:101F2000FF000003FA004003F5008003F000D00337
:101F3000EB002004E6007004E100E004DC00400552
:101F4000D700C005D2004006CD00D006C8008007EB
:101F5000C3003008BE00F008B900C009B400B00AE0
:101F6000AF00B00BAA00D00CA500000EA000500FCF
:101F70009B00C01096005012910000148C00C015F8
:101F80008700B0178200B0197D00D01B7800001EBA
:101F9000730040206E0090226900F0246400402706
:101FA0005F0090295A00E02B5500102E5000203081
:101FB0004B0010324600E033410090353C001037B2
:101FC000370070383200A0392D00B03A2800A03B0D
:101FD0002300603C1E00103D1900903D1400103E8F
:101FE0000F00703E0A00C03E0500003F0000403F69
:101FF000FBFF803FF6FFC03FF1FF45312045727285
:102000003A204D415854454D50004572723A204D8A
:10201000415854454D5020424544004D4158544587
:102020004D502074726967676572656400453120A0
:102030004572723A204D494E54454D5000457272DA
:102040003A204D494E54454D5020424544004D499B
:102050004E54454D5020747269676765726564001F
:102060004D383420582059205A204500202F002078
:1020700042403A0020403A0057726974696E672006
:10208000746F2066696C653A20006F70656E20661B
:1020900061696C65642C2046696C653A20006F703C
:1020A000656E206661696C65642C2046696C653AD2
:1020B000200046696C652073656C65637465640A0D
:1020C000002053697A653A200046696C65206F707C
:1020D000656E65643A20002066696C653A2000648C
:1020E0006F696E67006672657368004E6F772000D7
:1020F000454E4420535542524F5554494E450A00CF
:102100002220706F73002220706172656E743A2213
:1021100000535542524F5554494E452043414C4C73
:10212000207461726765743A22004B494C4C4544F7
:102130002E2000747279696E6720746F2063616C61
:102140006C207375622D67636F64652066696C65CA
:1021500073207769746820746F6F206D616E7920C9
:102160006C6576656C732E204D4158206C657665E4
:102170006C2069733A004572726F723A0043616E67
:102180006E6F74206F70656E207375626469722063
:10219000006563686F3A006F70656E206661696CF8
:1021A00065642C2046696C653A2000496E69746943
:1021B000616C697A6520454550524F4D00436F6E02
:1021C00074726F6C00526573746F7265206661691A
:1021D0006C73616665004C6F61642073657474692B
:1021E0006E677300496E697469616C697A65204530
:1021F0004550524F4D0053746F726520736574746F
:10220000696E67730046696C616D656E74004D6F31
:1022100074696F6E0054656D706572617475726576
:10222000004D61696E004D33303320553120452516
:1022300069205325690050726568656174204142C8
:102240005320636F6E66005072656865617420503C
:102250004C4120636F6E6600504944204175746F95
:1022600074756E6500504944204175746F74756EC5
:1022700065005049442D44005049442D44005049C4
:10228000442D49005049442D49005049442D5000E7
:102290005049442D500020082046616374002008F6
:1022A0002046616374002008204D617800200820DA
:1022B0004D6178002008204D6178002008204D698C
:1022C0006E002008204D696E002008204D696E00C8
:1022D0004F6666004F6E20004175746F74656D70B7
:1022E0000046616E2073706565640046616E207300
:1022F000706565640042656400426564004E6F7AF3
:102300007A6C65004E6F7A7A6C6500436F6E7472FA
:102310006F6C0053746F72652073657474696E67B7
:10232000730042656400426564004E6F7A7A6C65A2
:10233000004E6F7A7A6C650046616E207370656539
:10234000640046616E2073706565640054656D704D
:1023500065726174757265004E6F20436865636BCA
:1023600073756D2077697468206C696E65206E7571
:102370006D6265722C204C617374204C696E653AF5
:1023800020004B494C4C45442E200053544F505094
:1023900045442E20005072696E7465722073746F0C
:1023A000707065642064756520746F206572726F4B
:1023B00072732E2046697820746865206572726F8A
:1023C0007220616E6420757365204D39393920742F
:1023D0006F20726573746172742E202854656D705D
:1023E00065726174757265206973207265736574B6
:1023F0002E205365742069742061667465722072A2
:10240000657374617274696E67290A004E6F2043A8
:102410006865636B73756D2077697468206C696E8D
:1024200065206E756D6265722C204C617374204C52
:10243000696E653A2000636865636B73756D206D26
:1024400069736D617463682C204C617374204C69EE
:102450006E653A20004C696E65204E756D6265723E
:10246000206973206E6F74204C617374204C696E08
:1024700065204E756D6265722B312C204C61737432
:10248000204C696E653A20004D313130004D3331BA
:102490000053442072656164206572726F720A0095
:1024A000446F6E65207072696E74696E672066692C
:1024B0006C650A005072656865617420504C41205B
:1024C000456E64005072656865617420504C41200F
:1024D000426564005072656865617420504C41002B
:1024E0005072657061726500507265686561742034
:1024F00041425320456E64005072656865617420E6
:1025000041425320426564005072656865617420E1
:102510004142530050726570617265004D3432382B
:10252000005072656865617420504C4100436F6FC4
:102530006C646F776E00507265686561742041420B
:10254000530044697361626C6520737465707065D3
:102550007273004D38340053657420686F6D6520C8
:102560006F666673657473004175746F20686F6D74
:102570006500473238004D6F7665206178697300D9
:102580004D61696E004D6F76652058004D6F766520
:102590002059004D6F7665205A0045787472756435
:1025A0006572004D6F766520302E316D6D004D6F78
:1025B000766520316D6D004D6F76652031306D6D23
:1025C000004D6F7665206178697300457874727587
:1025D000646572004D6F7665205A004D6F766520F8
:1025E00059004D6F766520580045787472756465A2
:1025F00072004D6F7665205A004D6F766520590048
:102600004D6F7665205800507265706172650045A7
:102610004550524F4D206461746173697A6520653D
:1026200072726F722E0A00290A0020627974657333
:102630003B20637263200053657474696E67732076
:1026400053746F726564202800290A00206279742F
:1026500065733B2063726320002073746F7265643E
:102660002073657474696E6773207265747269652E
:10267000766564202800202863616C63756C617442
:10268000656429210A0020213D2000454550524F14
:102690004D20435243206D69736D61746368202D32
:1026A000202873746F7265642920002053697A654D
:1026B0003A2000496E6465783A2000204D61726CC2
:1026C000696E3D563535290A0028454550524F4D13
:1026D0003D00454550524F4D2076657273696F6ECF
:1026E000206D69736D61746368200020746F6F20C2
:1026F0006C6F6E6720657874727573696F6E207089
:10270000726576656E7465640A0020636F6C642080
:10271000657874727573696F6E2070726576656E18
:102720007465640A0020496E76616C69642065787E
:1027300074727564657220000000000000000000E3
:102740000000000000005C4300005C4300007A438E
:10275000436C69636B20746F20726573756D652EB1
:102760002E2E0050726F7465637465642050696E1C
:102770000A0020573A004520436F6F6C696E672E40
:102780002E2E00452048656174696E672E2E2E003E
:10279000456E64657220332050726F204F66662E3E
:1027A00000205A3A0020593A0020436F756E742079
:1027B000583A0020453A00205A3A0020593A005829
:1027C0003A003A004361703A00454550524F4D205F
:1027D0004F4B0A0048617264636F6465642044650E
:1027E0006661756C742053657474696E6773204CF0
:1027F0006F616465640A00F4010000F40100006484
:10280000000000881300000000FA430000FA4300B3
:1028100000A0400000C8410000A0420000A042000B
:1028200000C8430000BA4220286D6D2900204400F2
:1028300020490020204D33303120500050494420A1
:1028400073657474696E67733A0A0020460020420B
:102850000020480020204D3134352053004D617454
:10286000657269616C206865617475702070617251
:10287000616D65746572733A0A00205A0020590030
:1028800020204D323036205800486F6D65206F662D
:10289000667365743A0A00204500205A00205900EA
:1028A00020580020540020530020204D3230352085
:1028B000510020453C6D61785F655F6A65726B3ED3
:1028C0000020583C6D61785F785F6A65726B3E20CE
:1028D000593C6D61785F795F6A65726B3E205A3C46
:1028E0006D61785F7A5F6A65726B3E004164766104
:1028F0006E6365643A20513C6D696E5F7365676D08
:10290000656E745F74696D655F75733E20533C6DD1
:10291000696E5F66656564726174653E20543C6DE6
:10292000696E5F74726176656C5F6665656472611D
:1029300074653E0020540020520020204D32303477
:10294000205000416363656C65726174696F6E202D
:1029500028756E6974732F7332293A20503C707257
:10296000696E745F616363656C3E20523C7265748E
:10297000726163745F616363656C3E20543C747282
:102980006176656C5F616363656C3E0A002045009B
:10299000205A0020590020204D3230312058004D5F
:1029A0006178696D756D20416363656C65726174F2
:1029B000696F6E2028756E6974732F7332293A0A15
:1029C00000204500205A0020590020204D3230338D
:1029D0002058004D6178696D756D2066656564727B
:1029E000617465732028756E6974732F73293A0AB0
:1029F00000204500205A0020590020204D39322067
:102A0000580053746570732070657220756E697418
:102A10003A0A0020204D3230302044300A00202075
:102A20004D3230302044002044697361626C65642B
:102A30000A0046696C616D656E7420736574746913
:102A40006E67733A0020204D3134392043203B20FB
:102A5000556E69747320696E2043656C7369757374
:102A60000A002020473231202020203B00486F6D93
:102A7000696E67206661696C656400545249474716
:102A800045524544006F70656E003A20007A5F6DD4
:102A9000696E00795F6D696E00785F6D696E0052D6
:102AA00065706F7274696E6720656E6473746F70A1
:102AB000207374617475730A005654726176206DC8
:102AC000696E005654726176206D696E00565472BC
:102AD0006176206D696E00566D696E00566D696E87
:102AE00000566D696E00566D6178204500566D6127
:102AF00078204500566D6178204500566D6178203C
:102B00005A00566D6178205A00566D6178205A003F
:102B1000566D6178205900566D6178205900566DC8
:102B20006178205900566D6178205800566D6178A3
:102B3000205800566D61782058004D6F74696F6E93
:102B400000416D6178204500416D6178204500416C
:102B50006D6178205A00416D6178205A00416D61A5
:102B600078205900416D6178205900416D617820CD
:102B70005800416D6178205800412D74726176656E
:102B80006C00412D74726176656C00412D72657424
:102B90007261637400412D726574726163740041E7
:102BA0006363656C00416363656C004D6F74696FAE
:102BB0006E0056652D6A65726B0056652D6A6572EA
:102BC0006B0056652D6A65726B00567A2D6A6572C8
:102BD0006B00567A2D6A65726B0056792D6A6572A4
:102BE0006B0056792D6A65726B0056792D6A657295
:102BF0006B0056782D6A65726B0056782D6A657287
:102C00006B0056782D6A65726B004D6F74696F6E3C
:102C1000004D3234004D323320257300556E6B6EFB
:102C20006F776E20636F6D6D616E643A2022005382
:102C3000442063617264206F6B0A006F70656E528E
:102C40006F6F74206661696C65640A00766F6C75DD
:102C50006D652E696E6974206661696C65640A0031
:102C6000534420696E6974206661696C0A00456E80
:102C700064657220332050726F2052656164792E32
:102C8000005072696E74696E672E2E2E0050726944
:102C90006E7420706175736564005072696E742083
:102CA00061626F7274656400496E69742E205344CA
:102CB0002063617264004D3231004E6F2053442016
:102CC00063617264004368616E67652053442063EA
:102CD000617264004D3231005072696E7420667208
:102CE0006F6D2053440053746F70207072696E745E
:102CF00000526573756D65207072696E7400416273
:102D00006F7574205072696E7465720050617573CE
:102D100065207072696E7400436F6E74726F6C0020
:102D2000507265706172650054756E6500496E661B
:102D30006F2073637265656E0042616279737465BA
:102D400070205A004261627973746570205A00469F
:102D50006C6F7700466C6F770046616E207370650C
:102D600065640046616E2073706565640042656449
:102D700000426564004E6F7A7A6C65004E6F7A7A15
:102D80006C65005370656564005370656564004D43
:102D900061696E004572726F722077726974696E34
:102DA0006720746F20454550524F4D210A006265DF
:102DB000640A002C2073797374656D2073746F70CE
:102DC00070656421204865617465725F49443A20EA
:102DD000004265642068656174696E672066616998
:102DE0006C65640048656174696E67206661696C32
:102DF00065640045312048656174696E67206661CD
:102E0000696C65640048656174696E672066616914
:102E10006C656400453120544845524D414C205268
:102E2000554E415741590042454420544845524D62
:102E3000414C2052554E4157415900546865726DBE
:102E4000616C2052756E6177617900526573656EB1
:102E5000643A20006F6B00627573793A2070617577
:102E600073656420666F7220696E7075740A006203
:102E70007573793A2070617573656420666F72208E
:102E8000757365720A00627573793A2070726F63A8
:102E9000657373696E670A004B494C4C45442E209C
:102EA000004B494C4C206361757365642062792046
:102EB000746F6F206D75636820696E6163746976E5
:102EC000652074696D65202D2063757272656E745E
:102ED00020636F6D6D616E643A200000ACDDE6D753
:102EE00011241FBECFEFD0E4DEBFCDBF12E0A0E0C3
:102EF000B1E0E4EAFBED01E00BBF02C007900D92E8
:102F0000AC35B107D9F723E1ACE5B2E001C01D92C1
:102F1000AA32B207E1F717E1CFE6D7E104C0219763
:102F2000FE010E9430EDCE36D107C9F70E9468D865
:102F30000C94C5ED0C9400002F923F924F925F923B
:102F40006F927F928F929F92AF92BF92CF92DF92B9
:102F5000EF92FF920F931F93CF93DF93CDB7DEB71E
:102F6000C958D1090FB6F894DEBF0FBECDBF21E01E
:102F700020930E1380917F128D3409F484C7843519
:102F800011F40C944130873411F00C948530809109
:102F90007D1290917E128430910509F45DC544F450
:102FA00097FD6DC72091500182309105DCF415C06A
:102FB0008A35910509F45BC724F44C9709F48AC556
:102FC0005EC78B35910509F456C78C35910509F01C
:102FD00056C70E94EBAB0C94873021110C948C30B7
:102FE0000C948730222311F40C94873011E002975F
:102FF00009F010E00E94B2A982E50E94EF828823C6
:1030000009F436C10E9475826B017C01409068030F
:103010005090690360906A0370906B0380916C0319
:1030200090916D03A0916E03B0916F038CA79DA743
:10303000AEA7BFA720917302309174024091750230
:103040005091760228AB39AB4AAB5BAB80917702EB
:1030500090917802A0917902B0917A028CAB9DABED
:10306000AEABBFAB20E030E0A901C701B6010E94C2
:10307000ABE5882309F4D6C4A301920168A979A914
:103080008AA99BA90E94ABE581110DC02CA53DA585
:103090004EA55FA56CA97DA98EA99FA90E94ABE54D
:1030A000882309F4BFC420E030E0A901C701B601BC
:1030B0000E94ABE5881F8827881F18130BC020E0EB
:1030C00030E040E85FE328962CAF3DAF4EAF5FAFF6
:1030D00028970AC080E090E0A0E8BFEB28968CAF6C
:1030E0009DAFAEAFBFAF2897A301920168A979A9A0
:1030F0008AA99BA90E94DBE96CAF7DAF8EAF9FAF21
:103100002CA53DA54EA55FA56CA97DA98EA99FA95B
:103110000E94DBE924966CAF7DAF8EAF9FAF249702
:103120002CAD3DAD4EAD5FADCA01B9010E9411E6B7
:103130004B015C0124962CAD3DAD4EAD5FAD2497A7
:10314000CA01B9010E9411E69B01AC01C501B4019D
:103150000E94DCE90E948AEC68AF79AF8AAF9BAF2E
:1031600020E030E040E05FE30E9411E64B015C01AB
:10317000A7019601C701B6010E9411E66B017C010F
:10318000A5019401C501B4010E9411E69B01AC01A7
:10319000C701B6010E94DBE90E948AEC9B01AC01E9
:1031A00028966CAD7DAD8EAD9FAD28970E9411E63F
:1031B0004B015C0128A939A94AA95BA9C301B20145
:1031C0000E94DCE920E030E040E05FE30E9411E68D
:1031D0006B017C0124966CAD7DAD8EAD9FAD2497C7
:1031E000905828AD39AD4AAD5BAD0E94D6EA9B013F
:1031F000AC01C501B4010E9411E69B01AC01C701FD
:10320000B6010E94DCE9A30192010E94DBE96B0197
:103210007C012CA93DA94EA95FA96CA57DA58EA511
:103220009FA50E94DCE920E030E040E05FE30E94DF
:1032300011E62B013C0128AD39AD4AAD5BAD6CAD5B
:103240007DAD8EAD9FAD0E94D6EA9B01AC01C5015C
:10325000B4010E9411E69B01AC01C301B2010E94BE
:10326000DCE92CA53DA54EA55FA50E94DBE914C0B5
:1032700089E40E94EF82882329F00E9475826B0105
:103280007C0103C0C12CD12C76018AE40E94EF821C
:103290008823D9F00E9475826CAB7DAB8EAB9FAB5F
:1032A00020E030E0A901C701B6010E94ABE5811121
:1032B0001AC020E030E0A9016CA97DA98EA99FA9C0
:1032C0000E94ABE581110FC0ADC320E030E0A90141
:1032D000C701B6010E94ABE5882309F4A3C31CAA69
:1032E0001DAA1EAA1FAAA701960150582CA73DA7E8
:1032F0004EA75FA78CA99DA9AEA9BFA9B05888AB5E
:1033000099ABAAABBBABCA01B9010E9411E64B0154
:103310005C0128A939A94AA95BA9CA01B9010E947F
:1033200011E69B01AC01C501B4010E94DCE90E94D9
:103330008AEC64966CAF7DAF8EAF9FAF649720919F
:1033400068033091690340916A0350916B0328AF81
:1033500039AF4AAF5BAFA701960168AD79AD8AADD1
:103360009BAD0E94DCE928966CAF7DAF8EAF9FAF1E
:10337000289780916C0390916D03A0916E03B0919A
:103380006F038CAF9DAFAEAFBFAF2CA93DA94EA9C7
:103390005FA9BC01CD010E94DCE968966CAF7DAFEE
:1033A0008EAF9FAF68972091730230917402409165
:1033B00075025091760224962CAF3DAF4EAF5FAFB1
:1033C000249728962CAD3DAD4EAD5FAD2897249641
:1033D0006CAD7DAD8EAD9FAD24970E94DBE96B0196
:1033E0007C018091770290917802A0917902B0914E
:1033F0007A022C968CAF9DAFAEAFBFAF2C9768967C
:103400002CAD3DAD4EAD5FAD6897BC01CD010E94C6
:10341000DBE94B015C012091700330917103409115
:1034200072035091730360962CAF3DAF4EAF5FAF08
:10343000609760917B0270917C0280917D029091F7
:103440007E020E94DBE92B013C0180917F0290917A
:103450008002A0918102B0918202A0968CAF9DAFB4
:10346000AEAFBFAFA0972091740330917503409128
:103470007603509177036C962CAF3DAF4EAF5FAFA4
:103480006C97A70196016CA57DA58EA59FA50E94AE
:1034900011E6A4966CAF7DAF8EAF9FAFA497A50148
:1034A000940168A979A98AA99BA90E9411E69B01A8
:1034B000AC01A4966CAD7DAD8EAD9FADA4970E947E
:1034C000DCE9A4966CAF7DAF8EAF9FAFA497A5014A
:1034D00094016CA57DA58EA59FA50E9411E64B01C8
:1034E0005C01A701960168A979A98AA99BA90E94F4
:1034F00011E69B01AC01C501B4010E94DBE9A49671
:103500002CAD3DAD4EAD5FADA4970E945BEA6B0163
:103510007C0120E030E0A9010E94ABE587FF0AC0F2
:103520002BED3FE049EC50E4C701B6010E94DCE915
:103530006B017C01112351F02BED3FE049EC50E48D
:10354000C701B6010E94DBE96B017C0120E030E09D
:10355000A901C701B6010E94ABE5811124C02496E0
:103560002CAD3DAD4EAD5FAD249768AD79AD8AAD64
:103570009BAD0E94ABE5811116C02C962CAD3DADE4
:103580004EAD5FAD2C976CAD7DAD8EAD9FAD0E9405
:10359000ABE5811108C0BBEDCB2EBFE0DB2EB9EC53
:1035A000EB2EB0E4FB2EA701960164966CAD7DADC9
:1035B0008EAD9FAD64970E9411E64B015C0120E047
:1035C00030E0A901C301B2010E94ABE58823C9F034
:1035D000A5019401C501B4010E9411E64B015C01F3
:1035E000A3019201C301B2010E9411E69B01AC014B
:1035F000C501B4010E94DCE90E948AEC4B015C0128
:103600000DC020E030E0A901C501B4010E943CECEE
:1036100087FF04C0B7FAB094B7F8B0942FE632E150
:1036200043E85AE3C501B4010E94ABE587FF02C03D
:103630000C948730C501B4010E947EEB0E944FEBD1
:103640001B01672B19F422242394312CB10180E053
:1036500090E00E94B0E54B015C019B01AC01C70109
:10366000B6010E94D6EA68AF79AF8AAF9BAFA501D9
:103670009401C301B2010E94D6EA64966CAF7DAF9B
:103680008EAF9FAF64976C962CAD3DAD4EAD5FADE8
:103690006C97A0966CAD7DAD8EAD9FADA0970E944E
:1036A000DBE9A50194010E94D6EAA0966CAF7DAF3C
:1036B0008EAF9FAFA09728AD39AD4AAD5BADCA01C3
:1036C000B9010E9411E620E030E040E05FE30E9493
:1036D00011E69B01AC0160E070E080E89FE30E948E
:1036E000DBE92C966CAF7DAF8EAF9FAF2C976096C9
:1036F0008CAD9DADAEADBFAD609789879A87AB8726
:10370000BC876C962CAD3DAD4EAD5FAD6C972D87F3
:103710003E874F87588B60914E0170914F01072E65
:10372000000C880B990B0E94B2E5209100013091AA
:10373000010140910201509103010E9411E62AE02B
:1037400037ED43E25CE30E9411E668A779A78AA7F8
:103750009BA70E9418409B01AC0128533F4F4F4F3D
:103760005F4F60962CAF3DAF4EAF5FAF60974CA4FC
:103770005DA46EA47FA441E050E022965FAF4EAFFF
:10378000229759E15CAF22962EAD3FAD22972215CC
:10379000330509F41CC10E945AD10E941840DC0173
:1037A000CB0160962CAD3DAD4EAD5FAD6097821BF9
:1037B000930BA40BB50BB7FD10C00E9418409B01E2
:1037C000AC0128533F4F4F4F5F4F60962CAF3DAF3A
:1037D0004EAF5FAF60970E9414D33CAD31503CAF09
:1037E000332309F441C02C962CAD3DAD4EAD5FADF9
:1037F0002C9768A979A98AA99BA90E9411E66B0157
:103800007C0128AD39AD4AAD5BADB201C3010E9468
:1038100011E6A70196010E94DCE97B018C012C9640
:103820002CAD3DAD4EAD5FAD2C97B201C3010E94F2
:1038300011E64B015C0128AD39AD4AAD5BAD68A91D
:1038400079A98AA99BA90E9411E69B01AC01C50137
:10385000B4010E94DBE92B013C01C701D80188AB10
:1038600099ABAAABBBAB53C022964EAD5FAD2297CE
:10387000BA0180E090E00E94B0E528AD39AD4AADD4
:103880005BAD0E9411E64B015C010E94D1EA6B0125
:103890007C01C501B4010E947CEC4B015C01A701D5
:1038A00096016CA57DA58EA59FA50E9411E62B0112
:1038B0003C01A50194016CA97DA98EA99FA90E9434
:1038C00011E69B01AC01C301B2010E94DCE92B01AE
:1038D0003C01A50194016CA57DA58EA59FA50E9424
:1038E00011E64B015C01A70196016CA97DA98EA987
:1038F0009FA90E9411E69B01AC01C501B4010E9481
:10390000DBE968AB79AB8AAB9BAB59E15CAF920169
:10391000A30128966CAD7DAD8EAD9FAD28970E941A
:10392000DCE969837A838B839C8328A939A94AA916
:103930005BA968966CAD7DAD8EAD9FAD68970E941A
:10394000DCE96D837E838F83988764962CAD3DADD3
:103950004EAD5FAD649769857A858B859C850E94A5
:10396000DCE969877A878B879C87A0962CAD3DAD73
:103970004EAD5FADA0976D857E858F8598890E943D
:10398000DCE96D877E878F87988B80914101882342
:1039900021F0CE0101960E944F3CE090D60218A281
:1039A00019A21AA21BA2CE0180966C018E01085D9D
:1039B0001F4F9E01235F3F4FAE01475F5F4FBE0128
:1039C0006B5F7F4F4F970E94F997811121C0E09064
:1039D000D6021CA21DA21EA21FA2DE0194966D019A
:1039E0008E01085D1F4F2FE732E04BE752E067E79B
:1039F00072E083E792E00E94F99780E1E3E7F2E06A
:103A0000A8E6B3E001900D928A95E1F70C94873017
:103A10002296EEADFFAD229731962296FFAFEEAF24
:103A20002297B1CEE6E7F1E284918F010F5F1F4F3D
:103A3000882321F00E940283F801F6CFEBE9F1E040
:103A400084918F010F5F1F4F882311F40C948730EE
:103A50000E940283F801F4CF80E50E94EF82882360
:103A600029F00E9431826B017C0103C0C12CD12C52
:103A7000760183E50E94EF82882361F00E947582BF
:103A800020E030E04AE754E40E9411E60E944FEB48
:103A90006B017C010E94D5508091270C811105C0DB
:103AA00060E081EB91E00E94F3580E941840C60E3E
:103AB000D71EE81EF91E0E941840DC01CB018C19AC
:103AC0009D09AE09BF09B7FD02C00C9487300E9462
:103AD00014D3F1CF80915B038770873071F48FE44A
:103AE0000E94EF82882319F00E94658203C08FE450
:103AF0000E94A88281110C9487300E94D550809139
:103B0000000190910101A0910201B0910301809305
:103B1000630290936402A0936502B0936602809161
:103B20004E0190914F01909362028093610284E66E
:103B300090E090934F0180934E0111E010935A034F
:103B400088E50E94A8828CAB89E50E94A882282E75
:103B50008AE50E94A88288AF3CA9311105C02110D6
:103B600005C0382E312605C0211002C0312C01C0FD
:103B700038AC80E1E8E6F3E0A3E7B2E001900D9213
:103B80008A95E1F782E50E94EF82882369F00E941E
:103B900075824B015C0120E030E0A9010E94ABE599
:103BA000882309F440C006C0812C912CF0EAAF2E86
:103BB000F0E4BF2E311006C04CA9411103C02220F1
:103BC00009F42AC180927B0290927C02A0927D022D
:103BD000B0927E0220917003309171034091720384
:103BE00050917303C501B4010E943CEC1816DCF43B
:103BF00019821A821B821C8220916C0330916D0302
:103C000040916E0350916F03609168037091690356
:103C100080916A0390916B03DE0111966D0185011D
:103C200074010E94CCAA31100EC0BCA9B11103C00E
:103C30002110EDC0F1C0211006C080E00E94E13CDF
:103C40003320B1F3E4C010926C0310926D03109214
:103C50006E0310926F031092680310926903109222
:103C60006A0310926B030E942782E7E5F8E0249133
:103C700021962FAF2197EBE4F8E085909590A590E1
:103C8000B490EFE4F8E0C590D590E590F490A701EA
:103C90009601C501B4010E943CEC18162CF4A50154
:103CA0009401C701B60104C0A7019601C501B40182
:103CB0000E94D6EA2B013C01EEE0F8E08591959157
:103CC000A591B4918CA79DA7AEA7BFA7EAE0F8E0A5
:103CD000259135914591549128AB39AB4AAB5BABFB
:103CE0009C01AD0168A979A98AA99BA90E94ABE5AD
:103CF00087FD07C01CA50DA53EA53CAF4FA54CA751
:103D000006C018A909A95AA95CAF8BA98CA7A30161
:103D10009201C301B2010E9411E620E030E040E8C8
:103D20005FE30E94DCE90E948AEC9B01AC01612FF9
:103D3000702F8CAD9CA50E9411E669837A838B83DA
:103D40009C83E8E5F8E014912091700330917103B1
:103D500040917203509173032CA73DA74EA75FA714
:103D600020E030E040EC5FE3C701B6010E9411E6BD
:103D70006B017C01612F110F770B880B990B0E944F
:103D8000B2E59B01AC01C701B6010E9411E62B010F
:103D90003C0120E030E040EC5FE3C501B4010E944B
:103DA00011E66B017C0121963FAD2197632F330F04
:103DB000770B880B990B0E94B2E59B01AC01C70100
:103DC000B6010E9411E6AE014F5F5F4F6A01ECA49D
:103DD000FDA40EA51FA5A30192010E94CCAA0E94DA
:103DE0008AB110926C0310926D0310926E031092C0
:103DF0006F03109268031092690310926A03109285
:103E00006B0331101ACF5CA9511117CF11CF81E08C
:103E10000E94E13C311003C058AD552319F082E0F7
:103E20000E94E13C0E9427828091590380935A03AB
:103E30008091630290916402A0916502B091660244
:103E40008093000190930101A0930201B0930301BC
:103E5000809161029091620290934F0180934E0194
:103E600083E0809342010E94A7A70C9487301092B0
:103E700060020C948730209360020C9487300E947B
:103E8000B8BF0C94873080917D1290917E1282375A
:103E9000910509F465C60CF0C7C08B34910509F48F
:103EA0004AC40CF067C08831910509F4FCC1ACF537
:103EB0008231910509F4B5C5BCF497FF02C00C949A
:103EC0003E30823091050CF48EC1419711F00C9474
:103ED0003E3060E08AEB91E00E94F3585E985E9875
:103EE00015985E980C9487308531910509F4C0C10E
:103EF0003CF4449711F00C943E30E2EDF1E077C1D0
:103F00008631910509F4B8C1479711F00C943E3001
:103F1000E0917B12F0917C12B9C18D31910511F4C1
:103F20000C948730C4F48A31910509F4CBC10CF4A8
:103F3000C3C18B31910509F4D3C14C9711F00C9496
:103F40003E3040E060E080917B1290917C120E94B4
:103F50006A750C9487308F31910509F4FDC20CF419
:103F600059C28032910509F4E6C28A9709F49AC3CE
:103F70000C943E308836910509F4E9C36CF582351E
:103F8000910509F445C57CF48D34910509F4DBC332
:103F90000CF4D5C38135910511F00C943E300E948C
:103FA000C5A80C9487308435910509F43AC50CF402
:103FB00033C58535910509F438C58C35910511F067
:103FC0000C943E3036E5C32E31E0D32E43EAE42E86
:103FD00041E1F42E10E044C58D36910509F4BDC4CD
:103FE0009CF48A36910509F4F1C40CF474C48B3640
:103FF000910509F409C58C36910511F00C943E30F9
:10400000109215010C9487308F36910509F4E1C3A5
:104010000CF4CCC38037910509F429C4813791058C
:1040200009F42DC40C943E308D3D910511F40C948F
:10403000142B0CF05EC08B39910509F467C41CF594
:104040008737910509F4A7C674F48537910509F4FB
:1040500045C60CF054C68337910511F00C943E30E0
:10406000EDEBF3E0DFC58937910509F49FC60CF449
:1040700096C68C38910509F474C48139910509F408
:104080009BC60C943E308C3C910509F48FC7F4F428
:10409000883C910509F40AC734F48E3B910509F474
:1040A0007EC40C943E30893C910509F447C78B3C93
:1040B000910511F00C943E30EBE9EE2EECE0FE2E73
:1040C00006E511E0F4E0DF2ED00E61C78E3C9105CD
:1040D00009F484C514F40C944E28833D910511F421
:1040E0000C94272A8C3D910511F40C94072B0C9409
:1040F0003E308A39A1E09A0709F4BDC394F58D32A8
:10410000E1E09E0711F40C94DF2B9CF4823221E055
:10411000920711F40C94AB2B8C3231E0930711F41D
:104120000C94B62B823E910511F00C943E300C9409
:10413000822B8F3241E0940711F40C94D42C14F4A8
:104140000C94802C8336A1E09A0711F40C941C3057
:104150008039914011F00C943E300E94D5500C945F
:104160008730873FE1E09E0711F40C943B30ECF47C
:10417000843F21E0920711F40C9435303CF48C3AE2
:10418000914011F40C94BB280C943E30853F51E0D3
:10419000950711F40C943830863F914011F00C943F
:1041A0003E300E9453B50C9487308B38B3E09B07A8
:1041B00011F40C9487304CF4883F914011F00C942A
:1041C0003E300E94FAA60C948730803A23E0920792
:1041D00009F4B5C1873E934011F00C943E300E9423
:1041E000E5A60C9487300E9428A90C94873084910E
:1041F0008F010F5F1F4F882321F00E940283F80177
:10420000F6CF1092560940E050E0BA0189E097E0FD
:104210000E9437CA8BE1E9E0F7E0DE0115960190D4
:104220000D928A95E1F780910707909108079C838A
:104230008B838CE891E09A83898340E050E0BE0153
:104240006F5F7F4F80E090E00E943F73CE01019648
:104250000E94E43DE3ECF1E084918F010F5F1F4F7A
:10426000882311F40C9487300E940283F801F4CF64
:104270000E94EABD0C9487301092B2061092B306E9
:104280000C948730803209F410823196808181113C
:10429000F9CF40E061E080917B1290917C120E9406
:1042A0006A750C9487308091B30681112093B20611
:1042B0000E9479CF0C9487301092B2060E94B3CF3F
:1042C0000C9487308091B306882311F40C948730C6
:1042D00083E50E94EF8281110C947E310C9487302B
:1042E00083E40E94A882882309F454C0E0E1F2E04C
:1042F00084918F010F5F1F4F882321F00E9402835A
:10430000F801F6CF8091A408882391F0BE016F5F79
:104310007F4F81EA98E00E94A1358E010F5F1F4F09
:10432000D8018D918D01882381F10E940283F8CFFD
:10433000E3EEF1E084918F010F5F1F4F882329F195
:104340000E940283F801F6CF8091A211882309F41C
:1043500081C27EE8C72E72E0D72EE12CF12C20E03E
:104360008091A21190E00E2C02C0959587950A9439
:10437000E2F780FD57C2FFEFEF1AFF0A32E0C30EEB
:10438000D11C45E0E416F10459F78AE00E9402834B
:104390000C9487308091B306882371F18091B20626
:1043A000882351F1EDEEF1E084918F010F5F1F4FF3
:1043B000882321F00E940283F801F6CF6091520910
:1043C0007091530980915409909155094AE00E94D7
:1043D000AA858FE20E94028360914E0970914F0975
:1043E00080915009909151094AE00E94AA858AE083
:1043F0000E9402830C948730EFEFF1E084918F01EB
:104400000F5F1F4F882311F40C9487300E940283A2
:10441000F801F4CF8091B306882311F40C9487300F
:1044200081EA98E00E9404CA81EA98E00E947C3503
:104430001092B1061092B00600917B1210917C127E
:104440008091B306882311F40C9487300E94567231
:10445000B801CE0180960E949E718C01892B11F4C7
:104460000C94873068A179A16115710511F06C5F1A
:104470007F4F19821C8222E0A801CE0101960E9482
:104480005D3B811102C0F12C14C0CE0101960E9447
:104490000C718823C1F361E0CE0101960E9485353D
:1044A000009789F325EEFC0120831C820E94A9C796
:1044B000F82ECE0101960E94FC82FF2011F1EFE15F
:1044C000F2E084917F012FEFE21AF20A882321F0B3
:1044D0000E940283F701F5CFD8018D918D018823C9
:1044E00019F00E940283F8CF8AE00E9402831092A2
:1044F00052091092530910925409109255090C94C4
:104500008730EDE2F2E084917F01BFEFEB1AFB0A06
:10451000882321F00E940283F701F5CFF8018191F1
:104520008F01882319F00E940283F8CF8EE20E9447
:1045300002830C9487300E94E7A80C948730809106
:104540007B1290917C1221E02093B10640E060E064
:104550000E946A750C9487300E9445CFECE3CE2E02
:10456000D12CE12CF12CA70196010E949FE9762E17
:10457000672ECA01B901A70196010E949FE96B014C
:104580007C01CA01B90128E130E040E050E00E941E
:104590009FE94B015C01C9016DE671E00E94E9EC05
:1045A0008E010F5F1F4F6115710599F06F927F9219
:1045B000DF92CF929F928F929F938F937F936F936F
:1045C0008DE692E09F938F931F930F930E9442E595
:1045D00012C00097B1F06F927F92DF92CF929F92BC
:1045E0008F929F938F938DE592E09F938F931F936C
:1045F0000F930E9442E50FB6F894DEBF0FBECDBF09
:1046000036C081149104A104B10479F06F927F92B5
:10461000DF92CF929F928F9281E592E09F938F934A
:104620001F930F930E9442E5E6CFC114D104E10429
:10463000F10469F06F927F92DF92CF9289E492E069
:104640009F938F931F930F930E9442E5D4CF6F9255
:104650007F9285E492E09F938F931F930F930E9424
:1046600042E50F900F900F900F900F900F9060E029
:10467000C8010E942F59E1E9F1E284917F01BFEF67
:10468000EB1AFB0A882321F00E940283F701F5CF81
:10469000B80181E892E00E94B64F8AE00E9402834E
:1046A0000C94873083E50E94EF82882311F40C94E8
:1046B00087300E945182E82E80E50E94EF82882395
:1046C00011F40C9487300E945182182F87FF02C08A
:1046D0000C94873089E40E94EF82882349F00E947D
:1046E0006582811111C0E2E6F5E08DE28E0F07C010
:1046F00089E40E94A882F5CF31968E1729F0949113
:104700001913FACF0C94363361E0812F0E94303FA9
:104710006E2D812F0E945164F12CB701812F0E94D0
:104720006C3F143011F00C948730F092CC0CE09276
:10473000CB0C0C9487300E9479CF0C9487300E9468
:10474000B3CF0C9487300E94C8CF0C94873088E692
:1047500090E00E94C9AC81110C9487308091A21125
:1047600083FF02C00C94873083E50E94EF82882388
:10477000C9F00E9475820E9448EB7093E511609326
:10478000E41180E00E943DCE0E94758220E030E07E
:104790004AEA52E40E94ABE5181624F00E94C8CF02
:1047A0000E9411C40E94DD4F0C9487308EE40E9459
:1047B000EF82882311F40C9487300E944182609329
:1047C00025067093260680932706909328060C945E
:1047D000873083E50E94A882882359F083E50E94F0
:1047E000EF82882319F00E94518201C080E08093FB
:1047F000A211E1E9F1E284918F010F5F1F4F88233D
:1048000021F00E940283F801F6CFECE9F2E08491F6
:104810008F010F5F1F4F882309F496CD0E940283FA
:10482000F801F5CFBB24B394B20E222319F08CE229
:104830000E940283F60125913491F9018491890146
:104840000F5F1F4F882321F00E9402839801F5CF4C
:104850002B2D91CDE8E9F2E084918F010F5F1F4F7E
:10486000882309F492CD0E940283F801F5CF83EAF0
:1048700092E00E94EC3D0E9429A70C94873083E5CA
:104880000E94EF82882369F00E9451828D3320F4C8
:10489000809351010C9487308CE3809351010C94E8
:1048A0008730E1E9F1E284918F010F5F1F4F882388
:1048B00021F00E940283F801F6CF4091510150E0AF
:1048C00060E070E08CEA92E00E94634F8AE00E9410
:1048D00002830C94873089E690E00E94C9AC811174
:1048E00011C0E3EBF2E084918F010F5F1F4F88232B
:1048F00021F00E940283F801F6CF0E94026F8AE045
:104900000E94028310920E130C940F3583E50E94CF
:10491000EF82882311F40C9487300E945182182F63
:104920008D3308F01CE310931B130E9418406B0199
:104930007C01212F30E0A8EEB3E00E94CCE9C60E46
:10494000D71EE81EF91EC0921713D0921813E092DA
:104950001913F0921A130C9487300E940BAD0C942B
:1049600087308091A21183FF02C00C94873083E5C9
:104970000E94EF82882311F40C9487300E94758284
:104980000E9448EB6D37710514F06DE770E070938D
:10499000E3116093E2110E94F2CD0C948730809174
:1049A000A21183FF02C00C94873083E50E94EF823E
:1049B00025968FAF259781110C948F3182E50E9447
:1049C000EF8281110C948F310C94873080E50E9426
:1049D000EF82811106C083E50E94EF82882361F097
:1049E00006C00E94518281110C948730F4CF0E943E
:1049F00041826F3F710510F06FEF70E07093CC0C47
:104A00006093CB0C0C9487300E94D8A80C9487300C
:104A100010925F020C94873081E080935F020C94C7
:104A200087300E9472A80C94873083E50E94A88288
:104A3000882311F40C9487300E94758220E030E0C6
:104A40004AE754E40E9411E60E944FEB609313136F
:104A50007093141380931513909316130C9487304E
:104A6000D6018D916D010E94A882882309F46DC042
:104A7000133009F063C00E9475824B015C0120E095
:104A800030E040EA51E40E94ABE587FF4EC0A5014B
:104A900094016091AF117091B0118091B11190911A
:104AA000B2110E94D6EA2B013C019B01AC0160913E
:104AB000770C7091780C8091790C90917A0C0E940F
:104AC00011E66093770C7093780C8093790C909337
:104AD0007A0CA30192016091A70C7091A80C8091AF
:104AE000A90C9091AA0C0E9411E66093A70C7093F8
:104AF000A80C8093A90C9093AA0C6091870C7091DC
:104B0000880C8091890C90918A0C0E94B0E5A301D9
:104B100092010E9411E60E944FEB6093870C709304
:104B2000880C8093890C90938A0C8092AF1190929C
:104B3000B011A092B111B092B21107C00E9475825B
:104B4000F70160837183828393831F5FF4E0EF0E2C
:104B5000F11C143009F084CF0E94C0510C948730AE
:104B60000E94D55083E50E94EF82882309F456C045
:104B70000E9441826230710509F050C00E94D9D56F
:104B80008BE50E9402836091021370910313809160
:104B900004139091051342E00E942E864091061363
:104BA0005091071360910813709109138BED92E0F7
:104BB0000E94804F40910A1350910B1360910C1387
:104BC00070910D1388ED92E00E94804F8DE50E9458
:104BD00002838AE00E9402830C94873066E5C62E29
:104BE00061E0D62E7CE5E72E73E0F72E10E0D601CB
:104BF0008D916D010E94A882882351F00E947582D8
:104C0000F7016083718382839383812F0E94ABAB12
:104C10001F5FF4E0EF0EF11C133049F70E94A7A7C5
:104C20000C94873084918F010F5F1F4F882321F0F0
:104C30000E940283F801F6CF60E08DEA93E00E94C3
:104C400063A761E086EA93E00E9463A761E08BE9D5
:104C500093E00E9463A761E08BE893E00E9463A762
:104C600060E082E893E00E9463A761E088E793E058
:104C70000E9463A760E08EE693E00E9463A760E075
:104C800086E693E00E9463A760E088E593E00E94D7
:104C900063A760E08AE493E00E9463A760E08BE38F
:104CA00093E00E9463A760E08DE293E00E9463A717
:104CB00060E087E193E00E9463A760E086E093E014
:104CC0000E9463A760E081EF92E00E9463A761E029
:104CD0008EED92E00E9463A70C94873080917B1246
:104CE00090917C12DC012C91211104C00E9411C40E
:104CF0000C94873060E00E942F590C94873000910B
:104D00007B1210917C1283E0D12C40E08150E1F0C5
:104D1000F8019081292F2B7F2134C1F72181213384
:104D2000A9F7913421F0953421F441E002C0DD244B
:104D3000D39498012E5F3F4F89012F5F3F4FD801D9
:104D40009C919032C9F3E2CF442369F0E1E9F1E2AA
:104D500084917F01BFEFEB1AFB0A882321F00E94A8
:104D60000283F701F5CFDD2069F0E4E8F4E08491F7
:104D70007F012FEFE21AF20A882321F00E940283BA
:104D8000F701F5CFD8018D918D01882309F4FDCA73
:104D90000E940283F7CF0E9461B10C94873081E0BA
:104DA00080935A03809359030C94873010925A03CE
:104DB000109259030C94873083E50E94EF82882378
:104DC00019F00E94418202C060E070E08B0111275F
:104DD00002301105D4F0E6E7F1E284918F010F5F14
:104DE0001F4F882321F00E940283F801F6CFE8E8E4
:104DF000F4E084918F010F5F1F4F882311F40C940E
:104E000087300E940283F801F4CF88E40E94EF8289
:104E10008823A9F00E9441826A3A71053CF065300E
:104E2000B1E07B072CF064E071E002C06AEA70E058
:104E3000F801EE0FFF1FE259F64F7183608386E49D
:104E40000E94EF828823A9F00E944182F801EE0FB0
:104E5000FF1FEE58F64F718360836F3F710519F0A5
:104E600014F06FEF70E077FF02C060E070E07183D4
:104E7000608382E40E94EF82882311F40C948730CF
:104E80000E9441826530710534F06F3671052CF057
:104E90006EE670E002C065E070E0000F111FF801DF
:104EA000E659F64F718360830C94873088EC90E06C
:104EB0000E94C9AC81110C94873084E40E94A882BE
:104EC0008823C1F10E94758211E020E030E0A90141
:104ED0000E94ABE5811101C010E01093060511237B
:104EE00049F10E947582E091120524E0E29FF001F1
:104EF0001124EE5FFA4F608371838283938320E0F5
:104F000030E0A901609102057091030580910405CC
:104F1000909105050E94ABE581110CC080E090E006
:104F2000A0EEBFE38093020590930305A0930405D0
:104F3000B09305050E948B470C948730ABEBEA2EAB
:104F4000A1E1FA2E06E511E0B4E0DB2ED00ED80187
:104F50008D918D010E94A882882349F00E9475825C
:104F60000E944FEBF7016083718382839383F4E0A7
:104F7000EF0EF11CD012EBCF0E940D500C94873035
:104F8000F4E0EF0EF11CD01611F40C948730D80128
:104F90008D918D010E94A882882391F30E947582D1
:104FA000F7016083718382839383EACF83E50E9454
:104FB000EF828823A1F00E9475826093930C709316
:104FC000940C8093950C9093960C60938F0C709337
:104FD000900C8093910C9093920C10E001C011E022
:104FE00080E50E94EF82882359F00E9475826093C9
:104FF000930C7093940C8093950C9093960C10E006
:1050000082E50E94EF82882359F00E9475826093A6
:10501000970C7093980C8093990C90939A0C10E0D5
:1050200084E50E94EF82882361F00E94758260937C
:105030008F0C7093900C8093910C9093920C0C9425
:105040008730112311F40C9487304091930C5091C8
:10505000940C6091950C7091960C80EB94E00E94FA
:10506000804F4091970C5091980C6091990C7091E1
:105070009A0C8DEA94E00E94804F40918F0C5091E1
:10508000900C6091910C7091920C8AEA94E00E94CD
:10509000804F8AE00E9402830C94873081E50E9451
:1050A000A882882351F00E9431826093AF0C7093E4
:1050B000B00C8093B10C9093B20C83E50E94A8824F
:1050C000882351F00E9475826093C70C7093C80CBE
:1050D0008093C90C9093CA0C84E50E94A88288230F
:1050E00051F00E9475826093C30C7093C40C80933E
:1050F000C50C9093C60C88E50E94A882882351F0C5
:105100000E94758260936B0C70936C0C80936D0C95
:1051100090936E0C89E50E94A882882351F00E942A
:10512000758260936F0C7093700C8093710C9093E8
:10513000720C8AE50E94A882882351F00E94758231
:105140006093730C7093740C8093750C9093760C31
:1051500085E40E94A882882311F40C9487300E9471
:1051600075826093770C7093780C8093790C909390
:105170007A0C0C9487308091F902082F017011E0AD
:10518000012781FBFF24F0F8F12682FB882780F9B4
:105190001827011102C0FF2019F0E1E9F1E215C062
:1051A0001111FBCF5EEF852E57E0952E28E633E0F8
:1051B0003DA72CA7AE014F5F5F4F5A0107E518E0EE
:1051C0001A0153E0500F58AB7BC084916F012FEF51
:1051D000C21AD20A882321F00E940283F601F5CF79
:1051E000E0EEF4E084916F013FEFC31AD30A882305
:1051F00021F00E940283F601F5CF002369F0EEED65
:10520000F4E084916F014FEFC41AD40A882321F08F
:105210000E940283F601F5CFFF2069F0ECEDF4E087
:1052200084916F015FEFC51AD50A882321F00E948F
:105230000283F601F5CF111103C0E2EDF4E00DC0D9
:10524000EAEDF4E084916F019FEFC91AD90A88232F
:10525000A1F30E940283F601F5CF84916F01AFEFB5
:10526000CA1ADA0A882321F00E940283F601F5CFD8
:10527000111103C048E452E002C040E252E0F110D4
:1052800003C028E432E002C022E232E0011103C090
:1052900088E492E002C084E292E05F934F933F93F0
:1052A0002F939F938F9380EC94E09F938F931F9203
:1052B0000E943EA50FB6F894DEBF0FBECDBF27C734
:1052C000F4016591759185919491ACA5BDA5CD90A2
:1052D000DD90ED90FD90BDA7ACA7A70196010E94BF
:1052E000DBE92B013C0120E030E040EA51EC0E9478
:1052F0003CEC87FD10C020E030E040EA51E4C301FF
:10530000B2010E94ABE5181634F0F10140825182DF
:10531000628273820EC0F80184911816B4F7F7FA0E
:10532000F094F7F8F094D101CD92DD92ED92FC92D9
:105330001397D101CD90DD90ED90FD901D0120E0FF
:1053400030E040EA51ECC701B6010E943CEC87FF17
:1053500003C0E6E7F1E20BC020E030E040EA51E4B0
:10536000C701B6010E94ABE5181674F5F2CF84911F
:105370008F010F5F1F4F882321F00E940283F801E5
:10538000F6CFE4E0F5E084918F010F5F1F4F882393
:1053900021F00E940283F801F6CF61E086EF94E0ED
:1053A0000E94F3580E945D6388E290E099A388A36D
:1053B00088EC90E09DA38CA3BE01605E7F4FCE0180
:1053C00084960E945B77A3C6B4E08B0E911C0F5F9E
:1053D0001F4FE8A9E01374CF4CE5E42E43E0F42E10
:1053E00010E0F50181919191A191B1915F01F701D7
:1053F00081939193A193B1937F01812F0E94ABABD5
:105400001F5F133071F70E94A7A760E086EE94E05B
:105410000E94F35883E992E09DA38CA304E610E078
:1054200019A308A3BE016C5D7F4FCE0180960E9438
:105430005B778AEB92E09DA38CA319A308A3BE011E
:105440006C5D7F4FCE0180960E945B7760C6E1E97C
:10545000F1E284918F010F5F1F4F882321F00E949A
:105460000283F801F6CF83E50E94A882882321F009
:105470000E94658280934101EAE4F5E084918F0106
:105480000F5F1F4F882321F00E940283F801F6CF9F
:1054900080914101811103C0E6E4F5E002C0E2E43D
:1054A000F5E084918F010F5F1F4F882321F00E9448
:1054B0000283F801F6CFEAE3F5E084918F010F5FF4
:1054C0001F4F882321F00E940283F801F6CF20911C
:1054D000FC093091FD094091FE095091FF0960914E
:1054E000080A7091090A80910A0A90910B0A0E9499
:1054F000DCE9AB01BC0188E395E00E94804F20917C
:10550000000A3091010A4091020A5091030A609109
:105510000C0A70910D0A80910E0A90910F0A0E9458
:10552000DCE9AB01BC0185E395E00E94804F20914E
:10553000040A3091050A4091060A5091070A6091C9
:10554000100A7091110A8091120A9091130A0E9418
:10555000DCE9AB01BC0182E395E00E94804FEAE206
:10556000F5E084918F010F5F1F4F882321F00E9487
:105570000283F801F6CF2091FC093091FD0940919A
:10558000FE095091FF0960913501709136018091BB
:105590003701909138010E94DCE9AB01BC0188E23F
:1055A00095E00E94804F2091000A3091010A4091BD
:1055B000020A5091030A6091390170913A01809179
:1055C0003B0190913C010E94DCE9AB01BC0185E20A
:1055D00095E00E94804F2091040A3091050A409185
:1055E000060A5091070A60913D0170913E01809139
:1055F0003F01909140010E94DCE9AB01BC0182E2D5
:1056000095E00E94804F8AE00E94028380C583E576
:105610000E94EF82882309F47AC50E944182709328
:105620004F0160934E0173C58DED90E00E94C9ACAF
:1056300081116DC583E50E94EF828823D9F1009125
:10564000120510E00E944182000F111FF801E45B77
:10565000FE4F718360838091120590E08C01000FF2
:10566000111F000F111F98012D5B3E4F7901880F0C
:10567000991FFC01E45BFE4F60817181072E000CD5
:10568000880B990B0E94B2E52AE037ED43E25CE318
:105690000E9411E6F801E650FE4E208131814281E0
:1056A00053810E9411E6D7016D937D938D939C9356
:1056B00013972DC5E1E9F1E284918F010F5F1F4F30
:1056C000882321F00E940283F801F6CF85E40E942E
:1056D000028380911205805D0E940283E091120591
:1056E000F0E0EE0FFF1FE45BFE4F608171818AE501
:1056F00095E00E949D4F85E20E9402838AE00E940D
:10570000028305C580E50E94A882882309F4FFC4AE
:105710000E9441826B017C0183E50E94EF82882315
:1057200021F00E9441828B0102C00FEF1FEFC801E0
:105730000196039708F0EBC4D7FCE9C49C2DE2E680
:10574000F5E08DE28E0F2491921709F48FC7319600
:105750008E13F9CF8EC78AE50E94EF828111B1C7FF
:1057600083E50E94EF828111ACC7D1C483E50E941A
:10577000EF82882319F00E94418202C064E071E048
:1057800079A368A380E50E94EF82882339F00E9404
:1057900041826938B3E17B0730F402C068EE73E000
:1057A0007A83698304C088E893E19A838983BE0180
:1057B000605E7F4FCE0101960E945B77A8C485E4AE
:1057C0000E94EF82811110C080E50E94A882882388
:1057D00091F00E94758260935D0970935E098093D9
:1057E0005F099093600907C00E945182882361F38A
:1057F000E6E7F1E26EC089E40E94A882882381F086
:105800000E9475822CEA35EC47E25EE30E9411E6C5
:10581000609365097093660980936709909368099E
:1058200084E40E94A882882381F00E9475822CEA79
:1058300035EC47E25EE30E94D6EA6093610970931B
:1058400062098093630990936409E1E9F1E284912C
:105850008F010F5F1F4F882321F00E940283F80100
:10586000F6CF40915D0950915E0960915F0970919A
:10587000600987E995E00E94804F2CEA35EC47E209
:105880005EE3609165097091660980916709909166
:1058900068090E94D6EAAB01BC0183E995E00E9449
:1058A000804F2CEA35EC47E25EE36091610970912C
:1058B000620980916309909164090E9411E6AB012D
:1058C000BC018FE895E00E94804F8AE00E9402832D
:1058D0001EC484918F010F5F1F4F882321F00E9407
:1058E0000283F801F6CFEBE9F5E084918F010F5FB9
:1058F0001F4F882309F40BC40E940283F801F5CFDF
:1059000083E50E94A882182F882371F00E94758277
:105910000E9448EB709348016093470121E0672B98
:1059200009F020E02093CD0C80E50E94A882882316
:1059300059F02091470130914801232B11F00E942A
:1059400065828093CD0CE3C31111E1C3E1E9F1E27B
:1059500084918F010F5F1F4F882321F00E940283E3
:10596000F801F6CF8091CD0C811103C069E272E09D
:1059700002C066E272E082EC95E00E94B64F609150
:1059800047017091480181EB95E00E949D4FEDEA3F
:10599000F5E084918F010F5F1F4F882309F4B7C38F
:1059A0000E940283F801F5CF85E40E94EF828823EC
:1059B00021F00E9441827B0102C0E12CF12C83E4A2
:1059C0000E94EF82882331F00E944182AE966FAF31
:1059D000AE9704C025E0AE962FAFAE9785E50E9446
:1059E000EF82882319F00E94658203C085E50E943A
:1059F000A882EA968FAFEA97F7FC07C0812C912C1A
:105A0000F6E1AF2EF3E4BF2E06C0812C912CECE81A
:105A1000AE2EE2E4BE2E83E50E94EF82882321F0C1
:105A20000E9475824B015C01E114F10411F41092A3
:105A300012050E9418402B013C01EE2069F0E4E4BD
:105A4000F7E084918F010F5F1F4F882309F45FC334
:105A50000E940283F801F5CFEEE6F7E084917F0122
:105A60003FEFE31AF30A882321F00E940283F70133
:105A7000F5CFC501B4010E9448EB072E000C880B3E
:105A8000990B0E94B2E56CAB78AF8CAF21969FAFBB
:105A90002197D301C201805E914BAF4FBF4FCE57CC
:105AA000DF4F88839983AA83BB83C258D0400E946A
:105AB000DDCF8FE78093100581E080931501E59697
:105AC0004CAE5DAE6EAE7FAEE597EE964CAE5DAE83
:105AD0006EAE7FAEEE97E1961FAEE197C258DF4FF4
:105AE000188219821A821B82CE57D04065961FAE4B
:105AF000659790E429969FAF2997ACE12D96AFAFBB
:105B00002D97B6E46996BFAF699761961FAE61970E
:105B10006D961FAE6D97A1961FAEA197A5961FAE6D
:105B2000A597AD961CAE1DAE1EAE1FAEAD97A99645
:105B30001CAE1DAE1EAE1FAEA997C12CD12C760196
:105B40002FE730E040E050E028AB39AB4AAB5BAB2D
:105B50007FE7872E912CA12CB12CE9961CAE1DAEAF
:105B60001EAE1FAEE99731E0E0963FAFE097269674
:105B70001FAE1EAE269710E0212C312C00E0AE9611
:105B80004FADAE97042E000C550BAF965FAF4EAFE6
:105B9000AF9780911501882309F4FDC00E94184039
:105BA0006CA77DA78EA79FA780910F05882309F476
:105BB000D4C00E9424CF1091CE0C2090CF0C3090F6
:105BC000D00C0091D10C212F322D432D502F6196F6
:105BD0006FAD61976D967FAD6D97A1968FADA197D3
:105BE000A5969FADA5970E94ABE587FF0CC0619677
:105BF0001FAF61976D962FAE6D97A1963FAEA1979F
:105C0000A5960FAFA597212F322D432D502F6596C6
:105C10006FAD659729967FAD29972D968FAD2D97FE
:105C200069969FAD69970E943CEC181664F46596DE
:105C30001FAF659729962FAE29972D963FAE2D97CA
:105C400069960FAF6997E0965FADE0972CA938ADE4
:105C50004CAD552309F460C021965FAD2197612FAB
:105C6000722D832D902F0E943CEC18160CF075C0FD
:105C70008CA59DA5AEA5BFA584199509A609B70950
:105C8000CA57DF4F88839983AA83BB83C658D04005
:105C900088589341A109B109B7FD5FC0D501C4017E
:105CA00028A939A94AA95BA9821B930BA40BB50BA0
:105CB000B595A7959795879580931005CA57DF4F9F
:105CC00088819981AA81BB81C658D040E9968CAF62
:105CD0009DAFAEAFBFAFE9979CA961969FAF6197AB
:105CE000A8AD6D96AFAF6D97BCADA196BFAFA197B4
:105CF0002196EFAD2197A596EFAFA5972CA53DA5D1
:105D00004EA55FA5E5962CAF3DAF4EAF5FAFE597D3
:105D1000E0961FAEE09721C021965FAD2197612FDD
:105D2000722D832D902F0E94ABE587FF16C08CA5A6
:105D30009DA5AEA5BFA5E5962CAD3DAD4EAD5FAD25
:105D4000E597821B930BA40BB50BAC01BD01485822
:105D500053416109710977FFEFC420E030E040EA68
:105D600051E46CA978AD8CAD21969FAD21970E942E
:105D7000DCE99B01AC01612F722D832D902F0E94D5
:105D80003CEC18167CF4E0EDF6E084918F010F5F97
:105D90001F4F811103C00E94DDCFB9C10E94028351
:105DA000F801F3CF8CA59DA5AEA5BFA5EE962CADB1
:105DB0003DAD4EAD5FADEE97821B930BA40BB50BC3
:105DC000B7FD9DC00E94026F8AE00E9402838CA5ED
:105DD0009DA5AEA5BFA58053984FAF4FBF4FEE9680
:105DE0008CAF9DAFAEAFBFAFEE97E1969FADE197A1
:105DF000911168C0C258DF4F288139814A815B8187
:105E0000CE57D040612F722D832D902F0E943CECF5
:105E100018160CF040C020E030E040E050E4612F64
:105E2000722D832D902F0E94DCE9C258DF4F6883CA
:105E300079838A839B83CE57D0402CA53DA54EA560
:105E40005FA5205E314B4F4F5F4FCE57DF4F28830A
:105E500039834A835B83C258D04020E030E040EC75
:105E600050E46CA978AD8CAD21969FAD21970E942E
:105E7000DBE99B01AC0181E0E1968FAFE197612FF7
:105E8000722D832D902F0E943CEC1816C4F1E196E0
:105E90001FAEE19734C08CA59DA5AEA5BFA5CE577A
:105EA000DF4F288139814A815B81C258D040821BF3
:105EB000930BA40BB50BB7FD22C04FEA56E061EC83
:105EC00076E01AC020E030E040EA51E46CA978ADF9
:105ED0008CAD21969FAD21970E94DBE99B01AC011F
:105EE000612F722D832D902F0E94ABE587FF07C095
:105EF0004CE856E06FE976E080E00E9400D08CA587
:105F00009DA5AEA5BFA5880F991FAA1FBB1FE5962B
:105F10002CAD3DAD4EAD5FADE597821B930BA40B51
:105F2000B50B84199509A609B70981389F44A24188
:105F3000B10568F0EEE6F6E084918F010F5F1F4F28
:105F4000882309F428CF0E940283F801F5CF269612
:105F50004EAD5FAD2697AF968EAD9FADAF978417D0
:105F600095070CF066C0E1E1F6E084918F010F5FC8
:105F70001F4F882321F00E940283F801F6CFB7015A
:105F8000A6018DEF95E00E94804F8AE00E94028377
:105F9000A9964CAD5DAD6EAD7FADA99789EE95E04C
:105FA0000E94804F8AE00E940283AD964CAD5DADA9
:105FB0006EAD7FADAD9785ED95E00E94804F8AE094
:105FC0000E940283EA969FADEA97992309F49FC045
:105FD000C0925D09D0925E09E0925F09F09260097B
:105FE0002CEA35EC47E25EE3A9966CAD7DAD8EAD53
:105FF0009FADA9970E9411E66093650970936609A9
:1060000080936709909368092CEA35EC47E25EE3D8
:10601000AD966CAD7DAD8EAD9FADAD970E94D6EACD
:106020006093610970936209809363099093640996
:106030006EC00E945859ADCDE6E7F1E284918F0120
:106040000F5F1F4F882321F00E940283F801F6CFD3
:10605000E2E8F7E084918F010F5F1F4F882309F476
:1060600056C00E940283F801F5CF0E9467934FC08B
:106070000E9462B64CC00E941EA749C00E94B8BFD1
:1060800046C0F0907D120E94D550FF2029F1E1E931
:10609000F1E284918F010F5F1F4F882321F00E944E
:1060A0000283F801F6CF84E50E9402836F2D70E031
:1060B00080E090E04AE00E94AA8580E20E9402838C
:1060C000E3EAF7E084918F010F5F1F4F8823F9F017
:1060D0000E940283F801F6CF1092D602E1E9F1E2C4
:1060E00084918F010F5F1F4F882321F00E9402834C
:1060F000F801F6CF6091D60270E081E997E00E9446
:106100009D4F8AE00E94028302C00E94B8BF109295
:106110000E130E9416D683C40E94B2A98091410139
:10612000882321F083E792E00E944F3C8091A211E6
:1061300083FDA5C0C0907F02D0908002E0908102D4
:10614000F0908202209174033091750340917603A0
:1061500050917703C701B6010E94ABE5882309F48B
:106160008EC06091CE0C7091CF0C8091D00C90912C
:10617000D10C2091CD0C211129C00E9448EB209117
:106180004701309148016217730704F5C092740308
:10619000D0927503E0927603F0927703E1E9F1E2A1
:1061A00084918F010F5F1F4F882321F00E9402838B
:1061B000F801F6CFE0E8F1E084918F010F5F1F4F07
:1061C000882321F00E940283F801F6CF80907F029D
:1061D00090908002A0908102B0908202209174037E
:1061E000309175034091760350917703C501B40156
:1061F0000E94DBE96B017C0120E030E0A9010E94F4
:106200003CEC87FF04C0F7FAF094F7F8F094E091C3
:10621000D60224E0E29FF0011124ED5BFE4F2081C5
:10622000318142815381C701B6010E9411E620E00D
:1062300030E048E453E40E943CEC181604F58092E8
:10624000740390927503A0927603B0927703E1E90C
:10625000F1E284918F010F5F1F4F882321F00E948C
:106260000283F801F6CFE1E6F1E084918F010F5F40
:106270001F4F882321F00E940283F801F6CF60911E
:106280004E0170914F01072E000C880B990B0E9454
:10629000B2E520910001309101014091020150913D
:1062A00003010E9411E62AE037ED43E25CE30E941D
:1062B00011E669837A838B839C83E090D60218A6CB
:1062C00019A61AA61BA6AE01485D5F4F6A018E0192
:1062D0000F5F1F4F2FE732E04BE752E067E772E0B6
:1062E00083E792E00E94F99780E1E3E7F2E0A8E615
:1062F000B3E001900D928A95E1F709CF0E944182A7
:10630000AB01BC0140935209509353096093540967
:106310007093550981EA98E00E9437CAF8CE0E942E
:1063200075820E9448EB6D3771050CF09CC170932B
:10633000E3116093E2110E94F2CD0E94758220E089
:1063400030E040EA50E40E943CEC181614F40E943D
:1063500079CF6091E2117091E311072E000C880B48
:10636000990B0E94B2E52091FA023091FB02409114
:10637000FC025091FD020E943CEC18161CF08AEBC6
:1063800092E002C089EC92E060E00E94F35881E064
:10639000809315018091D6028093120518AA19AA3C
:1063A0001AAA1BAA68961CAE1DAE1EAE1FAE689739
:1063B0001CA629961FAE29975CE32D965FAF2D97FB
:1063C0008CE169968FAF699796E461969FAF61976C
:1063D000C12CD12C50E8E52E6FEBF62E812C912CA0
:1063E00054016091E2117091E311072E000C880BAB
:1063F000990B0E94B2E5162F072F782E692E262FB3
:10640000372F482F592FB601C7010E94ABE58823CB
:1064100001F12091FA023091FB024091FC0250916F
:10642000FD02612F702F872D962D0E94ABE5881FEE
:106430008827881F8CA72596AFAD2597AA2369F0DA
:10644000882359F080911501882309F460CE0C94BB
:1064500076261C2D0D2D7E2C6F2C0E9418406B0172
:106460007C01DC01CB0168962CAD3DAD4EAD5FAD3E
:106470006897821B930BA40BB50BB7FD3DC0D701EA
:10648000C60188519C4FAF4FBF4F68968CAF9DAFF0
:10649000AEAFBFAF68970E94026FE6EBF2E0849167
:1064A0002F019FEF491A590A882321F00E94028385
:1064B000F201F5CF81149104A104B104B9F0D50122
:1064C000C401805F984DAF4FBF4FBC01CD016C1927
:1064D0007D098E099F0928EE33E040E050E00E94DC
:1064E0009FE9CA01B9010E94128603C08FE30E948E
:1064F00002838AE00E9402830E9414D30E94184003
:1065000060930F13709310138093111390931213D1
:10651000A091FA02ACABB091FB02B8AFE091FC02E3
:10652000ECAFF091FD022196FFAF21979D01AF01E5
:10653000612F702F872D962D0E94DBE91B012C0106
:1065400020E030E0A9010E943CEC87FF04C057FA2C
:10655000509457F8509481149104A104B10459F453
:1065600020E030E040E85FE3C201B1010E94ABE50A
:1065700087FF0DC00AC020E030E040E450E4C201D3
:10658000B1010E943CEC181614F4460157012CA5E9
:10659000222309F44CC088A999A9AAA9BBA9892BCF
:1065A0008A2B8B2B61F0D701C60128A939A94AA9EA
:1065B0005BA9821B930BA40BB50BB7FD38C02CA9AC
:1065C00038AD4CAD21965FAD219729966FAD2997D7
:1065D0002D967FAD2D9769968FAD699761969FAD8A
:1065E00061970E94DBE920E030E040EC5FE30E942D
:1065F000ABE587FD27CFD701C601805A9541AF4F44
:10660000BF4F88AB99ABAAABBBAB9CA929969FAFF8
:106610002997A8AD2D96AFAF2D97BCAD6996BFAFAA
:1066200069972196EFAD21976196EFAF61978091C1
:106630001501882309F406CF81149104A104B10443
:1066400029F4C12ED02EE72CF62CCBCEF0E1CF1AB8
:10665000F7E2DF0AE108F108C818D908EA08FB08E0
:10666000F7FEF0CEEECF6DE770E061CE0E9462DE05
:106670004ECD0E94D550BC2C60E08C2D0E94303F46
:106680000F3FBFEF1B0759F48C2D0E94286431E0A7
:1066900020E0892B09F030E0032F122F05C00130D4
:1066A000110561F000E010E08B2D0E942864801736
:1066B000910709F42CCD0E9414D3F6CF01E010E02D
:1066C000F3CF0E94758220E030E040E050EC0E9461
:1066D000ABE587FD12C00E94758220E030E040E00B
:1066E00050E40E943CEC18161CF00E94758209C010
:1066F00060E070E080E090E404C060E070E080E082
:1067000090EC2091AB113091AC114091AD115091B2
:10671000AE11E0915B03E2FFFACC0091F811109109
:10672000F9110E9411E60E9448EB600F711F7093EF
:10673000F9116093F811EBCC26964EAD5FAD26971C
:10674000452B09F43AC1E9964CAC5DAC6EAC7FAC1C
:10675000E997480E591E6A1E7B1EE9962CAD3DAD89
:106760004EAD5FADE997281B390B4A0B5B0BCA0195
:10677000B90128A939A94AA95BA90E948FE9A301F7
:1067800092010E9411EDD501C401820F931FA41F35
:10679000B51F84319105A105B105FCF04C015D01E7
:1067A0008C3E9105A105B1052CF05BEE852E912C58
:1067B000A12CB12C40E884169104A104B104DCF0B2
:1067C0008EEF90E0A0E0B0E088199909AA09BB0912
:1067D00088AB99ABAAABBBAB12C044E1842E912C21
:1067E000A12CB12C24E130E040E050E028AB39ABE3
:1067F0004AAB5BAB04C088AA99AAAAAABBAAB501F6
:10680000A4018CE397E00E9407D848A959A96AA976
:106810007BA987E397E00E9407D865964FAD6597FF
:1068200029965FAD29972D966FAD2D9769967FAD0F
:10683000699780E397E00E94804F61964FAD619722
:106840006D965FAD6D97A1966FADA197A5967FAD43
:10685000A59789E297E00E94804F26964EAD5FADE6
:106860002697433051050CF4A8C068A979A98AA9D4
:106870009BA90E94B2E520E030E040E850E40E948D
:1068800011E66B017C0165962FAD659729963FADAA
:1068900029972D964FAD2D9769965FAD69976196B3
:1068A0006FAD61976D967FAD6D97A1968FADA197F6
:1068B000A5969FADA5970E94DBE92BED3FE049E44B
:1068C00050E40E9411E620E030E040E05FE30E94E7
:1068D00011E69B01AC01C701B6010E94D6EA6B012B
:1068E0007C01C301B2010E94B2E52FE632E143E828
:1068F0005AE30E9411E62B013C01B701A60183E295
:1069000097E00E94804FB301A2018DE197E00E94C1
:10691000804F2AE939E949E15FE3C701B6010E94E6
:1069200011E66B017C019B01AC010E94DCE9A30133
:1069300092010E94D6EAA9966CAF7DAF8EAF9FAF51
:10694000A997A3019201C701B6010E9411E620E0B8
:1069500030E040E05EE30E9411E6AD966CAF7DAFA3
:106960008EAF9FAFAD97EDE0F7E084913F015FEF11
:10697000651A750A882321F00E940283F301F5CF7E
:10698000B701A60187E097E00E94804FA9964CAD21
:106990005DAD6EAD7FADA99781E097E00E94804F1D
:1069A000AD964CAD5DAD6EAD7FADAD978BEF96E026
:1069B0000E94804F8AE00E94028388A999A9AAA90F
:1069C000BBA9880D991DAA1DBB1DB595A7959795C7
:1069D00087958093100526968EAD9FAD26970196DC
:1069E00026969FAF8EAF26979CA965969FAF659719
:1069F000A8AD2996AFAF2997BCAD2D96BFAF2D9707
:106A00002196EFAD21976996EFAF69974CA45DA4ED
:106A10006EA47FA4F1E0E096FFAFE0979EC9C75750
:106A2000DF4F0FB6F894DEBF0FBECDBFDF91CF9121
:106A30001F910F91FF90EF90DF90CF90BF90AF909C
:106A40009F908F907F906F905F904F903F902F908E
:106A500008950F931F93CF93DF93FC01238122238B
:106A600011F080E044C08B01EC01FB01878980318B
:106A700039F18032B1F783E08B83F801428D538D79
:106A8000648D758D4D8B5E8B6F8B788F9E012F5E25
:106A90003F4FC8010E9435C9882319F31A8F098F07
:106AA00081E08983188619861A861B861C821D82BE
:106AB0001E821F82188A1C861D861E861F8617C08E
:106AC00082E08B831D8A1E8A1F8A188EFB01808DAF
:106AD000918DA0E0B0E025E0880F991FAA1FBB1F91
:106AE0002A95D1F7898B9A8BAB8BBC8BD7CFDF9153
:106AF000CF911F910F910895CF93DF93EC010E94E6
:106B000004CA1B82DF91CF910895CF93DF93EC01EC
:106B100041E0611101C040E06C857D858E859F85D7
:106B20000E94E9C7882341F0888920E2829FC00142
:106B30001124855E954F02C080E090E0DF91CF91F7
:106B40000895CF93DF93EB01FC012381211102C053
:106B500080E028C02250223020F48FE288831982FE
:106B600020C060E00E948535009791F3FC0190E021
:106B700080E02EE23081303269F0883029F4DE0185
:106B8000A90FB11D2C939F5FDE01A90FB11D3081AC
:106B90003C939F5F8F5F31968B3061F7C90FD11D9A
:106BA000188281E0DF91CF9108953F924F925F92DA
:106BB0006F927F928F929F92AF92BF92CF92DF920D
:106BC000EF92FF920F931F93CF93DF93CDB7DEB772
:106BD0002C970FB6F894DEBF0FBECDBF5C01DC0171
:106BE00059968D909C905A97F40181859285A38542
:106BF000B4859C01AD012F5F3F4F4F4F5F4F2987F9
:106C00003A874B875C87D5011496CD90DD90ED9047
:106C1000FC901797C114D104E104F10439F0BFEFDF
:106C2000CB1ADB0AEB0AFB0A312C07C0F401C08047
:106C3000D180E280F38033243394260137011D8212
:106C40001E821F821886F40181859285A385B485F2
:106C50002D813E814F815885281739074A075B07E8
:106C600008F064C089859A85AB85BC858C159D0527
:106C7000AE05BF0550F482E0C82ED12CE12CF12CDA
:106C800092E0492E512C612C712C9E012F5F3F4FB9
:106C9000B701A601C4010E94B4C8882309F446C004
:106CA00089819A81AB81BC81892B8A2B8B2B41F006
:106CB000260137019FEF491A590A690A790A05C066
:106CC000C414D504E604F70491F02D813E814F8170
:106CD00058852F5F3F4F4F4F5F4F2D833E834F832C
:106CE00058873FEFC31AD30AE30AF30AACCF0FEF7A
:106CF0001FEF2FEF3FE0B301A201C4010E9422C8A1
:106D0000F82E882399F0D50114964D915D916D91DF
:106D10007C911797411551056105710549F0930163
:106D20008201C4010E9422C8811102C0F12C29C035
:106D3000D50114964D925D926D927C9217973320F7
:106D400051F0D301C2010196A11DB11DF401808350
:106D50009183A283B383F50185899689A789B08D34
:106D6000892B8A2B8B2B69F4D50155964D925D9218
:106D70006D927C92589711968C911197806811961C
:106D80008C938F2D2C960FB6F894DEBF0FBECDBF1F
:106D9000DF91CF911F910F91FF90EF90DF90CF90F7
:106DA000BF90AF909F908F907F906F905F904F902B
:106DB0003F90089561E0FC0180810C9451648EBD88
:106DC0000DB407FEFDCF08958FEF8EBD0DB407FE05
:106DD000FDCF8EB508950F931F93CF93DF938B0153
:106DE0000E941840EB010E94E4368F3F49F00E9458
:106DF00018406C1B7D0B60177107A8F380E001C081
:106E000081E0DF91CF911F910F910895CF92DF9292
:106E1000EF92FF921F93CF93DF9300D000D0CDB7B6
:106E2000DEB76C01162FFC019281892F806A86954E
:106E30008CBD90FD03C081E0963009F480E08DBDEB
:106E400060E0F601808129833A834B835C830E9452
:106E500051646CE271E0C6010E94EB36812F8064C0
:106E60000E94DF3688E1E82EF12C5C814B813A816B
:106E70002981DA01C9010E2C04C0B695A795979512
:106E800087950A94D2F729833A834B835C830E94C7
:106E9000DF36F8E0EF1AF10829813A814B815C81F5
:106EA00088EFE8168FEFF80621F7112321F018304C
:106EB00021F08FEF03C085E901C087E80E94DF362B
:106EC0001C3011F40E94E43610E00E94E436F60112
:106ED000838387FF04C01F3F11F01F5FF6CF0F9021
:106EE0000F900F900F90DF91CF911F91FF90EF9037
:106EF000DF90CF9008950F931F93CF93DF93EC0112
:106F000089018C81833039F089E0440F551F661F59
:106F1000771F8A95D1F79A01AB0168E1CE010E94F3
:106F20000637882311F086E034C08EEF8EBD80E0F6
:106F300090E00DB407FEFDCFF801E80FF91F2081A6
:106F40002EBD0DB407FEFDCF21812EBD0296811509
:106F500022E0920771F70DB407FEFDCF8FEF0E947C
:106F6000DF368FEF0E94DF360E94E4368B838F710D
:106F7000853031F083E18983CE010E94DA360AC080
:106F800068E572E0CE010E94EB36182F811107C030
:106F900087E18983CE010E94DA3610E012C020E03A
:106FA00030E0A9016DE0CE010E940637811104C0D6
:106FB0000E94E436882311F086E1EBCFCE010E94D7
:106FC000DA36812FDF91CF911F910F910895EF92C3
:106FD000FF920F931F93CF93DF93EC0179018C8184
:106FE000833039F089E0440F551F661F771F8A955B
:106FF000D1F79A01AB0161E1CE010E9406378823E7
:1070000031F084E08983CE010E94DA363CC00E94D0
:1070100018408B010E94E4368B838F3F49F40E9415
:107020001840601B710B6D327140A0F381E103C009
:107030008E3F49F08FE08983CE010E94DA368FEFD0
:107040000E94DF3620C08FEF8EBDF701D701A1501F
:10705000BE4F0DB407FEFDCF9EB591938EBDEA17CE
:10706000FB07B9F70DB407FEFDCF8EB58C930E94D8
:10707000E4360E94E436CE010E94DA368FEF0E9499
:10708000DF3681E001C080E0DF91CF911F910F9149
:10709000FF90EF9008952F923F924F925F926F92E0
:1070A0007F928F929F92AF92BF92CF92DF92EF9298
:1070B000FF920F931F93CF93DF9300D000D0CDB7F3
:1070C000DEB79C838B834B015A01DC0113968C91B4
:1070D000811103C08FEF9FEFEBC0EB81FC818181B9
:1070E00080FFF8CFAB81BC8151960D911D912D9100
:1070F0003C91549718964D915D916D917C911B97A1
:10710000C501A0E0B0E068017901C41AD50AE60A19
:10711000F70AC816D906EA06FB0618F45801A41A9D
:10712000B50A75018B819C8104969A838983612CB1
:1071300092E0792EE114F10409F48BC0AB81BC819B
:1071400018964D915D916D917C911B976A01B1E00C
:10715000DB22EB81FC8123811A012B0189E056940B
:107160004794379427948A95D1F7818D928D223058
:1071700061F4FC01828D938DA48DB58DBC01CD0190
:10718000620D731D841D951D4AC0DC0114961C916F
:1071900011501221C114D10401F511111EC0452B4B
:1071A000462B472B59F4EB81FC8185899689A78969
:1071B000B08D84839583A683B7830FC0AB81BC81D8
:1071C00014964D915D916D917C91179729813A812B
:1071D0000E94B4C8882309F47DCFEB81FC81218D06
:1071E000328D84819581A681B7810297A109B10969
:1071F000F901058404C0880F991FAA1FBB1F0A94B8
:10720000D2F74685578560897189840F951FA61F1F
:10721000B71FBC01CD01610F711D811D911D93012F
:107220002C193D0987012E153F0508F48901011528
:10723000F2E01F0779F520911B0C30911C0C409156
:107240001D0C50911E0C621773078407950719F4E3
:1072500021C0C5012DC09401AB01BC018091240C5B
:107260009091250C0E94E737882309F433CF800ED4
:10727000911EEB81FC8180859185A285B385800F6D
:10728000911FA11DB11D80879187A287B387E01A46
:10729000F10A50CF40E00E94E9C7882309F41ACFD1
:1072A000B601655E754FA801C4010E945BEDDFCF9A
:1072B0000F900F900F900F90DF91CF911F910F9132
:1072C000FF90EF90DF90CF90BF90AF909F908F9006
:1072D0007F906F905F904F903F902F9008954F92C6
:1072E0005F926F927F92AF92BF92CF92DF92EF92B6
:1072F000FF920F931F93CF93DF931F92CDB7DEB70B
:107300008C017B015A01D22EDB0159968D919C9103
:107310005A97F801928F818F40E050E0BA01C7017F
:107320000E9437CAC12CF70180859185A285B3855B
:10733000418952896389748984179507A607B7071D
:1073400008F063C025E0B695A795979587952A958F
:10735000D1F7F82FFF707F2ED70113968C918230D2
:1073600008F464C041E050E0BE016F5F7F4FC70189
:107370000E944B38019719F4898190E002C08FEF89
:107380009FEF019609F452C0F70180859185A2858F
:10739000B3854F96A11DB11D80879187A287B387C2
:1073A000F0E27F9EC0011124BC01655E754F61153E
:1073B0007105E1F1DB012C91222319F0253ED1F476
:1073C00069C1C1100EC040911B0C50911C0C609102
:1073D0001D0C70911E0CF8014487558766877787CE
:1073E000708AFC01E55EF54F8081882361F0CC2432
:1073F000C39499CF4BE050E0C5010E944EED892B1C
:1074000009F091CF15C0CC24C3948D2D82748234A1
:1074100069F4CC2009F48AC0D80150967C9061E0D0
:10742000C8010E948535009709F007C180E035C189
:10743000D7FCFCCFF0E27F9EA00111249A01255ECB
:10744000354FD9011B968C91817121F08D2D827160
:1074500009F068C080911B0C90911C0CA0911D0C30
:10746000B0911E0CF80184879587A687B787708A2C
:10747000FA01E55EF54F4489558960E070E0BA0194
:1074800055274427D80155964D935D936D937C9372
:107490005897828D938DA0E0B0E0482B592B6A2B32
:1074A0007B2BD80155964D935D936D937C935897A4
:1074B000D9011B968C91887159F4848D958DA68D78
:1074C000B78DF801818B928BA38BB48B81E010C0B8
:1074D000803141F598012F5E3F4FD80159968D912B
:1074E0009C915A970E9435C98823E1F084E0F80105
:1074F00083838D2D8F70D80111968C931197F8018D
:10750000148215821682178218961D921D921D9262
:107510001C921B97D4FEB1C0C8010E940C7181114E
:10752000ACC084CFD80113961C9280CFF701838121
:10753000823009F47BCF81899289A389B489803E06
:107540009F4FAF41B10508F071CFC7010E94D535FB
:10755000882309F46BCF0E94A9C7882309F466CF5A
:10756000D70159962D913C915A9714968D919D91E2
:107570000D90BC91A02D0297A109B109F9010584D4
:1075800004C0880F991FAA1FBB1F0A94D2F7468414
:10759000578460887188480E591E6A1E7B1E81E0E0
:1075A0008093230C40921B0C50921C0C60921D0C7B
:1075B00070921E0C80E092E0EBE1FAE0DF019C01AA
:1075C0001D9221503040E1F7CC24C394D701599645
:1075D000ED91FC915A978481C81698F42BE13AE01A
:1075E000B301A2014C0D511D611D711D8091240C30
:1075F0009091250C0E947B37882309F417CFC39400
:10760000E5CF80E092E0A0E0B0E0058404C0880F00
:10761000991FAA1FBB1F0A94D2F7F701418952890B
:1076200063897489840F951FA61FB71F818B928B66
:10763000A38BB48B8BE19AE0712C20E2DC011D92CC
:107640002A95E9F72BE0F501DC0101900D922A95CE
:10765000E1F721E238E2FC01318B208B40E058E079
:1076600057874687338B228B318F208F578B468BE2
:107670000E94A9C78111DECED9CED5FE09C0F8017E
:107680004189528963897489C8010E9437CA05C03B
:1076900081E003C0C110ABCE96CE0F90DF91CF91A9
:1076A0001F910F91FF90EF90DF90CF90BF90AF9020
:1076B0007F906F905F904F9008952F923F924F92DE
:1076C0005F926F927F928F929F92AF92BF92CF9272
:1076D000DF92EF92FF920F931F93CF93DF93CDB77B
:1076E000DEB7C254D1090FB6F894DEBF0FBECDBFCE
:1076F0004C015B018A01322E1C8E1F8E19821C8266
:107700006115710511F410E0A7C0FC01838181119E
:10771000FACFFA0180818F3209F09CC0F501838194
:107720008250823060F0618D728DCE0101960E9490
:107730002935882341F3CE0101967C0101C07501F2
:10774000C8018C010196F80120812F32D1F36E011E
:10775000FCE1CF0ED11C3601CE0101962C012396FF
:10776000CFAE23972D2C9BE09150E7E3F0E0EC0F98
:10777000FD1FE90FF11D80E280839111F5CFD80143
:1077800027E04A2F3B2F8D91811107C08FA98032AE
:1077900009F4B9CF842F932F2CC08F32B9F38E32D6
:1077A00031F42A3009F4AFCF98E02AE0EACFEAE5D5
:1077B000F8E03491332321F031963813FACFA3CF78
:1077C000291708F4A0CF813208F49DCF8F3709F430
:1077D0009ACF31E0390FE7E3F0E0EC0FFD1FE90F3E
:1077E000F11D9FE9980F9A3108F480528083932FFE
:1077F000C8CF8C01FC01208101962F32D1F32223C6
:10780000F9F021E0AE01495C5F4FB701C6010E946B
:107810006F39882309F477CFEA14FB0419F0C70104
:107820000E947C35C614D70441F023969FAD239760
:10783000822D7601C92ED82E96CF942D852DF9CF85
:10784000232DAE01495C5F4FB701C4010E946F391F
:10785000182F02C07B017BCFCE0101960E94FC82D3
:10786000CE014C960E94FC82812FCE5BDF4F0FB67B
:10787000F894DEBF0FBECDBFDF91CF911F910F9166
:10788000FF90EF90DF90CF90BF90AF909F908F9040
:107890007F906F905F904F903F902F900895CF9280
:1078A000DF92EF92FF92CF93DF93EC01C090080A32
:1078B000D090090AE0900A0AF0900B0AA7019601FD
:1078C000688179818A819B810E94ABE587FF04C032
:1078D000C882D982EA82FB82C0900C0AD0900D0A3D
:1078E000E0900E0AF0900F0AA70196016C817D814D
:1078F0008E819F810E94ABE587FF04C0CC82DD8230
:10790000EE82FF82C0903501D0903601E0903701C1
:10791000F0903801A7019601688179818A819B8165
:107920000E943CEC181624F4C882D982EA82FB82B9
:10793000C0903901D0903A01E0903B01F0903C01B9
:10794000A70196016C817D818E819F810E943CEC14
:10795000181624F4CC82DD82EE82FF82C090100AD9
:10796000D090110AE090120AF090130AA701960134
:10797000688579858A859B850E94ABE587FF04C071
:10798000C886D986EA86FB86C0903D01D0903E012C
:10799000E0903F01F0904001A7019601688579854C
:1079A0008A859B850E943CEC181624F4C886D986EB
:1079B000EA86FB86DF91CF91FF90EF90DF90CF902A
:1079C00008954F925F926F927F928F929F92AF92A3
:1079D000BF92DF92EF92FF920F931F93CF93DF93AB
:1079E000D82EC82FD0E0FE01E95AF74F64917E01EE
:1079F000EE0CFF1CEE0CFF1CF701E55BF74F45900A
:107A0000559065907490062E000C770B880B990B9F
:107A10000E94B2E54B015C0120E030E040EC5FE306
:107A2000C301B2010E9411E6A50194010E9411E672
:107A3000AB01BC0100E010E098018D2D0E9437AA37
:107A4000F701E15CF74F2591359145915491C501BE
:107A5000B4010E9411E64B015C0120E030E0A90175
:107A60000E94ABE5882309F448C000E010E09801CB
:107A7000B501A40170588D2D0E9437AAFE01E45C67
:107A8000F74F4491411117C0E1E9F1E28491EF0110
:107A90002196882321F00E940283FE01F7CFEAE1BC
:107AA000F8E08491EF012196882321F00E9402835F
:107AB000FE01F7CF4AE0F701E65FF74F459055909A
:107AC00065907490642F70E080E090E00E94B2E5D1
:107AD0009B01AC01C301B2010E94D6EA2B013C011B
:107AE000A5019401C501B4010E94DCE9AB01BC0110
:107AF000930182018D2D0E9437AA81E090E00D2C28
:107B000001C0880F0A94EAF790915B03982B909339
:107B10005B039091F902892B8093F902F701E959EF
:107B2000FD4F10821182128213828D2D0E94ABAB09
:107B3000F701E250F84F85919591A591B491E70135
:107B4000C859DC4F88839983AA83BB830E9427820C
:107B5000F701ED58FD4F88819981AA81BB8180830F
:107B60009183A283B383DF91CF911F910F91FF90F7
:107B7000EF90DF90BF90AF909F908F907F906F902D
:107B80005F904F9008950F931F93CF93DF938C01D5
:107B9000E1E9F1E28491EF012196882321F00E942E
:107BA0000283FE01F7CFB80181EF97E00E94B64F44
:107BB00082E20E9402838AE00E94028381E0DF91D8
:107BC000CF911F910F9108952CE831E0FC01318392
:107BD000208304960C94FC828C01E6E7F1E2849108
:107BE000EF012196882321F00E940283FE01F7CF46
:107BF000E1EDF7E08491EF012196882321F00E94C6
:107C00000283FE01F7CF0E94DDCF0E94C5D50E94FE
:107C10004A5C61E0C8010E94F3580E945D63C09114
:107C20003006C695C6950E940A73DC2FDD0F1D2F06
:107C30001C0F84E00E94F76D10926606C0936706E1
:107C400066E187E29CE00E94E36D10926606D093A5
:107C5000670682EC97E00E94A67210926606109367
:107C6000670685EB97E00E94A6720E9461728111FF
:107C7000E0CF2FEF8BE49DE1215080409040E1F771
:107C800000C00000F8942FEF84E39CE02150804076
:107C90009040E1F700C000000E94DDCFA895FECF24
:107CA0003FB7F8948091880290918902A0918A024E
:107CB000B0918B0226B5A89B05C02F3F19F0019605
:107CC000A11DB11D3FBFBA2FA92F982F8827820F62
:107CD000911DA11DB11DBC01CD0142E0660F771FB2
:107CE000881F991F4A95D1F708950895FC01A68130
:107CF000B7818281481B8581483018F0A80FB11DDB
:107D00004770382F369536953695562F577080E840
:107D100090E002C0959587955A95E2F7439F402DD4
:107D20001124669566956695E62FF0E0E40FF11D47
:107D3000EA0FFB1F3081222311F0832B02C08095B4
:107D4000832380830895FB014181DC0112962C91ED
:107D50001297421768F013962C911397241740F04E
:107D6000608115962C91621718F424810C94763E4C
:107D70000895FC0180819281980F9283218192174E
:107D800060F494819F5F94839381890F821710F030
:107D90008FEF820F838381E0089580E00895FC01D6
:107DA00012828081815083831482089580E0089537
:107DB0000B96FC01849108950A96FC018491089524
:107DC000FC01849108950E94E03E882321F08230D6
:107DD00011F083E0089586E00895FC01E60FF11D9F
:107DE000849190E0982F88273196E4918E0F911D11
:107DF000089568E00C94ED3E66E00C94ED3E81E061
:107E0000089590E0FC013197EA30F10540F5EA5B16
:107E1000FF4F0C9430ED809180008F7703C08091EC
:107E200080008F7D80938000089584B58F7702C095
:107E300084B58F7D84BD08958091B0008F7703C095
:107E40008091B0008F7D8093B00008958091900064
:107E50008F7703C0809190008F7D8093900008956C
:107E6000CF93DF9390E0FC01EC58F74E2491FC0196
:107E7000EC5AF74E8491882361F190E0880F991FA6
:107E8000FC01E659F74FC591D491FC01E05CF74E37
:107E9000A591B491611109C09FB7F894888120958C
:107EA00082238883EC912E230BC0623061F49FB74C
:107EB000F8943881822F809583238883EC912E2B30
:107EC0002C939FBF06C08FB7F894E8812E2B288390
:107ED0008FBFDF91CF9108951F93CF93DF93182F1A
:107EE000EB0161E00E94303F209711F460E004C094
:107EF000CF3FD10539F461E0812FDF91CF911F9100
:107F00000C945164E12FF0E0EC56F74EE4914E2FC3
:107F100050E0FA013197EA30F10508F046C0E05B25
:107F2000FF4F0C9430ED84B5806884BDC7BD42C05E
:107F300084B5806284BDC8BD3DC0809180008068EA
:107F400080938000D0938900C093880033C08091D3
:107F50008000806280938000D0938B00C0938A0061
:107F600029C08091B00080688093B000C093B300B6
:107F700021C08091B00080628093B000C093B400B3
:107F800019C080919000806880939000D0939900F0
:107F9000C09398000FC08091900080628093900001
:107FA000D0939B00C0939A0005C0C038D1050CF057
:107FB000A2CF9CCFDF91CF911F9108958F929F9276
:107FC000AF92BF92CF92DF92EF92FF926B017C0152
:107FD0000E94503E4B015C01C114D104E104F10444
:107FE000F1F00E94503EDC01CB0188199909AA09E1
:107FF000BB09883E9340A105B10570F321E0C21A88
:10800000D108E108F10888EE880E83E0981EA11CD3
:10801000B11CC114D104E104F10419F7DDCFFF90C4
:10802000EF90DF90CF90BF90AF909F908F9008958A
:108030002FB7F89460918402709185028091860236
:10804000909187022FBF08951F920F920FB60F9243
:1080500011242F933F938F939F93AF93BF9380915E
:10806000840290918502A0918602B091870230919E
:10807000830223E0230F2D3720F40196A11DB11DAB
:1080800005C026E8230F0296A11DB11D209383028F
:108090008093840290938502A0938602B093870216
:1080A0008091880290918902A0918A02B0918B02FE
:1080B0000196A11DB11D8093880290938902A0931F
:1080C0008A02B0938B02BF91AF919F918F913F91A4
:1080D0002F910F900FBE0F901F901895CF92DF92A7
:1080E000FF920F931F93CF93DF9300D0CDB7DEB7EE
:1080F0006901DB0112960D911C911397423309F42B
:1081000071C0B8F4453109F47AC0473109F48BC025
:10811000443109F0A1C0D80115962C9115971696F7
:10812000ED91FC911797CF01820F911D820F911D48
:108130005EC0463409F487C0473409F488C04B3325
:1081400009F08AC0F90181819381913029F093303F
:1081500031F4482F885004C048E0480F01C0482F30
:1081600021E0D80113963C91381708F420E031E063
:10817000F8015281451708F430E051E0481708F043
:1081800050E0822F852B382319F4252309F464C08D
:10819000D6011296FC90913051F030F0923049F0B7
:1081A000933051F42FEF09C020E031E007C021E007
:1081B00004C020E03FEF02C020E030E0F7FE08C03E
:1081C000B601C8012A8339830E94A33E39812A81DE
:1081D000F6018081830F80838181820F8183FF0C70
:1081E00069F73AC0B901C8010E94A33E35C0119297
:1081F000E817F907E1F7C8010E94CF3E2DC0C8017A
:108200000E94B93E882349F1F80125810680F78153
:10821000E02DCF01820F911D820F911D1192E81761
:10822000F907E1F719C0D9011C92F8018281119672
:108230008C9311978581815012968C93129783812C
:1082400013968C9309C0D80115968C9103C0D80160
:1082500011968C91F601808381E00F900F90DF9151
:10826000CF911F910F91FF90DF90CF900895DB0188
:10827000ED91FC9109948F929F92BF92CF92DF92E1
:10828000EF92FF920F931F93CF93DF931F92CDB77F
:10829000DEB74C01062FF42E122F522FE62EE20EDF
:1082A000BB24BA946C018CE1C80ED11C8E2D851BA9
:1082B000583080F0F40162817381848FF58E178EBF
:1082C000B68E96014BE3C40159830E943741598110
:1082D0005850ECCF812F887F080F212F277021F174
:1082E00087E02827F40162817381048FF58E178E51
:1082F0002F5F27708FEF90E001C0880F2A95EAF773
:10830000868F9401245E3F4F4BE3C4010F90DF91B1
:10831000CF911F910F91FF90EF90DF90CF90BF9082
:108320009F908F900C9437410F90DF91CF911F91C8
:108330000F91FF90EF90DF90CF90BF909F908F9024
:108340000895EF92FF920F931F93CF93DF937C01D9
:10835000D62F122FC42F040F212F4C2F6D2FC701A2
:108360000E943B41CF5F0C13F7CFDF91CF911F915C
:108370000F91FF90EF900895EF92FF920F931F934C
:10838000CF93DF931F92CDB7DEB78C01DC0112963D
:10839000ED90FC901397D196ED91FC91D29782E0ED
:1083A000099520E030E04AE0B701C8010E9437415A
:1083B000F82ED801D196ED91FC91D29783E00995E2
:1083C000D801D196ED91FC91D29780E00995FF20DC
:1083D000A1F1F801628173819E012F5F3F4F46E456
:1083E000C8010E9437418981D8018C9312966D9102
:1083F0007C9113979E012F5F3F4F47E4C8010E9475
:1084000037418981F80181836281738120E030E006
:1084100048E4C8010E943741D8011B968C931B97F2
:1084200098012D5C3F4F12966D917C91139747E117
:10843000C8010E94374181E001C080E00F90DF91C8
:10844000CF911F910F91FF90EF90089588E290E0F7
:108450000197F1F708952EE93FE0009729F0F9011F
:108460003197F1F70197F9CF08950F93FC0101506F
:10847000040F84A996A9941718F0081728F402C0CD
:10848000081750F0041740F42150260F83A995A92E
:10849000961720F4281720F480E007C0281720F44E
:1084A00081E0261710F0F8CF81E00F910895DF9258
:1084B000EF92FF920F931F93CF93DF93EC01162F50
:1084C000F42EE22E0E943542882331F02E2D4F2DBE
:1084D000612FCE010E94A141DF91CF911F910F9199
:1084E000FF90EF90DF9008952F923F925F926F92EE
:1084F0007F928F929F92AF92BF92CF92DF92EF9234
:10850000FF920F931F93CF93DF931F92CDB7DEB7E8
:108510001C01C62E142FD22EDC011496ED90FC9077
:108520001597C7010E94E03E082FF10184819581D3
:108530000E94E33E982E013019F48FE0A82E02C06D
:10854000AA24AA94D10114968D919C9115970E940A
:10855000DC3E082FF101848195810E94D83EB82E1F
:10856000D10114968D919C9115970E94F93EB0E629
:10857000BD1530F4009721F0E80EF91E01E611C098
:10858000F101848195810E94FC3EF0E4FD1530F4F8
:10859000009721F0E80EF91E01E403C021E1E20E8C
:1085A000F11CBD1480F4D10150961C925097539643
:1085B0001C92539754961C92549751961C92519723
:1085C00052961C92C7C0B01670F3892D90E0F70147
:1085D00024912F3F21F4FFEFEF1AFF0A5AC00D112B
:1085E0004FC0D10114968D919C9115970E94E03E49
:1085F00097012F5F3F4FF701882311F08230E1F49C
:108600008491D10153968C935397F90124915496F8
:108610002C935497F7013396E4915096EC9350972E
:10862000F7013496E4915196EC935197F701359602
:10863000E4915296EC9320C08491982F9F709250B1
:10864000D10152969C93529782958F7051968C933C
:108650005197F9012491822F8F7054968C935497DF
:1086600022952F7053962C935397F7013296E491ED
:10867000E295EF705096EC93E114F10479F46AC03E
:10868000F7013296E491EA219C012E0F311DE20E92
:10869000F31E0B1509F487CF0F5F99CFF101848189
:1086A00095810E94E33EB82ED10153969C9053973A
:1086B0005496DC90549751968C915197C80E5296CF
:1086C0009C919D0D512E591A0D2D292D452D6C2D46
:1086D000C1010E9435428823D1F1C7018B0D911D44
:1086E0005C0187E0890DF82EF694F694F694D50C8B
:1086F00041019CE1890E911C6F2C712C5D1439F1A4
:108700005C2D8501802F8A198F15E8F4F80184917A
:10871000D10112966D917C9113975C965C935C9756
:108720005D965C925D975F961C925F975E968C93C8
:1087300094014BE3C10159830E9437410F5F1F4FE2
:108740005981585FDFCFA60CB71C5394D7CFF101E6
:10875000808901C080E00F90DF91CF911F910F9130
:10876000FF90EF90DF90CF90BF90AF909F908F9051
:108770007F906F905F903F902F9008958F929F927F
:10878000AF92BF92CF92DF92EF92FF92CF93FC0114
:10879000C080D180E280F38020E030E0A901C701F1
:1087A000B6010E94ABE587FF08C0C701B60190582B
:1087B00020E030E04AE754E406C020E030E04AE739
:1087C00054E4C701B6010E9411E620E030E040EA1F
:1087D00050E40E94DCE920E030E040E251E40E94F5
:1087E000D6EA0E9448EB6B017C01603AF6E87F070D
:1087F000F1E08F07910584F020EA36E841E050E08F
:108800000E9411EDCA01B9012AE030E040E050E0D9
:108810000E9411ED605D01C060E26093E61180E1AD
:10882000C81687E2D806E104F10494F0C701B60146
:1088300020E137E240E050E00E9411EDCA01B901A9
:108840002AE030E040E050E00E9411ED605D01C0A0
:1088500060E26093E711E8EECE16E3E0DE06E104A5
:10886000F10494F0C701B60128EE33E040E050E097
:108870000E9411EDCA01B9012AE030E040E050E069
:108880000E9411ED605D01C060E26093E811C701D4
:10889000B60124E630E040E050E00E9411ED8AE0AD
:1088A000882E912CA12CB12CCA01B901A5019401EB
:1088B0000E9411ED605D6093E9118EE28093EA11F0
:1088C000C701B601A50194010E9411EDC62FCA018E
:1088D000B901A50194010E9411ED605D6093EB1157
:1088E000C05DC093EC1186EE91E1CF91FF90EF90C7
:1088F000DF90CF90BF90AF909F908F9008958F9210
:108900009F92AF92BF92CF92DF92EF92FF92CF935E
:10891000FC01C080D180E280F38020E030E04AE7B3
:1089200054E4C701B6010E9411E64B015C0120E04E
:1089300030E0A901C701B6010E94ABE587FD05C083
:1089400020E030E040EA50E404C020E030E040EABB
:1089500050ECC501B4010E94DCE920E030E040E2C7
:1089600051E40E94D6EA0E9448EB6B017C0197FF1C
:108970000AC0F094E094D094C094C11CD11CE11CB6
:10898000F11C8DE201C08BE28093E611C701B601B4
:1089900020E137E240E050E00E9411ED8AE0882EAD
:1089A000912CA12CB12CCA01B901A50194010E94FE
:1089B00011ED605D6093E711C701B60128EE33E069
:1089C00040E050E00E9411EDCA01B901A5019401F7
:1089D0000E9411ED605D6093E811C701B60124E6C5
:1089E00030E040E050E00E9411EDCA01B901A5015C
:1089F00094010E9411ED605D6093E9118EE2809315
:108A0000EA11C701B601A50194010E9411EDC62F1C
:108A1000CA01B901A50194010E9411ED605D609346
:108A2000EB11C05DC093EC1186EE91E1CF91FF9008
:108A3000EF90DF90CF90BF90AF909F908F90089570
:108A40008F929F92AF92BF92CF92DF92EF92FF925E
:108A5000FC01C080D180E280F38020E030E0A901F9
:108A6000C701B6010E94ABE587FF08C0C701B60188
:108A7000905820E030E040E251E406C020E030E0D1
:108A800040E251E4C701B6010E9411E620E030E067
:108A900040EA50E40E94DCE920E030E040E251E4AA
:108AA0000E94D6EA0E9448EB6B017C016031F7E23C
:108AB0007F078105910584F020E137E240E050E036
:108AC0000E9411EDCA01B9012AE030E040E050E017
:108AD0000E9411ED605D01C060E26093E81188EED4
:108AE000C81683E0D806E104F10494F0C701B6018A
:108AF00028EE33E040E050E00E9411EDCA01B901D8
:108B00002AE030E040E050E00E9411ED605D01C0DD
:108B100060E26093E911E4E6CE16D104E104F104C9
:108B200094F0C701B60124E630E040E050E00E9436
:108B300011EDCA01B9012AE030E040E050E00E94A6
:108B400011ED605D01C060E26093EA11FAE0CF16BA
:108B5000D104E104F1049CF08AE0882E912CA12C30
:108B6000B12CC701B601A50194010E9411EDCA0103
:108B7000B901A50194010E9411ED605D01C060E2A0
:108B80006093EB11C701B6012AE030E040E050E00D
:108B90000E9411ED605D6093EC1188EE91E1FF9011
:108BA000EF90DF90CF90BF90AF909F908F900895FF
:108BB0008F929F92AF92BF92CF92DF92EF92FF92ED
:108BC000FC01C080D180E280F38020E030E048ECFE
:108BD00052E4C701B6010E9411E64B015C0120E09E
:108BE00030E0A901C701B6010E94ABE587FD05C0D1
:108BF00020E030E040EA50E404C020E030E040EA09
:108C000050ECC501B4010E94DCE920E030E040E214
:108C100051E40E94D6EA0E9448EB9B0177FF06C010
:108C200022273327261B370B8DE201C08BE280936E
:108C3000E711C90168EE73E00E94FDECCB01EAE0A8
:108C4000F0E0BF010E94FDEC805D8093E811C90156
:108C500064E670E00E94FDECCB01BF010E94FDECD8
:108C6000805D8093E911C901BF010E94FDEC282FAE
:108C7000CB01BF010E94FDEC805D8093EA118EE282
:108C80008093EB11205D2093EC1187EE91E1FF9032
:108C9000EF90DF90CF90BF90AF909F908F9008950E
:108CA0008F929F92AF92BF92CF92DF92EF92FF92FC
:108CB000CF93FC01C080D180E280F38020E030E0DF
:108CC0004AE754E4C701B6010E9411E64B015C017A
:108CD00020E030E0A901C701B6010E94ABE587FDA5
:108CE00005C020E030E040EA50E404C020E030E07D
:108CF00040EA50ECC501B4010E94DCE920E030E01C
:108D000040E251E40E94D6EA0E9448EB6B017C01EC
:108D100097FD10C020E137E240E050E00E9411EDE5
:108D2000CA01B9012AE030E040E050E00E9411EDB4
:108D3000605D09C0F094E094D094C094C11CD11C33
:108D4000E11CF11C6DE26093E711C701B60128EE4A
:108D500033E040E050E00E9411ED8AE0882E912C33
:108D6000A12CB12CCA01B901A50194010E9411EDF9
:108D7000605D6093E811C701B60124E630E040E091
:108D800050E00E9411EDCA01B901A50194010E94B1
:108D900011ED605D6093E9118EE28093EA11C701E5
:108DA000B601A50194010E9411EDC62FCA01B901B7
:108DB000A50194010E9411ED605D6093EB11C05D0F
:108DC000C093EC1187EE91E1CF91FF90EF90DF908F
:108DD000CF90BF90AF909F908F900895AC01952F4A
:108DE000991F9927991F29F022273327241B350B18
:108DF00001C09A01483E5340ACF0C90168EE73E0EF
:108E00000E94FDECCB01EAE0F0E0BF010E94FDEC26
:108E1000805D8093E911C90164E670E00E94FDEC79
:108E2000CB0112C024363105B4F0911102C080E2AA
:108E300001C08DE28093E911C90164E670E00E94EF
:108E4000FDECCB01EAE0F0E0BF010E94FDEC805DAB
:108E50008093EA110EC080E28093E9118093EA11B9
:108E60002A30310584F091118DE28093EA11EAE015
:108E7000F0E0C901BF010E94FDECCB01BF010E94DF
:108E8000FDEC805D05C0911102C080E201C08DE261
:108E90008093EB11C9016AE070E00E94FDEC805DF7
:108EA0008093EC1189EE91E108959C0197FD0EC02D
:108EB0008436910584F064E670E00E94FDECCB01FD
:108EC0006AE070E00E94FDEC805D06C0319521955E
:108ED00031098DE201C080E28093EA112A30310528
:108EE00064F0EAE0F0E0C901BF010E94FDECCB01B3
:108EF000BF010E94FDEC805D01C080E28093EB1118
:108F0000C9016AE070E00E94FDEC805D8093EC1185
:108F10008AEE91E10895CF92DF92EF92FF928091D5
:108F20000605882371F1C0900205D0900305E090FA
:108F30000405F090050520E030E0A901C701B60165
:108F40000E94ABE58823E9F020E030E040E05FE3F9
:108F5000C701B6010E9411E69B01AC010E9411E617
:108F60002BED3FE049E450E40E9411E69B01AC0187
:108F700060E070E080E89FE30E94D6EA6B017C012C
:108F800006C0C12CD12C80E8E82E8FE3F82EC092C9
:108F9000FA11D092FB11E092FC11F092FD11609158
:108FA0004C0170914D01072E000C880B990B0E940B
:108FB000B2E52AE037ED43E25CE30E9411E6A70147
:108FC00096010E9411E660934301709344018093DF
:108FD000450190934601FF90EF90DF90CF90089568
:108FE000CF93DF9380916C0690916D06891B8F70F3
:108FF00009F445C090916906992351F0833030F40B
:109000008FEF890F19F0809369063BC010926906B3
:10901000E0916D068DE4E89FF0011124EE52F34FCC
:10902000808180FD2EC08091AB0C9091AC0CA09102
:10903000AD0CB091AE0CEF01C75BDF4F4881598199
:109040006A817B81841B950BA60BB70B8093AB0CBD
:109050009093AC0CA093AD0CB093AE0C80916D06C8
:109060008F5F8F7080936A0690916D0680916B067A
:1090700098130AC080916A0680936B0605C00E940F
:10908000EDB080E090E001C0CF01DF91CF91089575
:109090000F930FB70F9300916E000F930B7F009308
:1090A0006E0000916F000D7F00936F000F930BB760
:1090B0000F930CB70F921F922F933F934F935F9391
:1090C0006F937F938F939F93AF93BF93EF93FF9390
:1090D00011240E94B848FF91EF91BF91AF919F91E9
:1090E0008F917F916F915F914F913F912F911F9041
:1090F0000F900CBF0F910BBF0F910260F89400937B
:109100006F000F9100936E000F910FBF0F91189594
:1091100080918C0280FF03C0459A8FEF02C0459872
:1091200081E08093040180918C0281FF03C0479A03
:109130008FEF02C0479881E08093050180918C02F7
:1091400082FF03C02A988FEF02C02A9A81E08093A1
:10915000060180918C0283FF03C0289A8FEF02C022
:10916000289881E080930701000000000000089526
:109170003F924F925F926F927F928F929F92AF92A7
:10918000BF92CF92DF92EF92FF920F931F93CF93F4
:10919000DF93F8948FEF9FEF90938900809388007E
:1091A0009AE0392EC0E0D0E0CC24CA94DC2C7601C1
:1091B00078948091D0029091D102A091D202B09186
:1091C000D302892B8A2B8B2B09F0CDC180910412FD
:1091D0008823D1F010920412809102129091031210
:1091E000892B91F010928D021092031210920212AC
:1091F00090916C0680916D06981731F080916D0604
:109200008F5F8F7080936D06809102129091031290
:10921000892B09F4A8C14091CC025091CD026091F4
:10922000CE027091CF029091BB020091C8021091C2
:10923000C9022091CA023091CB02041B150B260BE8
:10924000370B892F90E0A0E0B0E0081719072A0734
:109250003B0710F4D901C801282F840F951FA61FC2
:10926000B71F8093CC029093CD02A093CE02B0930F
:10927000CF0280918400909185004E968090A30249
:109280009090A402A090A502B090A60240919302F3
:10929000509194026091950270919602480D591D6B
:1092A0006A1D7B1D4093A3025093A4026093A50204
:1092B0007093A60277FD1CC05F9A80901112909067
:1092C0001212A0901312B090141240910401042EB7
:1092D000000C550B660B770B480D591D6A1D7B1D45
:1092E0004093111250931212609313127093141240
:1092F0008090A7029090A802A090A902B090AA0224
:1093000040919702509198026091990270919A024F
:10931000480D591D6A1D7B1D4093A7025093A8025A
:109320006093A9027093AA0277FD1CC0469A8090B0
:10933000151290901612A0901712B090181240912A
:109340000501042E000C550B660B770B480D591DBB
:109350006A1D7B1D409315125093161260931712CD
:10936000709318128090AB029090AC02A090AD0266
:10937000B090AE0240919B0250919C0260919D0280
:1093800070919E02480D591D6A1D7B1D4093AB02D2
:109390005093AC026093AD027093AE0277FD1CC097
:1093A0002B9A8090191290901A12A0901B12B090D4
:1093B0001C1240910601042E000C550B660B770B16
:1093C000480D591D6A1D7B1D4093191250931A12A6
:1093D00060931B1270931C128090AF029090B002A9
:1093E000A090B102B090B20240919F025091A002B1
:1093F0006091A1027091A202480D591D6A1D7B1D4A
:109400004093AF025093B0026093B1027093B202E6
:1094100077FD1CC0299A80901D1290901E12A0907A
:109420001F12B090201240910701042E000C550B22
:10943000660B770B480D591D6A1D7B1D40931D124D
:1094400050931E1260931F1270932012409184005B
:109450005091850048175907C8F34091A3025091D5
:10946000A4026091A5027091A60277FD15C08090BC
:109470008F0290909002A0909102B09092024819B1
:1094800059096A097B094093A3025093A40260938F
:10949000A5027093A6025F984091A7025091A8027E
:1094A0006091A9027091AA0277FD15C080908F0289
:1094B00090909002A0909102B090920248195909A0
:1094C0006A097B094093A7025093A8026093A902FE
:1094D0007093AA0246984091AB025091AC02609101
:1094E000AD027091AE0277FD15C080908F02909012
:1094F0009002A0909102B0909202481959096A090D
:109500007B094093AB025093AC026093AD02709321
:10951000AE022B984091AF025091B0026091B1021F
:109520007091B20277FD15C080908F0290909002EA
:10953000A0909102B0909202481959096A097B09DA
:109540004093AF025093B0026093B1027093B202A5
:109550002998215041F0409184005091850048178E
:109560005907C8F38ACE8091D0029091D102A09180
:10957000D202B091D302892B8A2B8B2B09F020C306
:10958000E0910212F0910312309739F18091CC02F0
:109590009091CD02A091CE02B091CF024091C8022D
:1095A0005091C9026091CA027091CB02841795074D
:1095B000A607B707C8F010928D02109203121092FE
:1095C000021290916C0680916D06981731F080918F
:1095D0006D068F5F8F7080936D0680ED882E87E01B
:1095E000982EA12CB12C4FC14091C4025091C502BC
:1095F0006091C6027091C702481759076A077B0736
:1096000008F467C08091C0029091C102A091C2028B
:10961000B091C30242A953A964A975A91127859FD6
:10962000012D969F9001A69F300DA59F200D311D05
:10963000869F000D211D311F959F000D211D311F9B
:10964000A49F000D211D311F949F010D211F311F6B
:109650000695211F311F789F200D311D799F300DF8
:10966000112443AD54AD65AD76AD420F531F611D5E
:10967000711D4093BC025093BD026093BE02709373
:10968000BF0207A910AD21AD32AD0417150726079B
:10969000370740F40093BC021093BD022093BE0232
:1096A0003093BF028090BC029090BD02A090BE0299
:1096B000B090BF0224E730E141E0F90145905590B8
:1096C00065907490481459046A047B0408F4BFC27E
:1096D000CAC24091B7025091B8026091B90270912C
:1096E000BA02481759076A077B0708F063C08091E0
:1096F000B3029091B402A091B502B091B60242A912
:1097000053A964A975A91127859F012D969F9001E2
:10971000A69F300DA59F200D311D869F000D211D98
:10972000311F959F000D211D311FA49F000D211D8C
:10973000311F949F010D211F311F0695211F311FDD
:10974000789F200D311D799F300D1124890120E073
:1097500030E08090BC029090BD02A090BE02B0901C
:10976000BF02FF96081519052A053B0580F44081C4
:10977000518162817381801A910AA20AB30A841608
:109780009506A606B70638F44A015B0104C080803E
:109790009180A280B38024E730E141E0F901459057
:1097A000559065907490481459046A047B0408F439
:1097B000C3C2CEC28091090190910A01A0910B0110
:1097C000B0910C01B7FF57C087A990ADA1ADB2AD64
:1097D00024E730E141E0F90185909590A590B4909F
:1097E00088169906AA06BB0658F4B695A7959795CC
:1097F0008795440F2C5F3F4FF0E120393F0759F721
:109800004093BB0280329105A105B10508F42EC337
:109810008097A109B109811528E09207A105B1053A
:1098200008F4FFC244E0949FF00111249F012C58DA
:10983000334FF901329645915491EE27859FB0013F
:10984000849F610D7E1F06946E1F7E1F1124AB0145
:1098500060E070E0F90185919491A0E0B0E0841B94
:10986000950BA60BB70B8093090190930A01A09367
:109870000B01B0930C018090090190900A01A09017
:109880000B01B0900C018091021290910312892B70
:1098900009F08EC10E94F047909303128093021248
:1098A000892B09F485C1E0910212F09103128081A5
:1098B00083FF3EC085899689A789B08D8093111258
:1098C00090931212A0931312B0931412818D928D63
:1098D000A38DB48D8093151290931612A093171236
:1098E000B0931812858D968DA78DB0A18093191213
:1098F00090931A12A0931B12B0931C1281A192A1F3
:10990000A3A1B4A180931D1290931E12A0931F12C5
:10991000B093201290916C0680916D06981709F40F
:10992000B9CF80916D068F5F8F7080936D06B2CF37
:10993000058916892789308D81E0011511052105DA
:10994000310509F480E0818C928CA38CB48C811455
:109950009104A104B10409F08260458D568D678D94
:1099600070A1411551056105710509F0846080936E
:109970008D021092B3021092B4021092B5021092AE
:10998000B6021092C0021092C1021092C20210924E
:10999000C30285A196A1A7A1B0A58093C802909308
:1099A000C902A093CA02B093CB02442455243201C9
:1099B000481A590A6A0A7B0A4092AF025092B002D2
:1099C0006092B1027092B2024092AB025092AC022D
:1099D0006092AD027092AE024092A7025092A8022D
:1099E0006092A9027092AA024092A3025092A4022D
:1099F0006092A5027092A602000F111F221F331F52
:109A00000093930210939402209395023093960250
:109A1000880C991CAA1CBB1C8092970290929802F9
:109A2000A0929902B0929A02440F551F661F771FA9
:109A300040939B0250939C0260939D0270939E0200
:109A400041A152A163A174A1440F551F661F771F46
:109A500040939F025093A0026093A1027093A202D0
:109A6000880F991FAA1FBB1F80938F0290939002AB
:109A7000A0939102B09392021092CC021092CD0268
:109A80001092CE021092CF0282A593A5A4A5B5A5EF
:109A90008093C4029093C502A093C602B093C702FC
:109AA00086A597A5A0A9B1A98093B7029093B80203
:109AB000A093B902B093BA0281A580938E0296A9B1
:109AC00020918C0292130AC02091080130E0482FA7
:109AD000082E000C550B4217530731F090938C025F
:109AE000809308010E94884880915A0381110E9446
:109AF00009B1C0920901D0920A01E0920B01F092E3
:109B00000C01E0910212F091031283AD94ADA5AD6A
:109B1000B6AD8093BC029093BD02A093BE02B093F9
:109B2000BF0224E730E141E0F90185909590A590CE
:109B3000B49088169906AA06BB0658F4B695A79560
:109B400097958795440F2C5F3F4F50E1203935079B
:109B500059F74093BB0280329105A105B10508F485
:109B6000ADC18097A109B109811558E09507A105FC
:109B7000B10508F480C1F4E09F9F900111242C5896
:109B8000334FF901329645915491EE27859FB001EC
:109B9000849F610D7E1F06946E1F7E1F1124F901A4
:109BA00085909490A12CB12C861A970AA108B1082F
:109BB0008092D0029092D102A092D202B092D302AF
:109BC0008091D0029091D102A091D202B091D302A3
:109BD000AC01BD01009721E0A207B10520F04FEFD5
:109BE0005FEF60E070E0841B950BA60BB70B8093D2
:109BF000D0029093D102A093D202B093D302F894F2
:109C0000809184009091850040963A94332039F0F9
:109C1000C40FD51FC817D90708F4CACA01C0EC0180
:109C2000D0938900C09388007894DF91CF911F91E1
:109C30000F91FF90EF90DF90CF90BF90AF909F90EB
:109C40008F907F906F905F904F903F900895B69463
:109C5000A79497948794440F2C5F3F4F50E120398D
:109C6000350709F02ACD4093BB0240E284169104E7
:109C7000A104B10408F45AC020E2821A9108A10894
:109C8000B108811448E09406A104B104F8F054E04E
:109C9000959E900111242C58334FF901329645912D
:109CA0005491F82DEE27F59FB001F49F610D7E1FB2
:109CB00006946E1F7E1F1124F90185909490A12CAB
:109CC000B12C861A970AA108B10823C0B501A401D6
:109CD0007695679557954795FA01EC7FAF014C58FB
:109CE000574FFA0125913491FA013296659174919A
:109CF000E82DE770E69FA001E79F500D112403E0D7
:109D0000569547950A95E1F7241B350B4901A12C7F
:109D1000B12C880D991DAA1DBB1D8093C002909384
:109D2000C102A093C202B093C302ADCD10E2812E56
:109D3000912CA12CB12CA0CFB694A7949794879482
:109D4000440F2C5F3F4F50E12039350709F026CDF5
:109D50004093BB02F0E28F169104A104B10408F411
:109D60005AC020E2821A9108A108B108811448E083
:109D70009406A104B104F8F054E0959E90011124DA
:109D80002C58334FF901329645915491F82DEE2716
:109D9000F59FB001F49F610D7E1F06946E1F7E1F1C
:109DA0001124F90185909490A12CB12C861A970A60
:109DB000A108B10823C0B501A40176956795579510
:109DC0004795FA01EC7FAF014C58574FFA012591A6
:109DD0003491FA01329665917491E82DE770E69F0F
:109DE000A001E79F500D1124F3E056954795FA9591
:109DF000E1F7241B350B4901A12CB12C880D991DCD
:109E0000AA1DBB1D8093B3029093B402A093B50228
:109E1000B093B60238CDE0E28E2E912CA12CB12C5D
:109E2000A0CFAC01BD017695679557954795FA018E
:109E3000EC7FAF014C58574FFA0125913491FA014C
:109E40003296459154918770849FB001859F700D23
:109E50001124CB0143E0969587954A95E1F7A90136
:109E6000481B590BCA01A0E0B0E0FDCC80E290E0B5
:109E7000A0E0B0E0CDCCAC01BD01769567955795DB
:109E80004795FA01EC7F9F012C58374FF9018590D7
:109E90009490F9013296259134918770829FA001A8
:109EA000839F500D1124CA0123E0969587952A952A
:109EB000E1F7881A990AA12CB12C7ACE80E290E0C1
:109EC000A0E0B0E04ECECF92DF92EF92FF92CF9320
:109ED000DF936A017B01FC018491EF0121968823C5
:109EE00021F00E940283FE01F7CF4AE0C701B601CC
:109EF000DF91CF91FF90EF90DF90CF900C94AA85E7
:109F0000CF92DF92EF92FF92CF93DF936A017B01B2
:109F1000FC018491EF012196882321F00E940283A5
:109F2000FE01F7CF42E0C701B601DF91CF91FF906C
:109F3000EF90DF90CF900C942E860F931F93CF93CA
:109F4000DF938B01FC018491EF012196882321F09E
:109F50000E940283FE01F7CFB801110F880B990B05
:109F6000DF91CF911F910F910C9412860F931F9345
:109F7000CF93DF9300D0CDB7DEB7FC0184918F0182
:109F80000F5F1F4F811102C08B0108C069837A8364
:109F90000E940283F80169817A81F0CFF8018191F2
:109FA0008F01882319F00E940283F8CF0F900F9041
:109FB000DF91CF911F910F91089586E40E94A882AE
:109FC00080936909882351F00E947582609329016A
:109FD00070932A0180932B0190932C0183E50E94BA
:109FE000A882882351F00E9475826093310170939A
:109FF0003201809333019093340182E40E94A8825D
:10A00000882351F00E94758260932D0170932E0178
:10A0100080932F019093300108958F929F92AF9279
:10A02000BF92CF92DF92EF92FF920F931F93CF9345
:10A03000DF9300D000D0CDB7DEB78BEB882E81E167
:10A04000982E93EAA92E91E1B92E0BE71CE0C12CC2
:10A05000D12C7601C394F401619171918191919118
:10A060004F01F50121913191419151915F01298376
:10A070003A834B835C830E94B0E529813A814B810E
:10A080005C810E9411E60E944FEBF801619371938D
:10A09000819391938F01C616D706E806F90610F44E
:10A0A0006B017C01FBEC8F16F1E19F06A1F66FEFCF
:10A0B0007FEFCB01A70196010E949FE920938B0CB3
:10A0C00030938C0C40938D0C50938E0C0F900F900E
:10A0D0000F900F90DF91CF911F910F91FF90EF9014
:10A0E000DF90CF90BF90AF909F908F900895809118
:10A0F0006C0690916D06891B8F708F3019F40E9449
:10A1000014D3F5CF80916C068F5F8F70E0916C0651
:10A110009DE49E9FF0011124EE52F34FDF011D924A
:10A120009A95E9F798E090834091820650918306D2
:10A130006091840670918506458B568B678B708F76
:10A140004091860650918706609188067091890635
:10A15000418F528F638F748F40918A0650918B0686
:10A1600060918C0670918D06458F568F678F70A316
:10A1700040918E0650918F066091900670919106E5
:10A1800041A352A363A374A320916C0690916D0622
:10A19000291303C094E69093690680936C0680911E
:10A1A0006F00826080936F00089590916C0680919B
:10A1B0006D06981719F00E9414D3F7CF8091B31150
:10A1C0009091B411892BB9F70895EF92FF920F93F4
:10A1D0001F93CF93DF937B018A01E9012091A311A3
:10A1E0003091A4114091A5115091A611FC016081FC
:10A1F0007181828193810E9411E60E9449EC6093F3
:10A20000820670938306809384069093850620913E
:10A21000A7113091A8114091A9115091AA11F701ED
:10A2200060817181828193810E9411E60E9449ECD4
:10A2300060938606709387068093880690938906BC
:10A2400020E030E0A901F801608171818281938171
:10A250000E94DCE92091AB113091AC114091AD111D
:10A260005091AE110E9411E60E9449EC60938A065B
:10A2700070938B0680938C0690938D062091AF117E
:10A280003091B0114091B1115091B2116881798132
:10A290008A819B810E9411E60E9449EC60938E06A0
:10A2A00070938F06809390069093910690916C0620
:10A2B00080916D06981741F0DF91CF911F910F911A
:10A2C000FF90EF900C9477500E94D55080916F00D2
:10A2D00081FB992790F981FF05C080916F008D7FE8
:10A2E00080936F00409182065091830660918406AE
:10A2F00070918506409311125093121260931312BD
:10A3000070931412409186065091870660918806DA
:10A31000709189064093151250931612609317128C
:10A320007093181240918A0650918B0660918C06AA
:10A3300070918D064093191250931A1260931B125C
:10A3400070931C1240918E0650918F06609190067A
:10A350007091910640931D1250931E1260931F122C
:10A3600070932012992329F080916F00826080936E
:10A370006F00DF91CF911F910F91FF90EF900895A3
:10A380000F931F93CF93DF93C3EAD1E103EB1CE05C
:10A39000299139914991599160E070E080E89FE3FB
:10A3A0000E94D6EAF80161937193819391938F0192
:10A3B000F1E1C33BDF0761F724E733E040E753E017
:10A3C0006CE673E088E693E00E94E550DF91CF9160
:10A3D0001F910F910C940D5090916C0680916D0619
:10A3E000981719F00E9414D3F7CF8091B311909170
:10A3F000B411892BB9F70C94C5D5CF93DF93909105
:10A400006F0091FB222720F991FF05C090916F000A
:10A410009D7F90936F0094E0899FE0011124FE01DD
:10A42000EB5FFD4E6081718182819381222329F04F
:10A4300020916F00226020936F000E94B2E5CD54FE
:10A44000D34F288139814A815B810E9411E6DF91D7
:10A45000CF910895CF92DF92EF92FF920F931F93C7
:10A46000CF93DF9300D000D0CDB7DEB78091CF116E
:10A470009091D011A091D111B091D211B7FF08C025
:10A480001092CF111092D0111092D1111092D211BE
:10A490008091D3119091D411A091D511B091D61182
:10A4A0004091CF115091D0116091D1117091D21182
:10A4B00084179507A607B70744F48093CF119093AC
:10A4C000D011A093D111B093D21180914201882371
:10A4D00079F14091CF115091D0116091D1117091CB
:10A4E000D2118091D7119091D811A091D911B0912A
:10A4F000DA116A017B01C80ED91EEA1EFB1EC701D4
:10A50000B6010E94B0E520E030E048EC52E40E9441
:10A5100011E669837A838B839C83CE0101960E9426
:10A520002045BC018091DD119091DE110E947B637A
:10A530001091E30211110AC08091DF11882309F400
:10A5400042C080914201882309F43DC04091CF115F
:10A550005091D0116091D1117091D2118091D71189
:10A560009091D811A091D911B091DA116A017B01B3
:10A57000C80ED91EEA1EFB1EC701B6010E94B0E537
:10A5800020E030E048EC52E40E9411E60E944FEBDC
:10A59000E091DB11F091DC11309721F06083718341
:10A5A00082839383E091E011F091E111309731F0D3
:10A5B0008091DF11811101C0111109958091E30291
:10A5C00081110E9464631092E3020F900F900F902C
:10A5D0000F90DF91CF911F910F91FF90EF90DF903F
:10A5E000CF900895CF92DF92EF92FF920F931F9337
:10A5F000CF93DF9300D000D0CDB7DEB78091CF11DD
:10A600009091D011A091D111B091D211B7FF08C093
:10A610001092CF111092D0111092D1111092D2112C
:10A620008091D3119091D411A091D511B091D611F0
:10A630004091CF115091D0116091D1117091D211F0
:10A6400084179507A607B70744F48093CF1190931A
:10A65000D011A093D111B093D211809142018823DF
:10A6600079F14091CF115091D0116091D111709139
:10A67000D2118091D7119091D811A091D911B09198
:10A68000DA116A017B01C80ED91EEA1EFB1EC70142
:10A69000B6010E94B2E520E030E048EC52E40E94AE
:10A6A00011E669837A838B839C83CE0101960E9495
:10A6B0002045BC018091DD119091DE110E947B63E9
:10A6C0001091E302111109C08091DF11882309F470
:10A6D0003FC0809142018823D9F14091CF11509120
:10A6E000D0116091D1117091D2118091D7119091B8
:10A6F000D811A091D911B091DA116A017B01C80E6D
:10A70000D91EEA1EFB1EC701B6010E94B2E520E079
:10A7100030E048EC52E40E9411E6E091DB11F09148
:10A72000DC11309721F06083718382839383E09101
:10A73000E011F091E111309731F08091DF1181113A
:10A7400001C0111109958091E30281110E94646397
:10A750001092E3020F900F900F900F90DF91CF9126
:10A760001F910F91FF90EF90DF90CF900895CF92BF
:10A77000DF92EF92FF920F931F93CF93DF9300D05E
:10A7800000D0CDB7DEB78091CF119091D011A091BC
:10A79000D111B091D211B7FF08C01092CF11109211
:10A7A000D0111092D1111092D2118091D3119091A9
:10A7B000D411A091D511B091D6114091CF115091E3
:10A7C000D0116091D1117091D21184179507A6070D
:10A7D000B70744F48093CF119093D011A093D11177
:10A7E000B093D21180914201882379F14091CF1129
:10A7F0005091D0116091D1117091D2118091D711E7
:10A800009091D811A091D911B091DA116A017B0110
:10A81000C80ED91EEA1EFB1EC701B6010E94B2E592
:10A820002AE037ED43E25CE30E9411E669837A8314
:10A830008B839C83CE0101960E94BE43BC01809114
:10A84000DD119091DE110E947B631091E3021111E2
:10A8500009C08091DF11882309F43FC08091420133
:10A860008823D9F14091CF115091D0116091D1112D
:10A870007091D2118091D7119091D811A091D911D6
:10A88000B091DA116A017B01C80ED91EEA1EFB1EC7
:10A89000C701B6010E94B2E52AE037ED43E25CE36E
:10A8A0000E9411E6E091DB11F091DC11309721F06C
:10A8B0006083718382839383E091E011F091E111D1
:10A8C000309731F08091DF11811101C0111109958C
:10A8D0008091E30281110E9464631092E3020F9061
:10A8E0000F900F900F90DF91CF911F910F91FF90DC
:10A8F000EF90DF90CF900895CF92DF92EF92FF928A
:10A900000F931F93CF93DF9300D000D0CDB7DEB766
:10A910008091CF119091D011A091D111B091D2110D
:10A92000B7FF08C01092CF111092D0111092D11120
:10A930001092D2118091D3119091D411A091D51180
:10A94000B091D6114091CF115091D0116091D11199
:10A950007091D21184179507A607B70744F4809326
:10A96000CF119093D011A093D111B093D2118091B7
:10A970004201882379F14091CF115091D01160911B
:10A98000D1117091D2118091D7119091D811A091CD
:10A99000D911B091DA116A017B01C80ED91EEA1EE5
:10A9A000FB1EC701B6010E94B2E52AE037ED43E283
:10A9B0005CE30E9411E669837A838B839C83CE01DA
:10A9C00001960E947F44BC018091DD119091DE11BF
:10A9D0000E947B631091E302111109C08091DF1185
:10A9E000882309F43FC0809142018823D9F1409126
:10A9F000CF115091D0116091D1117091D2118091ED
:10AA0000D7119091D811A091D911B091DA116A01A2
:10AA10007B01C80ED91EEA1EFB1EC701B6010E94AB
:10AA2000B2E52AE037ED43E25CE30E9411E6E091F3
:10AA3000DB11F091DC11309721F060837183828308
:10AA40009383E091E011F091E111309731F0809122
:10AA5000DF11811101C0111109958091E30281116B
:10AA60000E9464631092E3020F900F900F900F907A
:10AA7000DF91CF911F910F91FF90EF90DF90CF90DA
:10AA80000895CF92DF92EF92FF920F931F93CF938F
:10AA9000DF9300D000D0CDB7DEB78091CF11909179
:10AAA000D011A091D111B091D211B7FF08C010926E
:10AAB000CF111092D0111092D1111092D211809119
:10AAC000D3119091D411A091D511B091D61140918C
:10AAD000CF115091D0116091D1117091D211841782
:10AAE0009507A607B70744F48093CF119093D01130
:10AAF000A093D111B093D21180914201882379F1B2
:10AB00004091CF115091D0116091D1117091D2111B
:10AB10008091D7119091D811A091D911B091DA11EB
:10AB20006A017B01C80ED91EEA1EFB1EC701B601D1
:10AB30000E94B2E52FE632E143E85AE30E9411E6B3
:10AB400069837A838B839C83CE0101960E9484C0A3
:10AB5000BC018091DD119091DE110E947B63109108
:10AB6000E302111109C08091DF11882309F43FC06D
:10AB7000809142018823D9F14091CF115091D01199
:10AB80006091D1117091D2118091D7119091D8110B
:10AB9000A091D911B091DA116A017B01C80ED91EBA
:10ABA000EA1EFB1EC701B6010E94B2E52FE632E1A4
:10ABB00043E85AE30E9411E6E091DB11F091DC11C9
:10ABC000309721F06083718382839383E091E01159
:10ABD000F091E111309731F08091DF11811101C0C6
:10ABE000111109958091E30281110E946463109212
:10ABF000E3020F900F900F900F90DF91CF911F9174
:10AC00000F91FF90EF90DF90CF900895CF92DF9259
:10AC1000EF92FF920F931F93CF93DF9300D000D05A
:10AC2000CDB7DEB78091CF119091D011A091D11105
:10AC3000B091D211B7FF08C01092CF111092D0116D
:10AC40001092D1111092D2118091D3119091D41100
:10AC5000A091D511B091D6114091CF115091D01142
:10AC60006091D1117091D21184179507A607B7078B
:10AC700044F48093CF119093D011A093D111B0934D
:10AC8000D21180914201882379F14091CF115091E6
:10AC9000D0116091D1117091D2118091D711909102
:10ACA000D811A091D911B091DA116A017B01C80EB7
:10ACB000D91EEA1EFB1EC701B6010E94B2E52AE0BA
:10ACC00037ED43E25CE30E9411E669837A838B836C
:10ACD0009C83CE0101960E945046BC018091DD11FB
:10ACE0009091DE110E947B631091E302111109C063
:10ACF0008091DF11882309F43FC0809142018823AD
:10AD0000D9F14091CF115091D0116091D111709132
:10AD1000D2118091D7119091D811A091D911B091F1
:10AD2000DA116A017B01C80ED91EEA1EFB1EC7019B
:10AD3000B6010E94B2E52AE037ED43E25CE30E94EF
:10AD400011E6E091DB11F091DC11309721F0608386
:10AD5000718382839383E091E011F091E111309748
:10AD600031F08091DF11811101C01111099580919D
:10AD7000E30281110E9464631092E3020F900F902E
:10AD80000F900F90DF91CF911F910F91FF90EF9057
:10AD9000DF90CF900895CF92DF92EF92FF920F93C2
:10ADA0001F93CF938091CF119091D011A091D11189
:10ADB000B091D211B7FF08C01092CF111092D011EC
:10ADC0001092D1111092D2118091D3119091D4117F
:10ADD000A091D511B091D6114091CF115091D011C1
:10ADE0006091D1117091D21184179507A607B7070A
:10ADF00044F48093CF119093D011A093D111B093CC
:10AE0000D211809142018823E1F14091CF115091FC
:10AE1000D0116091D1117091D2118091D711909180
:10AE2000D811A091D911B091DA118A019B01080FB4
:10AE3000191F2A1F3B1FC901B8010E94B2E56B010F
:10AE40007C0120E030E0A9010E94ABE587FD05C050
:10AE500020E030E040E05FE304C020E030E040E08C
:10AE60005FEBC701B6010E94DCE90E9448EBCB0111
:10AE70000E945547BC018091DD119091DE110E9426
:10AE80007B63C091E302C11108C08091DF11882368
:10AE9000C9F1809142018823A9F14091CF115091CD
:10AEA000D0116091D1117091D2118091D7119091F0
:10AEB000D811A091D911B091DA118A019B01080F24
:10AEC000191F2A1F3B1FC901B8010E94B2E5E0917A
:10AED000DB11F091DC11309721F060837183828364
:10AEE0009383E091E011F091E111309731F080917E
:10AEF000DF11811101C0C11109958091E302811117
:10AF00000E9464631092E302CF911F910F91FF9012
:10AF1000EF90DF90CF9008958091CF119091D01154
:10AF2000A091D111B091D211B7FF08C01092CF11EA
:10AF30001092D0111092D1111092D2118091D31190
:10AF40009091D411A091D511B091D6114091CF110B
:10AF50005091D0116091D1117091D2118417950741
:10AF6000A607B70744F48093CF119093D011A09314
:10AF7000D111B093D21180914201882399F0209190
:10AF8000D7113091D8118091CF119091D011820FAB
:10AF9000931F0E945547BC018091DD119091DE11F5
:10AFA0000E947B632091E302211108C08091DF1190
:10AFB000882339F180914201882319F14091D711FA
:10AFC0005091D8118091CF119091D011840F951F7D
:10AFD000E091DB11F091DC11309711F091838083C7
:10AFE000E091E011F091E111309731F08091DF11A3
:10AFF000811101C0211109958091E30281110E9404
:10B0000064631092E3020895CF92DF92EF92FF9271
:10B010006B017C0183E3C816D104E104F10470F0F4
:10B0200082E3C81AD108E108F10862E370E080E029
:10B0300090E00E94DE3F0E945AD1ECCFC701B601DA
:10B040000E94DE3FFF90EF90DF90CF900C945AD19A
:10B050000F931F93CF93DF9300D000D000D0CDB7D4
:10B06000DEB783E992E09E838D8304E610E01A83C5
:10B070000983BE016B5F7F4FCE0101960E945B7713
:10B080008AEB92E09C838B831A830983BE016D5FF8
:10B090007F4FCE0101960E945B7726960FB6F894FB
:10B0A000DEBF0FBECDBFDF91CF911F910F910895ED
:10B0B0000F931F93CF93DF93982F862F8A01D22F60
:10B0C000692F0E94B46D909163068091CE1189170B
:10B0D00048F1909165068091CD11981718F1C4E15F
:10B0E000F8018491882331F00E94116EC81B0F5F14
:10B0F0001F4FF6CFCC2329F080E20E949B72C150F3
:10B10000F9CF8091CE119AE79093660680936706F7
:10B110008D2F0E94296E80E2DF91CF911F910F91B8
:10B120000C949B72DF91CF911F910F91089584E948
:10B1300090E10E94BD7281E08093E60208950F9332
:10B140001F930E9418400091F5021091F602209181
:10B15000F7023091F802DC01CB01801B910BA20BAE
:10B16000B30BB7FD0CC089B183FB992790F981E03F
:10B1700089274A9B8260309B84608093F40280918F
:10B18000F40281709091F40291FD82609091F3023B
:10B19000891731F18130A9F028F0823041F08330F5
:10B1A00059F01CC0913089F0923099F017C0992362
:10B1B00061F0933071F012C0913059F0923071F417
:10B1C00004C0992331F0933049F49091F2029F5FCB
:10B1D00003C09091F20291509093F2028093F30297
:10B1E0001F910F9108950F931F93CF93DF938C01BD
:10B1F00067FF03C010926A0C60E080916A0C90E0D7
:10B20000262F062E000C330B281739071CF16093EC
:10B210006A0CC8010E94F8E4F801E80FF91FEF0179
:10B22000C01BD10BC334D10534F031978491807C9D
:10B230008038D9F3F4CFDD27AE01B80187E29CE076
:10B240000E9419E5C95DD34F188283E080934201C3
:10B250001092260CDF91CF911F910F910895CF93FB
:10B26000DF9320916A0C211120C0FC010190002085
:10B27000E9F73197EF01C81BD90BC334D10534F07E
:10B2800031972081207C2038D9F3F4CFBC01DD2711
:10B29000AE0187E29CE00E94ABEDC95DD34F1882FE
:10B2A00083E0809342011092260CDF91CF910895A4
:10B2B0004F925F926F927F928F929F92AF92BF92C6
:10B2C000CF92DF92EF92FF920F931F93CF93DF9372
:10B2D000CDB7DEB72A970FB6F894DEBF0FBECDBF4D
:10B2E00010910D011F3F09F44BC00E941840C090FF
:10B2F000D702D090D802E090D902F090DA02DC01B7
:10B30000CB018C199D09AE09BF09B7FD39C09091D9
:10B310006D0680916C068F5F8F70981789F11330DE
:10B3200009F43BC2E090D60224E01202F00111249D
:10B33000E65AFE4F20E030E040E752E46081718140
:10B34000828193810E94D6EA69837A838B839C836E
:10B350001D821E821F821886AE014B5F5F4F6A01FD
:10B360008E010F5F1F4F24E733E040E753E06CE6A8
:10B3700073E088E693E00E94F9978FEF80930D01C8
:10B380000E949F588091F40282FF44C08091F10294
:10B39000811142C091E09093F1022091E5022111C8
:10B3A00003C08091E40289278093E3021092E502B2
:10B3B00083E0809342011092F4020E941840DC0165
:10B3C000CB018C509E4FAF4FBF4F8093F5029093AF
:10B3D000F602A093F702B093F80288E893E19A8707
:10B3E000898782E090E09A838983BE01675F7F4FFF
:10B3F000CE0101960E945B7716E0115069F082E958
:10B4000096E00E94AB7E62E070E080E090E00E94F7
:10B41000DE3FF3CF1092F1020E9418406B017C01D5
:10B420008091ED029091EE02A091EF02B091F002B6
:10B43000A7019601281B390B4A0B5B0B57FF05C070
:10B440008091E202882309F4F2C1D701C6018C5928
:10B450009F4FAF4FBF4F8093ED029093EE02A093AA
:10B46000EF02B093F0028091F202082E000C990BCB
:10B4700097FF03C091958195910984302CF48091B8
:10B48000E302811194C0A4C08091E102882309F4F1
:10B4900067C08091F2028090DD029090DE02A09061
:10B4A000DF02B090E00281149104A104B10409F418
:10B4B0004AC0082E000C990B97FF03C09195819507
:10B4C0009109682F87FF02C063E0680F6595659555
:10B4D000062E000C770B880B990B0E94B2E52B010E
:10B4E0003C01C701B601681979098A099B090E94C4
:10B4F000B0E59B01AC01C301B2010E94D6EA20E095
:10B5000030E04AE754E40E9411E64B015C0120E080
:10B5100030E040E253E40E943CEC87FF0FC020E0A3
:10B5200030E046E952E4C501B4010E943CEC87FDDD
:10B530000AC02AE030E040E050E009C024E630E0F4
:10B5400040E050E004C021E030E040E050E0C09234
:10B55000DD02D092DE02E092DF02F092E00204C04F
:10B5600021E030E040E050E0A091F2020A2E000C11
:10B57000BB0B0E9439ED24E030E040E050E00E9437
:10B5800011ED8091CF119091D011A091D111B09176
:10B59000D211820F931FA41FB51F8093CF119093D8
:10B5A000D011A093D111B093D2111092F202D70111
:10B5B000C6018856954CAF4FBF4F8093E9029093D8
:10B5C000EA02A093EB02B093EC0281E08093420187
:10B5D00020914A0130914B014DE52F37340741F45A
:10B5E00080914901882309F4DAC081508093490190
:10B5F0002E57374671F48091CB119091CC11891759
:10B6000040F490914901992309F4D9C09150909345
:10B61000490180916F0081FB222720F981FF05C03D
:10B6200080916F008D7F80936F008091AB0C909123
:10B63000AC0CA091AD0CB091AE0C222329F020915E
:10B640006F00226020936F003AE0B695A79597951A
:10B6500087953A95D1F7009721E0A207B10520F030
:10B660008FEF9FEFA0E0B0E0969587952091420183
:10B67000211105C03091E2023111D5C059C00097A7
:10B6800041F04091E7025091E8024817590708F04D
:10B690004FC08091E202811113C0223050F024305B
:10B6A00028F0243031F41092420103C081E08093ED
:10B6B00042010E940A7381E08093DC028093E202DF
:10B6C00084E00E94F76D81E080934F06E0914A018B
:10B6D000F0914B0109951092DC028091E2028823DF
:10B6E00051F00E94617291E0811101C090E090934D
:10B6F000E20291117CC01092E3028090E7029090E8
:10B70000E802A12CB12C0E941840DC01CB018C195D
:10B710009D09AE09BF0988169906AA06BB0640F422
:10B720000E9418406C197D097093E8026093E7024B
:10B7300080914A0190914B018F579D4521F0809156
:10B74000DB02882379F048E9C40E4AE3D41EE11CE9
:10B75000F11CC092E902D092EA02E092EB02F09270
:10B76000EC020FC08091E9029091EA02A091EB02F5
:10B77000B091EC02C81AD90AEA0AFB0AF7FE0E9445
:10B780005D638091E202811152C08091420181305B
:10B7900009F04DC0109242014AC0E12CC5CD8CE0A9
:10B7A000809349018091E7029091E802019790937C
:10B7B000E8028093E70281E08093420119CF96E08E
:10B7C0009093490191E0909342018F5F8093CB1158
:10B7D000D701C6018856954CAF4FBF4F8093E90201
:10B7E0009093EA02A093EB02B093EC0212CF809008
:10B7F000E7029090E802A12CB12C0E941840DC01D5
:10B80000CB018C199D09AE09BF0988169906AA06B5
:10B81000BB0668F40E9418406C197D097093E80219
:10B820006093E70204C0009709F44ACF2ACF2A9612
:10B830000FB6F894DEBF0FBECDBFDF91CF911F9141
:10B840000F91FF90EF90DF90CF90BF90AF909F90BF
:10B850008F907F906F905F904F900895FC0180E0F3
:10B8600090E02491222339F02491207C203809F0A3
:10B8700001963196F6CF0895FC0120E030E09191D9
:10B88000992331F0907C9038D1F32F5F3F4FF7CF61
:10B89000C9010895CF93DF931F92CDB7DEB7809192
:10B8A0006806811107C081E0809368068FE296E008
:10B8B0000E94BC41609131067091320619829E014E
:10B8C0002F5F3F4F4FE08FE296E00E943741539841
:10B8D0005B9A52985A9A3898409A0E949F581092B0
:10B8E000F2020F90DF91CF910895CF93DF9300D0B4
:10B8F000CDB7DEB789839A830E94EA5C40E050E0CE
:10B90000BA0189819A810F900F90DF91CF910C94A9
:10B910000A5D282F1092E1028091CF119091D011F1
:10B92000A091D111B091D21181309048A105B105FB
:10B9300040F01092CF111092D0111092D1111092AC
:10B94000D2118091DC02882331F08091CF11809355
:10B95000090510920805809107051816FCF4082EB9
:10B96000000C990B821B910920910905022E000CF5
:10B97000330B2817390794F097FF02C080E090E05E
:10B9800080930905092E000CAA0BBB0B8093CF11E5
:10B990009093D011A093D111B093D2118091090549
:10B9A0006623A9F090910A05891714F480930A057B
:10B9B00020910A05022E000C330B2C5F3F4F482FBD
:10B9C000082E000C550B241735071CF48450809367
:10B9D0000A050895809126038630D8F496E0899F61
:10B9E000F0011124EE5FFC4F20914A0130914B0190
:10B9F000318320834091CF115091D0116091D111AA
:10BA00007091D21142835383648375838F5F8093D7
:10BA100026030895CF92DF92EF92FF920F931F9328
:10BA2000CF93DF93EC016A017B0180914A019091F1
:10BA30004B018C179D0709F459C024ECC233D2077F
:10BA4000A1F48F579D45B9F50E941840DC01CB0148
:10BA50008E519B4FAF4FBF4F8093FE029093FF02DA
:10BA6000A0930003B093010326C02DE5CF37D20782
:10BA700011F58253944CF9F40E9418400091FE0293
:10BA80001091FF022091000330910103DC01CB01F2
:10BA9000801B910BA20BB30BB7FF0DC080916C06FE
:10BAA00090916D06891B8F7021F48091B2068823D6
:10BAB00011F0C6EDD1ECD0934B01C0934A01C09276
:10BAC000CF11D092D011E092D111F092D211CF5774
:10BAD000DD4521F41092DB021092260382E0809370
:10BAE000420181E0809308051092E202DF91CF913C
:10BAF0001F910F91FF90EF90DF90CF9008954F929C
:10BB00005F926F927F92BF92CF92DF92EF92FF92FD
:10BB10000F931F93CF93DF93CDB7DEB72A970FB65E
:10BB2000F894DEBF0FBECDBF1092E1028091E30218
:10BB30001092E302882311F11091D40280916806DB
:10BB4000811107C081E0809368068FE296E00E9431
:10BB5000BC41609131067091320619839E012F5FBE
:10BB60003F4F4FE08FE296E00E94374140E050E0C7
:10BB7000BA0182E394EC0E940A5D8BC520914E01CC
:10BB800030914F014091CF115091D0116091D1115E
:10BB90007091D211C901840F951F2436310524F408
:10BBA000853691053CF416C02436310531F08436D3
:10BBB000910584F484E690E00DC04730510561059D
:10BBC000710514F0069706C04A3F5F4F6F4F7F4FD5
:10BBD0006CF4069690934F0180934E011092CF1112
:10BBE0001092D0111092D1111092D21180914E0169
:10BBF00090914F018A3091053CF0883E43E09407D4
:10BC00002CF087EE93E002C08AE090E090934F0121
:10BC100080934E010E94184000912803109129033F
:10BC200020912A0330912B036B017C01C01AD10AA9
:10BC3000E20AF30AF7FC13C0209127032095209312
:10BC40002703DC01CB018A549C4FAF4FBF4F809339
:10BC5000280390932903A0932A03B0932B03BB24BA
:10BC6000B39480912703811101C0B12C0E94975891
:10BC700080916306853198F4BB2049F08091CB0C0C
:10BC80009091CC0C892B19F004E816E102C004E570
:10BC900015E123E140E161E080E00E9462BF809114
:10BCA00063068D3108F0FCC0883070F56091E411B6
:10BCB0007091E511072E000C880B990B0E94B2E5DC
:10BCC00020E030E040E05FE30E94DCE90E9448EBC6
:10BCD000CB010E945547FC012081203229F42181AB
:10BCE000203221F436E003C030E001C033E026E228
:10BCF000231B2093660627E0209367060E944C6E64
:10BD000081E595E10E943E6E809163068D31A0F53C
:10BD100080916506853180F120E030E040E05FE30E
:10BD20006091CE0C7091CF0C8091D00C9091D10C81
:10BD30000E94DCE90E9448EBCB010E945547FC01C0
:10BD40008081803209F0C0C28181803209F0B5C2A1
:10BD500096E086E2891B809366068CE180936706F5
:10BD6000CF010E944C6E81E595E10E943E6E80916C
:10BD70006306853108F4A3C280916306883070F5AC
:10BD80006091E2117091E311072E000C880B990B62
:10BD90000E94B2E520E030E040E05FE30E94DCE991
:10BDA0000E9448EBCB010E945547FC0120812032C4
:10BDB00029F42181203221F436E003C030E001C0B3
:10BDC00033E029E4231B2093660627E020936706CF
:10BDD0000E944C6E81E595E10E943E6E8091630663
:10BDE0008D31A0F580916506853180F120E030E04D
:10BDF00040E05FE36091FA027091FB028091FC02E7
:10BE00009091FD020E94DCE90E9448EBCB010E9468
:10BE10005547FC018081803209F08CC281818032DB
:10BE200009F081C296E089E4891B809366068CE163
:10BE300080936706CF010E944C6E81E595E10E94D8
:10BE40003E6E80916306853108F46FC2809163066F
:10BE50008C3130F580916506843110F18091CB0CE6
:10BE60009091CC0C019644E6489F9001499F300D7B
:10BE7000112437FF02C021503F4F832F932F990F7A
:10BE8000990B009769F027E6209366062BE1209333
:10BE900067060E9455470E944C6E85E20E949B7285
:10BEA0008091A408882349F080916306843328F4A4
:10BEB000809165068A3208F06CC2809163068533F2
:10BEC00028F480916506813308F08BC28091A40824
:10BED000882369F180914E0990914F09A0915009F2
:10BEE000B09151090097A105B10509F1BC01CD013F
:10BEF0006D597F4F8F4F9F4F24E630E040E050E078
:10BF00000E949FE9609152097091530980915409F0
:10BF1000909155090E949FE9223048F08091630674
:10BF2000843328F480916506823308F061C28091E1
:10BF30006306813308F060C080916506893208F499
:10BF40005BC00E9445CF2B013C018CE3C82ED12C55
:10BF5000E12CF12CC301B201A70196010E949FE9D7
:10BF6000CA01B901A70196010E949FE9CA01F62EF4
:10BF7000E72E69018E010F5F1F4FE0E84E16E1E5E5
:10BF80005E06E1E06E06710408F44DC2B90128E1D5
:10BF900030E040E050E00E949FE929013A01EF9231
:10BFA000FF92C60168E170E00E94E9EC9F938F93D5
:10BFB0005F924F9281E395E19F938F931F930F932D
:10BFC0000E9442E50FB6F894DEBF0FBECDBF9AE0E7
:10BFD000491651046104710408F04FC298E0892F9A
:10BFE000880F980F9195955A9093660680E38093F9
:10BFF0006706C8010E944C6EE0912906F0912A065E
:10C00000848181112FC12091FC093091FD0940915B
:10C01000FE095091FF096091680370916903809156
:10C020006A0390916B030E94DCE96B017C0120E0C4
:10C0300030E0A9010E94ABE587FD05C020E030E0BB
:10C0400040E05FE304C020E030E040E05FEBC70188
:10C05000B6010E94DCE90E9448EBCB010E94EE464B
:10C06000BC0189E393E00E9496ED2091000A309193
:10C07000010A4091020A5091030A60916C03709189
:10C080006D0380916E0390916F030E94DCE96B0158
:10C090007C0120E030E0A9010E94ABE587FD05C0EE
:10C0A00020E030E040E05FE304C020E030E040E02A
:10C0B0005FEBC701B6010E94DCE90E9448EBCB01AF
:10C0C0000E94EE46BC0184E393E00E9496ED20912D
:10C0D000040A3091050A4091060A5091070A6091BE
:10C0E00070037091710380917203909173030E94A9
:10C0F000DCE96B017C0120E030E04AE754E40E9477
:10C1000011E62B013C0120E030E0A901C701B60196
:10C110000E94ABE587FD05C020E030E040EA50E436
:10C1200004C020E030E040EA50ECC301B2010E94BC
:10C13000DCE920E030E040E251E40E94D6EA0E94CF
:10C1400048EB6B017C0197FD16C06031F7E27F0779
:10C1500081059105D4F020E137E240E050E00E94F3
:10C1600011EDCA01B9012AE030E040E050E00E9440
:10C1700011ED605D0BC0F094E094D094C094C11CAC
:10C18000D11CE11CF11C6DE201C060E26093E7117B
:10C1900028EEC21623E0D206E104F10494F0C701B0
:10C1A000B60128EE33E040E050E00E9411EDCA01F4
:10C1B000B9012AE030E040E050E00E9411ED605DFE
:10C1C00001C060E26093E811C701B60124E630E0E7
:10C1D00040E050E00E9411ED6AE0462E512C612CA7
:10C1E000712CCA01B901A30192010E9411ED605D99
:10C1F0006093E911C701B601A30192010E9411EDFC
:10C200006B017C01672B682B692B79F08EE28093A0
:10C21000EA11CA01B901A30192010E9411ED605D0A
:10C220006093EB1180E38C0D15C0CA01B901A30125
:10C2300092010E9411ED662339F08EE28093EA119B
:10C24000605D6093EB1105C080E28093EB118093F9
:10C25000EA1180E28093EC1167EE71E18DE293E0E8
:10C260000E9496ED80916306883298F4809165066D
:10C270008D3178F02BE040E86DE180E00E944AC00B
:10C2800080916306873228F4809165068F3108F02B
:10C29000F6C080916306823328F4809165068B3264
:10C2A00008F07CC180916306803408F0F2C180916F
:10C2B0006506883308F091C1ECC193E04ACD8091C6
:10C2C0006506813118F458CD90E043CD6091E411BA
:10C2D0007091E511072E000C880B990B0E94B2E5B6
:10C2E0002091CE0C3091CF0C4091D00C5091D10CBC
:10C2F0000E943CEC181674F410924F0602E022E003
:10C3000041E16EE28FE296E00E94574281E0809325
:10C310004F0632CD02E022E041E16EE28FE296E08C
:10C320000E94574229CD93E07ECD809165068131F0
:10C3300018F48CCD90E077CD6091E2117091E3110B
:10C34000072E000C880B990B0E94B2E52091FA028F
:10C350003091FB024091FC025091FD020E943CECA6
:10C36000181674F410924F0602E022E042E160E5F4
:10C370008FE296E00E94574281E080934F0666CD9F
:10C3800002E022E042E160E58FE296E00E9457423F
:10C390005DCD07E028E04AE26AE28FE296E00E9483
:10C3A000574205E022E04CE262E38FE296E00E9411
:10C3B000574224E04AE061E38AE20E944AC0609169
:10C3C00031067091320682E380934B068BE28093B4
:10C3D0004C062BE436E042E38FE296E00E943741C0
:10C3E0006CCD24E04AE461E386E30E944AC06ECD4E
:10C3F00048E4249FB0011124072E000C880B990BF0
:10C400000E94B2E52AE037ED43E25CE30E9411E6C8
:10C410000E944FEB262F02E042E367E38FE296E0B3
:10C420000E94574284CDE4E6CE16D10498F4EF92F0
:10C43000FF923F932F9387E295E19F938F931F93F2
:10C440000F930E9442E50FB6F894DEBF0FBECDBF3A
:10C4500095E0C5CDEF92FF923F932F938FE195E149
:10C460009F938F931F930F930E9442E50FB6F8940A
:10C47000DEBF0FBECDBF96E0B2CD99E0B0CD83E078
:10C480008093660616E2109367068FE495E10E949A
:10C490003E6E8BE08093660610936706BB2029F002
:10C4A00089E393E00E944C6E19C08091F90280FDEF
:10C4B0000DC009E313E0F80181918F01882371F029
:10C4C0008F320CF08FE30E94296EF5CF80915B03D1
:10C4D00080FDE6CF8AE495E10E943E6E8BE2809378
:10C4E000660616E21093670688E495E10E943E6EA8
:10C4F00083E38093660610936706BB2029F084E3EC
:10C5000093E00E944C6E19C08091F90281FD0DC02C
:10C5100004E313E0F80181918F01882371F08F32D9
:10C520000CF08FE30E94296EF5CF80915B0381FDB3
:10C53000E6CF8AE495E10E943E6E83E5809366062D
:10C5400016E21093670686E495E10E943E6E8BE545
:10C550008093660610936706BB2029F08DE293E076
:10C560000E944C6E96CE8091F90282FD0EC00DE2C3
:10C5700013E0F80181918F01882309F48ACE8F326C
:10C580000CF08FE30E94296EF4CF80915B0382FD53
:10C59000E5CF8FE395E10E943E6E7BCE84E00E9462
:10C5A000F76D83E08093660612E31093670686E0DA
:10C5B0000E94296E0E9497588CE080936606109323
:10C5C000670680914E0190914F010E9455470E944D
:10C5D0004C6E85E20E949B7265CE109266068FE3D8
:10C5E0008093670687E29CE00E943C5CF82EF6E1AF
:10C5F000F81770F066E187E29CE00E94E36DF6E1D7
:10C60000FF1609F446C080E20E949B72F394F7CFB4
:10C610000091260C10E0095D134FC8010E943C5C9C
:10C62000E82E25E1C22E66E1C801CE1498F00E94E2
:10C63000E36D8EE20E949B7295E1D92EED1461F0BC
:10C640008EE20E949B7224E1E21631F064E16E19E1
:10C6500087E29CE00E94E36D80912C038B15C9F06A
:10C66000B0922C039091260C9F1588F481E0890FDD
:10C6700021E0280FE82FF0E0E95DF34F9081907CF6
:10C68000903811F4822FF4CF8093260C02C01092C0
:10C69000260C2A960FB6F894DEBF0FBECDBFDF91F1
:10C6A000CF911F910F91FF90EF90DF90CF90BF90AF
:10C6B0007F906F905F904F90089540E050E0BA01F6
:10C6C0008FE79DE50C940A5DE0912603EE2389F047
:10C6D000E150E093260386E0E89FF0011124EE5F2D
:10C6E000FC4F4281538164817581808191810C94DA
:10C6F0000A5D0C945D63AF92BF92CF92DF92EF928E
:10C70000FF920F931F93CF93DF935C016B010E9405
:10C710002E5CEC01C6010E943C5C04E110E0081BA9
:10C720001109DD270C171D071CF0FF24F39402C02C
:10C7300082E0F82E8091300690E06F2D70E06F5F00
:10C740007F4F0E94FDECE62EC6E0C60F8091630687
:10C75000C81750F04091650650E02C2F30E02B5068
:10C760003109421753079CF5D0E0C114D104C1F13F
:10C770008AE30E949B7282E0F8120FC0CE0D809176
:10C780006306C81768F12091650630E08C2F90E0B1
:10C790000B97281739071CF423C0DD2309F1902FCC
:10C7A000990F090F000F00936606C093670680E299
:10C7B0000E949B72C601DF91CF911F910F91FF9054
:10C7C000EF90DF90CF90BF90AF900C944C6E109292
:10C7D0006606C0936706C5010E94A672D1E0C5CF68
:10C7E000DF91CF911F910F91FF90EF90DF90CF904D
:10C7F000BF90AF900895CF92DF92EF92FF920F9388
:10C800001F93CF93DF936C017A018B01C0E0D0E0DE
:10C81000CE15DF0589F0D8016D918D01D601ED911E
:10C82000FC910190F081E02DC6010995892B11F44E
:10C830007E0102C02196ECCFC701DF91CF911F91FD
:10C840000F91FF90EF90DF90CF9008950E9441EDFF
:10C85000CF93DF93282F30E0F901EC56F74E849107
:10C86000F901EC58F74ED491F901EC5AF74EC49106
:10C87000CC2391F081110E94013FEC2FF0E0EE0FEC
:10C88000FF1FE65BF74EA591B491EC91ED2381E09B
:10C8900090E021F480E002C080E090E0DF91CF9151
:10C8A00008951F93CF93DF93282F30E0F901EC56C2
:10C8B000F74E8491F901EC58F74ED491F901EC5AF6
:10C8C000F74EC491CC23C9F0162F81110E94013F6D
:10C8D000EC2FF0E0EE0FFF1FE05CF74EA591B49156
:10C8E0008FB7F894111105C09C91ED2FE095E923C5
:10C8F00002C0EC91ED2BEC938FBFDF91CF911F9194
:10C9000008951F920F920FB60F9211240BB60F923B
:10C910002F933F934F935F936F937F938F939F9347
:10C92000AF93BF93EF93FF938091410390914203A4
:10C93000A0914303B0914403892B8A2B8B2B59F18F
:10C9400080914003E0913E03F0913F03908189275D
:10C9500080838091410390914203A0914303B09161
:10C960004403181619061A061B060CF045C08091E0
:10C97000410390914203A0914303B0914403019776
:10C98000A109B1098093410390934203A09343030B
:10C99000B093440331C080910E01E4EBF8E1E491DF
:10C9A0009FEF90930E01E13071F050F0E23089F08A
:10C9B000E330F9F4909171009D7F9093710019C05C
:10C9C00010926E0016C090916F009D7F90936F0043
:10C9D00010C0909170009D7F9093700091E09093B3
:10C9E000B0009091B100987F94609093B100109244
:10C9F000B30060E00E945164FF91EF91BF91AF914D
:10CA00009F918F917F916F915F914F913F912F9166
:10CA10000F900BBE0F900FBE0F901F9018951F9395
:10CA2000CF93DF9361E081E00E94895CD0910A0599
:10CA3000C0E0D1111EC010910905112331F0809181
:10CA40004201882309F47EC00DC08091E30288234F
:10CA5000B1F31092E3020E94646380910805882379
:10CA600071F378C081E0111180E024E045EF5EE1D0
:10CA700066C0D13009F510910905113031F080916F
:10CA80004201882309F45EC00FC08091E30288232D
:10CA9000B1F31092E3028FE696E60E94755C8091F6
:10CAA0000805882361F356C081E0113009F080E069
:10CAB00023E048EE5EE143C0D23001F51091090554
:10CAC000123029F0809142018823E1F10FC080915A
:10CAD000E3028823B9F31092E30281ED96E60E9407
:10CAE000755C80910805882369F334C081E01230B9
:10CAF00009F080E023E04DED5EE121C0D33011F577
:10CB000010910905133029F0809142018823D1F05A
:10CB10000FC08091E3028823B9F31092E3028CE105
:10CB200097E60E94755C80910805882369F312C01E
:10CB300081E0133009F080E023E041ED5EE16C2FED
:10CB40000E945858CF5FDF5FC53009F072CF84E094
:10CB500080930705DF91CF911F9108951F93CF9385
:10CB6000DF9361E081E00E94895CD0910A05C0E01A
:10CB7000D1111EC010910905112331F0809142019D
:10CB8000882309F4A1C00DC08091E3028823B1F38A
:10CB90001092E3020E94646380910805882371F378
:10CBA0009AC081E0111180E024E043EA5DE189C090
:10CBB000D13009F510910905113031F08091420111
:10CBC000882309F481C00FC08091E3028823B1F368
:10CBD0001092E30280E796EB0E94755C8091080555
:10CBE000882361F378C081E0113009F080E023E010
:10CBF0004AE95DE166C0D23009F5109109051230AD
:10CC000031F080914201882309F45EC00FC0809109
:10CC1000E3028823B1F31092E30288E79AEB0E94C3
:10CC2000755C80910805882361F355C081E012305E
:10CC300009F080E023E04DE85DE143C0D33001F529
:10CC400010910905133029F0809142018823E1F108
:10CC50000FC08091E3028823B9F31092E30283EDC1
:10CC600098EB0E94755C80910805882369F333C0B6
:10CC700081E0133009F080E023E048E85DE121C065
:10CC8000D43011F510910905143029F0809142013A
:10CC90008823D1F00FC08091E3028823B9F310926A
:10CCA000E30286E99AE60E94755C80910805882374
:10CCB00069F311C081E0143009F080E023E04FE710
:10CCC0005DE16C2F0E945858CF5FDF5FC53009F0DF
:10CCD0004FCFC0930705DF91CF911F910895CF9358
:10CCE000DF938091E3021092E302882321F0DF9129
:10CCF000CF910C94646360E085E00E94895CD091E0
:10CD00000A05C0E0D11109C0809142018823F1F1E8
:10CD100021E041E06AEC7EE136C0D13049F48091F7
:10CD20004201882399F120E041E064EC7EE12BC0D0
:10CD3000D23049F480914201882341F120E041E062
:10CD400069EB7EE120C0D33049F480914201882311
:10CD5000E9F020E041E06DEA7EE115C0D43049F40D
:10CD600080914201882391F020E041E069E97EE171
:10CD70000AC0D53059F480914201882339F020E06F
:10CD800041E06CE87EE18C2F0E94CAE0CF5FDF5F5C
:10CD9000C53009F0B7CF86E080930705DF91CF91CA
:10CDA0000895CF93DF938091E3021092E3028823EA
:10CDB00021F0DF91CF910C94646360E085E00E94E4
:10CDC000895CD0910A05C0E0D11109C0809142016F
:10CDD000882341F121E041E06BE77EE120C0D130C2
:10CDE00049F4809142018823E9F020E041E06EE6B9
:10CDF0007EE115C0D23049F480914201882391F040
:10CE000020E041E060E67EE10AC0D33059F4809131
:10CE10004201882339F020E041E063E57EE18C2F78
:10CE20000E94CAE0CF5FDF5FC53071F684E0809377
:10CE30000705DF91CF910895CF93DF938091E302AF
:10CE40001092E302882321F0DF91CF910C94646368
:10CE500060E085E00E94895CD0910A05C0E0D111B4
:10CE600009C0809142018823F1F121E040E064E4AF
:10CE70007EE136C0D13049F480914201882399F196
:10CE800020E040E068E37EE12BC0D23049F480919D
:10CE90004201882341F120E040E06AE27EE120C0C7
:10CEA000D33049F4809142018823E9F021E040E049
:10CEB0006AE17EE115C0D43049F4809142018823B3
:10CEC00091F020E040E06EE07EE10AC0D53059F4F8
:10CED00080914201882339F020E040E060E07EE16B
:10CEE0008C2F0E94CAE0CF5FDF5FC53009F0B7CF5B
:10CEF00086E080930705DF91CF910895BF92CF928E
:10CF0000DF92EF92FF920F931F93CF93DF93CDB7F2
:10CF1000DEB76F970FB6F894DEBF0FBECDBF81E0CE
:10CF200080935609109258091092570940E050E03A
:10CF3000BA0188E297E00E9437CA8BE1E8E2F7E0A5
:10CF4000DE01159601900D928A95E1F780912607F2
:10CF5000909127079C838B838CE891E09A83898347
:10CF600040E050E0BE016F5F7F4F80E090E00E94A4
:10CF70003F73CE0101960E94E43DC0905709D090C6
:10CF8000580961E081E00E94895C10910A0500E087
:10CF900041E0C41AD10811111FC0F0900905FF200B
:10CFA00029F0809142018823B9F00DC08091E302FD
:10CFB0008823B9F31092E3020E946463809108050C
:10CFC000882379F380C181E0F11080E024E04BEF09
:10CFD0005DE1602F0E94585865EB76E088E297E0AB
:10CFE0000E94A1358091B5068F3261F5113021F58F
:10CFF00080910905813029F0809142018823E1F078
:10D000000FC08091E3028823B9F31092E3020E94DB
:10D01000EABD10920A0580910805882369F353C17F
:10D0200081E090910905913009F080E020E242EF23
:10D030005DE1602F0E945858760192E0BB24B394C2
:10D04000B10E63C01130C1F790910905913009F01C
:10D0500047C08091E302882309F442C01092E302A2
:10D0600080917908882319F1815080937908882369
:10D0700061F090E001974FE1489F9001499F300D8A
:10D080001124C9018D5B984F02C085E097E02BE128
:10D09000FC013496A8E2B7E001900D922A95E1F7E1
:10D0A000FC0182819381909327078093260781E07A
:10D0B00090E0A0E0B0E020917908211103C080E069
:10D0C00090E0DC018093CF119093D011A093D11107
:10D0D000B093D21110920A0581E0809308058FC0A9
:10D0E00080914201882309F4A7CF81E0913009F0B3
:10D0F00080E020E24EEE5DE19CCF80914201811103
:10D10000AFC09B2DF1E0EF1AF1084FEFE416F406E3
:10D1100009F4D2C01913CEC060E070E0C7010E94CC
:10D1200025758091B40690910905882309F49DC066
:10D130009113E3CF8091E3028823F9F21092E30286
:10D140001D8218861C821B828CE891E09A83898359
:10D1500080912B07811157C065E077E0611571055B
:10D1600009F454C06C5F7F4F21E045EB56E0CE01DF
:10D1700005960E945D3B882309F44BC08BE1FE01BC
:10D180003596A8E2B7E001900D928A95E1F72B81E0
:10D190003C813093270720932607809179088A30B5
:10D1A000B8F491E0980F90937908FFE18F9FC00148
:10D1B0001124DC01A95BB84F4BE1E8E2F7E00190F4
:10D1C0000D924A95E1F7FC01ED5BF84F3383228322
:10D1D000CE0101960E94E43D10920A0582E090E0A3
:10D1E000A0E0B0E08093CF119093D011A093D11123
:10D1F000B093D21181E0809308051092E20283E09F
:10D200008093420160C064E277E0A8CF60E070E004
:10D21000ABCFE1E9F1E284918F010F5F1F4F8823CB
:10D2200021F00E940283F801F6CFE8EDFDE1849140
:10D230008F010F5F1F4F811103C005EB16E004C083
:10D240000E940283F801F3CFF80181918F018823B6
:10D2500019F00E940283F8CF8AE00E940283B8CFBF
:10D2600081E0911380E041E021C0911731F080917D
:10D270004201882309F445CF13C08091E30288233B
:10D28000B1F31092E30285EB96E00E94D5BF0E94B5
:10D290005D630E9411C480910805882341F313C087
:10D2A00081E090910905911380E040E0602F0E9499
:10D2B00049C127CF9F5F26CF0F5F1F5F053009F061
:10D2C0006ACE909307056F960FB6F894DEBF0FBE37
:10D2D000CDBFDF91CF911F910F91FF90EF90DF9025
:10D2E000CF90BF9008952F923F924F925F926F928E
:10D2F0007F928F929F92AF92BF92CF92DF92EF92E6
:10D30000FF920F931F93CF93DF9361E081E00E9420
:10D31000895CD0910A05C0E082E0282E85E0382E95
:10D320009CED892E95E0992EA12CB12C26ED422E54
:10D3300026E0522E612C712C31E4E32E35E5F32EDC
:10D340004BE8C42E47E4D42ED11121C01091090519
:10D35000112331F080914201882309F44BC00DC0A4
:10D360008091E3028823B1F31092E3020E94646388
:10D3700080910805882371F3C6C081E0111180E017
:10D3800024E040ED5DE16C2F0E94585833C0D1304D
:10D3900089F510910905113029F080914201811120
:10D3A00016C028C08091E3028823B9F31092E302EB
:10D3B000809106058D278093060583E080934201C6
:10D3C0000E948B4780910805882339F39CC0809187
:10D3D0000605811103C02FEB3DE102C023EC3DE1C6
:10D3E00081E0113009F080E001E047EC5DE16C2F55
:10D3F0000E9447DD80910605882309F47CC0D23065
:10D4000009F077C010910905123031F08091420186
:10D41000882309F46EC05EC08091E3028823B1F3D3
:10D420001092E30291E09093E1021092DD021092DB
:10D43000DE021092DF021092E0020E94EA5C83E0BA
:10D440008093420185EB9DE19093DE118093DD1185
:10D450003092DC112092DB118092D7119092D8117A
:10D46000A092D911B092DA114092D3115092D411F6
:10D470006092D5117092D61120E030E04AE754E472
:10D480006091020570910305809104059091050556
:10D490000E9411E620E030E84BEB54E40E94DBE907
:10D4A0000E944FEB6093CF117093D0118093D111F4
:10D4B0009093D211F0924B01E0924A01D092E11187
:10D4C000C092E0111092DF1180910805882309F4C1
:10D4D0009DCF19C082E095E00E9484C09C0181E04C
:10D4E000123009F080E000E04BEA5DE16C2F0E9411
:10D4F00047DD83E001C082E0CF5FDF5FC53009F028
:10D5000023CF80930705DF91CF911F910F91FF905B
:10D51000EF90DF90CF90BF90AF909F908F907F90D3
:10D520006F905F904F903F902F9008950F931F93AF
:10D53000CF93DF9361E081E00E94895CD0910A057E
:10D54000C0E011E0D11121C000910905002331F0A4
:10D5500080914201882309F4E9C00DC08091E30263
:10D560008823B1F31092E3020E946463809108055E
:10D57000882371F3E2C081E0011180E024E048E7F4
:10D580005DE16C2F0E945858D1C0D13091F50091C7
:10D590000905013031F080914201882309F4C6C0A9
:10D5A0001BC08091E3028823B1F31092E302D09371
:10D5B000E1021092DD021092DE021092DF02109260
:10D5C000E00263EA71E18EE69DE10E94EFDF809167
:10D5D0000805882301F3B1C083EA91E10E94BE43AC
:10D5E0009C0181E0013009F080E000E044E65DE16B
:10D5F0009AC0D23091F500910905023031F0809146
:10D600004201882309F492C01BC08091E302882361
:10D61000B1F31092E3021093E1021092DD02109236
:10D62000DE021092DF021092E00267EA71E18AE501
:10D630009DE10E94EFDF80910805882301F37DC002
:10D6400087EA91E10E94BE439C0181E0023009F02B
:10D6500080E000E040E55DE166C0D33091F50091E7
:10D660000905033031F080914201882309F45EC03E
:10D670001BC08091E3028823B1F31092E302109360
:10D68000E1021092DD021092DE021092DF0210928F
:10D69000E0026BEA71E186E49DE10E94EFDF809198
:10D6A0000805882301F349C08BEA91E10E94BE433B
:10D6B0009C0181E0033009F080E000E04CE35DE193
:10D6C00032C0D43099F500910905043029F08091D9
:10D6D0004201882359F11BC08091E3028823B9F3EA
:10D6E0001092E3021093E1021092DD021092DE022A
:10D6F0001092DF021092E0026FEA71E182E39DE195
:10D700000E94EFDF80910805882309F316C08FEA95
:10D7100091E10E94BE439C0181E0043009F080E069
:10D7200000E048E25DE16C2F0E9447DDCF5FDF5FE4
:10D73000C53009F007CFC0930705DF91CF911F9146
:10D740000F91089511980000000087FD5AC041987C
:10D7500000000000119A00000000880F11980000DE
:10D76000000087FD5AC0419800000000119A000097
:10D770000000880F11980000000087FD4CC0419800
:10D7800000000000119A00000000880F11980000AE
:10D79000000087FD3EC0419800000000119A000083
:10D7A0000000880F11980000000087FD30C04198EC
:10D7B00000000000119A00000000880F119800007E
:10D7C000000087FD22C0419800000000119A00006F
:10D7D0000000880F11980000000087FD14C04198D8
:10D7E00000000000119A00000000119800000000E5
:10D7F00086FD15C0419800000000119A000000004D
:10D800000895419AA5CF419AEBCF419ADDCF419A35
:10D81000CFCF419AC1CF419AB3CF419AA5CF419A78
:10D82000EACF6F927F928F929F92AF92BF92CF92E8
:10D83000DF92EF92FF920F931F93CF93DF935C01E0
:10D840007B01742E69018AE0481709F471C0A5E1D3
:10D850004A1349C0DB011296ED91FC911397928017
:10D86000C681D781139A0E94264280EE882E890CA9
:10D8700090E1692E690C88EF0E94A26B0E942642FB
:10D88000BFE1B91508F443C0892D807780680E94F4
:10D89000A26B892D8295807F0E94A26B0E942642F6
:10D8A00080E80E94A26B80E00E94A26B0E94264248
:10D8B0008AEF0E94A26B0E9426428E01005F1F4FDA
:10D8C0008881807F0E94A26B89918295807F0E94CF
:10D8D000A26BC017D107A1F70E94264293948394AC
:10D8E0009610C9CF13989601472DB701C501DF9156
:10D8F000CF911F910F91FF90EF90DF90CF90BF904D
:10D90000AF909F908F907F906F900C946E40882D79
:10D91000807780680E94A26B882D8295807F0E940C
:10D92000A26B0E94264280E80E94A26B80E8BCCFD6
:10D930000B9A1398399A4198099A119A139A0E944E
:10D94000264288E790E00E942B4288EF0E94A26B5B
:10D950000E94264280E20E94A26B80E00E94A26B9D
:10D960000E94264280E00E94A26B80E80E94A26B87
:10D970000E94264280E00E94A26B80E10E94A26B7E
:10D980000E9426428FE090E00E942B4280E20E949B
:10D99000A26B80E40E94A26B0E94264280E20E9459
:10D9A000A26B80E60E94A26B0E942642D0E08D2FDF
:10D9B000807780680E94A26B8D2F8295807F0E9465
:10D9C000A26B0E94264280E80E94A26B80E00E9427
:10D9D000A26B0E9426428AEF0E94A26B0E942642FE
:10D9E000C0E280E00E94A26B80E00E94A26B0E94D5
:10D9F0002642C150B1F788EF0E94A26B0E942642D6
:10DA0000DF5FD032A1F680E00E94A26B80EC0E9422
:10DA1000A26B0E942642139866CFCF92DF92EF92BC
:10DA2000FF920F931F93CF93DF931F92CDB7DEB773
:10DA30006C01DC01DC961C91DC97DB960C917C017F
:10DA4000B4E0EB0EF11CDC015996ED91FC915A9774
:10DA5000C70169830995482F410F2981602FC701AC
:10DA60000E947442F60123AD082E000C990B820F20
:10DA7000911D83AF81E090E00F90DF91CF911F91D6
:10DA80000F91FF90EF90DF90CF900895FC011382EB
:10DA900012828EE691E09183808313AE14AE15AEB0
:10DAA0009F012C5F3F4F11861086138612861586C4
:10DAB00081E0848782E28687138A128ADF01979643
:10DAC000CF01C5964FEF4D93A817B907E1F791E045
:10DAD00094A346ED5EE3528F418F938F148E158E83
:10DAE00080E4868F178E85E79EE396AB85AB7783C0
:10DAF0006683C9010C94BC41EF92FF920F931F9370
:10DB0000CF93DF931F92CDB7DEB78C017B0180E20C
:10DB100049830E94028349814F3F11F084E501C08F
:10DB200082E40E9402838AE30E940283F8016081FA
:10DB300071818281938142E00E942E86F7014081AB
:10DB40005181628173818CE690E20E94804F62E095
:10DB500070E080E090E00F90DF91CF911F910F91E6
:10DB6000FF90EF900C94DE3F9CE0899F802D112464
:10DB700091E0980F9093CD112CE0280F2093CE11B7
:10DB80004091630650E030E02E5F3F4F2417350789
:10DB9000CCF0292F30E04091650650E0241735077E
:10DBA0008CF4662341F08E5F0E9431C08091CE11CB
:10DBB0008E5F0E9431C08091CE11109266068093D4
:10DBC0006706089508950F931F93CF938C01C62F76
:10DBD000CC2349F0F80181918F01882321F00E9424
:10DBE0009B72C150F5CFCF911F910F910895CF93A4
:10DBF000C82F823059F02CF4813089F4CF910C94E5
:10DC00009758833031F0843021F009C084EB97E1DC
:10DC100002C084E990E10E94BD72C093E602CF91F8
:10DC20000895CF93C82F8FEF8C0F893060F484EB69
:10DC300097E10E94BD728C2F0E949B728091E60238
:10DC40000E94F76D03C08C2F0E949B7281E0CF91E0
:10DC50000895CF939FEF980F993068F4C82F84EB05
:10DC600097E10E94BD728C2F0E949B728091E60208
:10DC7000CF910C94F76DCF910C949B72CF93DF935F
:10DC8000EC01FE018491882321F00E94296E2196E7
:10DC9000F8CFDF91CF910895CF93DF93EC01899175
:10DCA000882319F00E94296EFACFDF91CF91089551
:10DCB000CF93DF93EC0161E271E00E94466D8AE749
:10DCC00091E099838883DF91CF9108954F925F927D
:10DCD0006F927F928F929F92AF92BF92CF92DF927C
:10DCE000EF92FF920F931F93CF93DF933C01B0E429
:10DCF000A0E06A2F70E0AB014B0F511D5595479581
:10DD00004A1711F04B130BC0E8EFFFE165917491D6
:10DD1000072E000C880B990B0E94B2E562C0CA0165
:10DD20000197880F991F880F991FFC01E650F14E4B
:10DD3000059114919A01220F331F220F331FF9010D
:10DD4000E650F14EC591D4916016710614F4B42FCB
:10DD5000D2CFA42FC615D7050CF4CBCF8450914E4B
:10DD6000FC01E590F490F901E450F14EC590D49097
:10DD7000B7010F2C000C880B990B0E94B2E54B01E8
:10DD80005C01B301601B710B072E000C880B990B13
:10DD90000E94B2E52B013C01B6016E197F09072EE6
:10DDA000000C880B990B0E94B2E59B01AC01C301EA
:10DDB000B2010E9411E66B017C01C01BD10BBE01B8
:10DDC000DD0F880B990B0E94B2E59B01AC01C701E6
:10DDD000B6010E94D6EA9B01AC01C501B4010E94C4
:10DDE000DCE9DF91CF911F910F91FF90EF90DF90D1
:10DDF000CF90BF90AF909F908F907F906F905F90EB
:10DE00004F9008950F931F93CF93DF93CDB7DEB755
:10DE100028970FB6F894DEBF0FBECDBF6091E41116
:10DE20007091E511072E000C880B990B0E94B2E54A
:10DE30006D837E838F8398878091CE0C9091CF0CD9
:10DE4000A091D00CB091D10C89839A83AB83BC8311
:10DE50004DEFBE016B5F7F4FCE0101960E947C6D3E
:10DE60006091E2117091E311072E000C880B990B61
:10DE70000E94B2E56D837E838F8398878091FA023A
:10DE80009091FB02A091FC02B091FD0289839A83DC
:10DE9000AB83BC834FEFBE016B5F7F4FCE0101961A
:10DEA0000E947C6DE4E7F0E284918F010F5F1F4FC9
:10DEB000882321F00E940283F801F6CFE091120539
:10DEC000F0E0E05FFA4F608170E080E090E00E9457
:10DED0001286EFE6F0E284918F010F5F1F4F8823D7
:10DEE00021F00E940283F801F6CF6091110570E0E5
:10DEF00080E090E00E94128628960FB6F894DEBF6C
:10DF00000FBECDBFDF91CF911F910F910895EF927A
:10DF1000FF920F931F93CF93DF93809120018F3750
:10DF200090F08F579091100590932206992311F04D
:10DF30005D9A01C05D9890911105909321069923F7
:10DF400059F05C9A0AC090912206891708F05D98F2
:10DF500090912106891708F05C988F5F80932001CB
:10DF60009091200681E089278093200681110E94EC
:10DF70009F5880911F0185301CF4C1E0C80F01C07B
:10DF8000C0E0823009F4AFC04CF48823F9F081304E
:10DF900009F0DDC010927B0087E4BBC0843009F437
:10DFA000C0C00CF4B3C0853009F0D1C090911F06F9
:10DFB000911102C080931F0680911F0681508093AB
:10DFC0001F06882309F4C3C0C5E0C1C080911E01AB
:10DFD0008F5F80311CF480931E01B9C010921E0126
:10DFE00080910F05811113C080911506909116063E
:10DFF00090930E0580930D05809113069091140661
:10E0000090930C0580930B0581E080930F058AE0C7
:10E01000E5E1F6E0DF011D928A95E9F7109214061A
:10E020001092130600910D0510910E0511950195A2
:10E0300011098091E4119091E511D1E018161906AB
:10E040002CF080911005811101C0D0E0809148032F
:10E0500090914903919581959109801791073CF41E
:10E060004AEF5FE16BE170E280E00E9400D08091B6
:10E070001101909112019195819591090817190745
:10E080004CF4DD2339F04DE250E26EE470E280E0C2
:10E090000E9400D0E090E211F090E31100910B0596
:10E0A00010910C05809146039091470380179107CA
:10E0B0003CF04AE050E26BE170E28FEF0E9400D04A
:10E0C00080910F0190911001081719070CF43FC0BF
:10E0D0001E141F04E4F54DE350E26EE470E28FEF8E
:10E0E0000E9400D034C080917A0086FD2DC08091BE
:10E0F0007800909179002091150630911606820FD4
:10E10000931F909316068093150621C010927B00F2
:10E1100086E480937C0080917A00806480937A000A
:10E1200016C080917A0086FD11C080917800909190
:10E1300079002091130630911406820F931F90935B
:10E1400014068093130603C0C2E001C0C4E0C0936C
:10E150001F0120E030E0A4E0C901880F991FFC01F5
:10E16000EC50FE4E408151814115510541F1F8942A
:10E170002230B9F463B1647015981416150614F4BE
:10E180002A9A01C02A980000000000002B9A7A2FDA
:10E190007A950000E9F72B98662311F02A9A01C0BE
:10E1A0002A987894FC01EC50FE4E808191811416DF
:10E1B000150614F4019701C00196918380832F5FA7
:10E1C0003F4F2330310509F0C7CF80915A038111A9
:10E1D0000E9409B18091B3119091B4110097A9F0F8
:10E1E00001979093B4118093B311892B71F480E659
:10E1F00090E29093EF118093EE11DF91CF911F91F8
:10E200000F91FF90EF900C94C781DF91CF911F91F8
:10E210000F91FF90EF9008958F929F92AF92BF92CF
:10E22000CF92DF92EF92FF920F931F93CF93DF93E2
:10E2300000D000D0CDB7DEB7FC018381813079F505
:10E24000818181FF2CC081899289A389B489892B1E
:10E250008A2B8B2B09F448C07F0140E050E0BA01C3
:10E26000CF010E9437CA8823D1F0F70185889688AC
:10E27000A788B08CC18CD28C82E090E0A0E0B0E0A6
:10E28000F60180839183A283B3839E012F5F3F4F6A
:10E29000B501A401C6010E94B4C8811102C080E08A
:10E2A0003CC000E010E09801B501A401C6010E9445
:10E2B00022C88823A1F389809A80AB80BC80F601B4
:10E2C0008789803141F4F8EF8F16FFEF9F06A10494
:10E2D000B10460F4DACF88EF88168FEF9806A806AD
:10E2E0008FE0B80618F4D1CF81E017C0F701158A86
:10E2F000168A178A108E118A128A138A148A8181CB
:10E3000080688183C7010E9404CA882341F240E0EB
:10E3100050E0BA01C7010E9437CA0F900F900F90CA
:10E320000F90DF91CF911F910F91FF90EF90DF90B1
:10E33000CF90BF90AF909F908F9008952F923F9273
:10E340004F925F926F927F928F929F92AF92BF9205
:10E35000CF92DF92EF92FF920F931F93CF93DF93B1
:10E36000CDB7DEB76F970FB6F894DEBF0FBECDBF47
:10E370006C012DB63EB61D8218861C821B828CE86D
:10E3800091E09A838983FB0180819E012F5F3F4F3B
:10E3900039018F3239F084E297E0F601918380836E
:10E3A0008B0162C085E097E0F601918380838B0149
:10E3B0000F5F1F4F0115110509F456C04DB65EB62B
:10E3C0006FE270E0C8010E9482ED4C010817190746
:10E3D00008F04AC07C01E01AF10AFF24C701019647
:10E3E0002DB73EB7281B390B0FB6F8943EBF0FBEB2
:10E3F0002DBF8DB79EB701965C01A701B8010E94A1
:10E40000ABEDF501EE0DFF1D1082F601608171810B
:10E410006115710511F06C5F7F4F21E0A501CE0100
:10E4200005960E945D3B811113C0B50187E991E219
:10E430000E94B64F8EE20E9402838AE00E9402830D
:10E440000FB6F8945EBE0FBE4DBE00E010E00CC0EB
:10E45000F6017182608284010F5F1F4F0FB6F8943E
:10E460005EBE0FBE4DBEA6CFC3010E94E43DC801F3
:10E470000FB6F8943EBE0FBE2DBE6F960FB6F89441
:10E48000DEBF0FBECDBFDF91CF911F910F91FF90E7
:10E49000EF90DF90CF90BF90AF909F908F907F9044
:10E4A0006F905F904F903F902F9008951092B2061A
:10E4B0008091A408882321F081EA98E00C947C35AF
:10E4C00008950F931F93CF93E0913D06F0913E0680
:10E4D000309719F08FE296E009950091310610917E
:10E4E0003206E0916006F091610682E00995E091C4
:10E4F0006006F091610681E0099520E030E045E199
:10E50000B8018FE296E00E943741C82F882341F07E
:10E5100022E636E047E1B8018FE296E00E943741FB
:10E52000E0916006F091610680E009958C2FCF9113
:10E530001F910F910895E0912B06F0912C06019008
:10E54000F081E02D682F8BE296E009940F931F93E2
:10E55000CF93DF93EC018C010A5E1F4FFE01849183
:10E56000882331F00E949B722196C017D107B1F722
:10E57000DF91CF911F910F91089520913306309133
:10E5800034062817390709F444C090933406809361
:10E590003306009709F437C020914606FC0121118B
:10E5A00007C03596E491E0934706FC013C960FC006
:10E5B000213039F43F96E491E0934706FC017096D0
:10E5C00006C03D96E491E0934706FC013E96849197
:10E5D0008093480680914706082E000C990B2091E5
:10E5E0004806821B910927FD939520914906203406
:10E5F00041F0829FC001112426E0969587952A95C7
:10E60000E1F780934A0686ED9EE39093450680935A
:10E6100044060895CF93DF9380916806811107C067
:10E6200081E0809368068FE296E00E94BC41C09131
:10E630003106D0913206E0916006F091610682E0E9
:10E640000995E0916006F091610681E0099520E06E
:10E6500030E044E1BE018FE296E00E94374122E6BD
:10E6600036E047E1BE018FE296E00E943741E0913B
:10E670006006F091610680E0DF91CF9109942F92BE
:10E680003F924F925F926F927F928F929F92AF9242
:10E69000BF92CF92DF92EF92FF920F931F93CF938F
:10E6A000DF93CDB7DEB7C257D1090FB6F894DEBFFE
:10E6B0000FBECDBF8C015B014A018DB79EB7AF96EF
:10E6C0009FAF8EAFAF97AD961FAEAD972B0194E085
:10E6D000490E511C7E01EFE5EE0EF11C9CE8692EFF
:10E6E00091E0792E80E490E08C0F9D1F0496E196D6
:10E6F0009FAF8EAFE197F5018781823008F482C128
:10E7000084859585A685B7858F719927AA27BB270C
:10E71000892B8A2B8B2B09F075C182EC96E0892B13
:10E7200011F01092C20642EC56E0BE016F5F7F4FBF
:10E73000C2010E949CC918160CF064C18C85282F58
:10E740002871203129F4909156099150923078F433
:10E750009981992309F456C1953E69F29E3259F286
:10E760009091C2069E3239F28A7029F6D4C02DB635
:10E770003EB6BE016F5F7F4FC7010E9493C7011570
:10E78000110521F0F80180818111BBC021E081E0F9
:10E7900090E0F70101900020E9F73197EE19FF09A9
:10E7A000E80FF91F32968DB79EB78E1B9F0B0FB6E1
:10E7B000F8949EBF0FBE8DBFEDB7FEB731966F01C7
:10E7C000211102C0B80102C067E472E0C6010E94D4
:10E7D00096EDB701C6010E9477ED67E472E0C601CD
:10E7E0000E9477ED25961FAE259728961FAE289795
:10E7F00024961FAE1EAE249722967FAE6EAE229751
:10E8000021E0A701B201E1968EAD9FADE1970E9494
:10E810005D3B81114DC080915609811149C0E1E9EC
:10E82000F1E284919F012F5F3F4F882381F0E296B0
:10E830002FAFE297E3963FAFE3970E940283E29601
:10E840002FADE297E3963FADE397F901EACFEDE70D
:10E85000F1E284919F012F5F3F4F811102C0970128
:10E8600010C0E2962FAFE297E3963FAFE3970E9486
:10E870000283E2962FADE297E3963FADE397F9016D
:10E88000E8CFF90181919F01882379F0E2962FAFBB
:10E89000E297E3963FAFE3970E940283E3963FAD92
:10E8A000E397E2962FADE297ECCF8AE00E940283D5
:10E8B0008BE1FE01EC5BFF4FDE01959601900D921E
:10E8C0008A95E1F724968EAD9FAD24979CA38BA3E8
:10E8D0007AA269A240E050E0BE016F5D7F4FC601A1
:10E8E0000E943F73CE0181960E94E43DCE01805C80
:10E8F0009F4F0E94E43D0FB6F8943EBE0FBE2DBE62
:10E90000FACEF80101900020E9F73197CF01801B82
:10E91000910B20E03ECF81E0203109F080E0809330
:10E92000B406811108C08985873409F0E4CE8A8550
:10E930008E3709F4E0CE80915609813029F082307B
:10E94000D9F18111D8CE0AC0809157099091580908
:10E9500001969093580980935709CDCEBE016F5F01
:10E960007F4F85EB96E00E9493C70115110529F4AE
:10E9700085EBC82E86E0D82E09C06801F60181918A
:10E980006F018823A9F30E940283F8CFF6018191D9
:10E990006F01882319F00E940283F8CF80E20E9461
:10E9A00002836D8D7E8D8F8D98A14AE00E94AA858D
:10E9B0008AE00E9402839FCEBE016F5F7F4F85EB8E
:10E9C00096E00E9493C78114910441F065EB76E0D4
:10E9D000C4010E9464ED892B69F414C0AD96FFADAB
:10E9E000AD978F2F90E020915B0930915C098217E1
:10E9F000930741F0AD962FADAD972F5FAD962FAF3A
:10EA0000AD9779CEAF96EEADFFADAF970FB6F89458
:10EA1000FEBF0FBEEDBFCE58DF4F0FB6F894DEBF7E
:10EA20000FBECDBFDF91CF911F910F91FF90EF905F
:10EA3000DF90CF90BF90AF909F908F907F906F901E
:10EA40005F904F903F902F9008950F931F93CF9317
:10EA5000DF93CDB7DEB76F970FB6F894DEBF0FBE6A
:10EA6000CDBF8B0122E02093560990935C098093DF
:10EA70005B0940E050E0BA0188E297E00E9437CAA3
:10EA80008BE1E8E2F7E0DE01159601900D928A95A0
:10EA9000E1F780912607909127079C838B838CE870
:10EAA00091E09A838983A801BE016F5F7F4F80E068
:10EAB00090E00E943F73CE0101960E94E43D6F9664
:10EAC0000FB6F894DEBF0FBECDBFDF91CF911F917F
:10EAD0000F910895DF92EF92FF920F931F93CF93C0
:10EAE000DF9300D000D01F92CDB7DEB72091B306E0
:10EAF000222309F494C1D62E7C018091A408882396
:10EB000009F4A5C0442309F45DC18091BC088823A1
:10EB100029F1E6E7F1E284918F010F5F1F4F88230F
:10EB200021F00E940283F801F6CFE3E3F1E2849141
:10EB30008F010F5F1F4F882321F00E940283F8018D
:10EB4000F6CF61E070E080E090E00E9412868AE0FB
:10EB50000E9402838AE291E20E94EC3D82EC98E0FE
:10EB60009A8389838FE28093C10881E08B8310E0D0
:10EB70000FE180917908181778F4019FC0011124E2
:10EB8000AE014D5F5F4FBE016F5F7F4F8D5B984F52
:10EB90000E9463C71F5FEDCF8B8187FD0FC0AE0161
:10EBA0004D5F5F4FBE016F5F7F4F8DE998E00E9420
:10EBB00063C789819A8101979A838983E981FA8160
:10EBC0001082E091BC0884E0E89FF0011124E35436
:10EBD000F74F8091520990915309A0915409B09137
:10EBE000550980839183A283B383E1E9F1E28491A3
:10EBF0008F010F5F1F4F882321F00E940283F801CD
:10EC0000F6CFB70181E191E20E94B64F6091BC0856
:10EC10009DE8699FB00111246F53774F86E091E220
:10EC20000E94B64F40915209509153096091540986
:10EC30007091550980E091E20E94634F8AE00E9442
:10EC400002838091BC088F5F8093BC0826C0442358
:10EC5000C1F0E1E9F1E284918F010F5F1F4F88233A
:10EC600021F00E940283F801F6CFE0EFF0E28491F8
:10EC70008F010F5F1F4F882381F00E940283F801EC
:10EC8000F6CF1092BC0892E09EC0B70187ED90E2EB
:10EC90000E94B64F8AE00E9402830E945672B7011A
:10ECA000CE0103960E949E718C01892B09F4B7C096
:10ECB0009B818C81692F782FDD2009F45AC0611562
:10ECC000710511F06C5F7F4F21E0A80181EA98E0A7
:10ECD0000E945D3B882309F448C08091B20890915E
:10ECE000B308A091B408B091B50880934E099093F1
:10ECF0004F09A0935009B0935109109252091092F4
:10ED000053091092540910925509B80189EC90E208
:10ED10000E94B64F40914E0950914F0960915009A1
:10ED20007091510981EC90E20E94634F8AE00E9449
:10ED30000283E2EBF0E284917F019FEFE91AF90A86
:10ED4000882321F00E940283F701F5CFB80180E00B
:10ED500090E00E9425758091C206882319F082EC0C
:10ED600096E001C0C80160E02AC0B8018EE990E2D7
:10ED700010C06115710511F06C5F7F4F26E5A80189
:10ED800081EA98E00E945D3B81110CC0B8018AE8DD
:10ED900090E20E94B64F8EE20E9402838AE00E94B7
:10EDA00002833DC081E08093B006B70188E790E21E
:10EDB0000E94B64F8AE00E94028360E0C8010E9470
:10EDC0002F592DC091E09D83E1E9F1E284918F01FB
:10EDD0000F5F1F4F882321F00E940283F801F6CFB6
:10EDE000EBEEF0E284918F010F5F1F4F882321F03B
:10EDF0000E940283F801F6CF9D81913019F0E5EE73
:10EE0000F0E202C0EFEDF0E284918F010F5F1F4F3F
:10EE1000882309F43ACF0E940283F801F5CF0F90BE
:10EE20000F900F900F900F90DF91CF911F910F9146
:10EE3000FF90EF90DF900895EF92FF921F93CF9392
:10EE4000DF931F92CDB7DEB7182FE6E7F1E284918A
:10EE50007F012FEFE21AF20A882331F099830E9492
:10EE60000283F7019981F3CFE12FF92F84917F017C
:10EE70009FEFE91AF90A882321F00E940283F70123
:10EE8000F5CF609125067091260680912706909116
:10EE900028060E9412868AE00E9402830E9433D6CE
:10EEA00010922406109223060F90DF91CF911F91AC
:10EEB000FF90EF9008950F931F93CF93DF938C01F2
:10EEC000EB0190919E0620919F06921307C082E964
:10EED00096E00E94AB7E0E945AD1F3CFF801A08148
:10EEE000B1814881598180919D0634E0839FF00172
:10EEF0001124EA56F94FB387A287558744879F5F4D
:10EF000090939E068F5F821719F080939D0602C032
:10EF100010929D06DF91CF911F910F9108952CEAD9
:10EF200035EC47E25EE36091760970917709809154
:10EF30007809909179090E94D6EA609361097093EB
:10EF40006209809363099093640908952CEA35EC73
:10EF500047E25EE360917A0970917B0980917C09B8
:10EF600090917D090E9411E660936509709366098E
:10EF7000809367099093680908952F923F924F926A
:10EF80005F926F927F928F929F92AF92BF92CF9239
:10EF9000DF92EF92FF920F931F93CF93DF9361E085
:10EFA00081E00E94895CD0910A05C0E073E0A72E41
:10EFB000EEE92E2EE2E23E2EF4E64F2E512C612C8D
:10EFC000712CBB24B394A2EC8A2EA2E29A2ED1110A
:10EFD00023C080910905882331F080914201882364
:10EFE00009F406C20DC08091E3028823B1F31092A8
:10EFF000E3020E94646380910805882371F362C371
:10F0000081E090910905911180E024E04BE053E20A
:10F010006C2F0E945858ECC1D130E1F58091090560
:10F02000813031F080914201882309F4E1C121C08F
:10F030008091E3028823B1F31092E302D093E102BE
:10F040001092DD021092DE021092DF021092E002B6
:10F0500001ED11EC24E031E040E050E064EE71E1BC
:10F0600084E093E20E947DDE809108058823D1F23E
:10F0700029C311E080910905813009F010E08091E9
:10F08000E4119091E5110E9455479C0100E04DEF7D
:10F0900052E2AAC1D230E1F580910905823031F007
:10F0A00080914201882309F4A3C121C08091E30229
:10F0B0008823B1F31092E302B092E1021092DD02D4
:10F0C0001092DE021092DF021092E00204ED11ECC9
:10F0D0002EE630E040E050E062EE71E189EF92E22E
:10F0E0000E947DDE809108058823D1F2EBC211E0F9
:10F0F00080910905823009F010E08091E211909131
:10F10000E3110E9455479C0100E045EF52E26CC1BB
:10F11000D330E1F580910905833031F080914201CF
:10F12000882309F465C121C08091E3028823B1F3EB
:10F130001092E302B092E1021092DD021092DE0220
:10F140001092DF021092E00200E010E02FEF30E0BA
:10F1500040E050E06BEC7CE08BEE92E20E947DDEC2
:10F16000809108058823D1F2ADC211E08091090594
:10F17000833009F010E08091CB0C9091CC0C0E9470
:10F1800055479C0100E041EE52E22EC1D43069F5B2
:10F1900090910905943029F080914201811113C0AA
:10F1A00027C18091E3028823B9F31092E302809192
:10F1B00069098B2580936909A09242018091080515
:10F1C000882351F37FC280916909811103C020ED2A
:10F1D00032E202C024ED32E281E0943009F080E0B6
:10F1E00001E048ED52E26C2F01C1D53009F047C073
:10F1F00080910905853031F080914201882309F41E
:10F20000F7C018C08091E3028823B1F31092E302A3
:10F21000E12CF12C02E813E420E030E0A90161E3E5
:10F2200071E089EC92E20E94DDDE8091080588237E
:10F2300019F348C283E48F9382E88F931F921F9241
:10F240001F921F9281E391E09F938F93ABEBB2E209
:10F25000BF93AF939F928F92CF9381E090910905D6
:10F26000953009F080E08F930E942ED8ADB7BEB7DD
:10F270001E960FB6F894BEBF0FBEADBFB9C0D63054
:10F2800009F049C080910905863031F08091420132
:10F29000882309F4ADC018C08091E3028823B1F33C
:10F2A0001092E302E12CF12C02E813E420E030E0BC
:10F2B000A9016DE271E084EB92E20E94DDDE8091B3
:10F2C0000805882319F3FEC1B3E4BF9382E88F9346
:10F2D0001F921F921F921F928DE291E09F938F9336
:10F2E000A6EAB2E2BF93AF93ADEAB2E2BF93AF93A7
:10F2F000CF9381E090910905963009F080E08F93DB
:10F300000E942ED8ADB7BEB71E960FB6F894BEBFFA
:10F310000FBEADBF6DC0D73009F06AC0809109053E
:10F32000873031F080914201882309F461C04EC0DA
:10F330008091E3028823B1F31092E3020E94EA5C19
:10F34000A09242013092DE112092DD1189E291E01B
:10F350009093DC118093DB111092D7111092D81189
:10F360001092D9111092DA114092D3115092D41107
:10F370006092D5117092D61120E030E048EC52E452
:10F380006091290170912A0180912B0190912C01AB
:10F390000E9411E60E944FEB6093CF117093D01141
:10F3A0008093D1119093D211A6E0B6E5B0934B01B2
:10F3B000A0934A011092E1111092E0111092DF1116
:10F3C00080910805882309F4ADCF7CC111E08091BC
:10F3D0000905873009F010E089E291E00E9450466B
:10F3E0009C0100E046E952E26C2F812F0E9447DD2C
:10F3F0002CEA35EC47E25EE360916509709166099D
:10F4000080916709909168090E94D6EA60937A0911
:10F4100070937B0980937C0990937D092CEA35ECED
:10F4200047E25EE36091610970916209809163092E
:10F43000909164090E9411E66093760970937709B0
:10F440008093780990937909D830A9F580910905BE
:10F45000883031F080914201882309F42BC11CC00F
:10F460008091E3028823B1F31092E302C12CD12CE6
:10F47000E12C18E1F12E0CE116E420E030E040E848
:10F480005FE36DE579E080E992E20E945ADF8091C6
:10F4900008058823F9F216C111E08091090588302A
:10F4A00009F010E08DE599E00E947F449C0100E0A6
:10F4B0004AE852E271C0D930B9F580910905893026
:10F4C00031F080914201882309F4F4C01EC080917C
:10F4D000E3028823B1F31092E30226EAC22E27E763
:10F4E000D22EE12C18E1F12E0CE116E42AE037EDE2
:10F4F00043E25CE36AE779E084E892E20E945ADF43
:10F50000809108058823E9F2DDC011E080910905AA
:10F51000893009F010E08AE799E00E947F449C015D
:10F5200000E04EE752E238C0DA30D9F580910905A3
:10F530008A3031F080914201882309F4BBC01EC09B
:10F540008091E3028823B1F31092E3028FE8C82E82
:10F5500087E7D82EE12C18E1F12E0CE116E420E02B
:10F5600030E040E85FE366E779E088E792E20E94F6
:10F570005ADF809108058823E9F2A4C011E0809148
:10F5800009058A3009F010E086E799E00E947F447F
:10F590009C0100E042E752E26C2F812F0E9447DD80
:10F5A00089C0DB30E1F5809109058B3031F0809125
:10F5B0004201882309F47EC021C08091E3028823A0
:10F5C000B1F31092E302B092E1021092DD021092C8
:10F5D000DE021092DF021092E00205E71BE724E052
:10F5E00031E046E950E067E271E085E692E20E9490
:10F5F0007DDE809108058823D1F264C011E08091FE
:10F6000009058B3009F010E08091270190912801C5
:10F610000E9455479C0100E048E552E2BDCFDC3036
:10F6200019F5809109058C3031F0809142018823D1
:10F6300009F440C00FC08091E3028823B1F3109217
:10F64000E3028AE89DEB0E94755C8091080588239F
:10F6500061F338C081E0909109059C3009F080E0A9
:10F6600023E047E452E223C0DD3021F58091090513
:10F670008D3029F0809142018823E1F00FC0809104
:10F68000E3028823B9F31092E30287E89DEB0E941E
:10F69000755C80910805882369F314C081E090911E
:10F6A00009059D3009F080E023E046E352E26C2F2B
:10F6B0000E945858CF5FDF5FC53009F088CC8EE0DC
:10F6C00080930705DF91CF911F910F91FF90EF90ED
:10F6D000DF90CF90BF90AF909F908F907F906F9072
:10F6E0005F904F903F902F9008950F931F93CF936B
:10F6F000DF93CDB7DEB76E970FB6F894DEBF0FBEBF
:10F70000CDBF809128018F93809127018F931F9205
:10F710001F9286E292E29F938F938E010F5F1F4F9D
:10F720001F930F930E9442E581E08093E402C80199
:10F730000E94B3811092E4020FB6F894DEBF0FBEB0
:10F74000CDBF6E960FB6F894DEBF0FBECDBFDF9172
:10F75000CF911F910F910895CF93DF9361E081E0E6
:10F760000E94895CD0910A05C0E0D11120C080912F
:10F770000905882331F080914201882309F41BC1D7
:10F780000DC08091E3028823B1F31092E3020E943E
:10F79000646380910805882371F315C181E090911D
:10F7A0000905911180E024E041E252E201C1D1302B
:10F7B00019F580910905813031F08091420188234B
:10F7C00009F4F9C00FC08091E3028823B1F31092CD
:10F7D000E3028DEB97E70E94755C80910805882312
:10F7E00061F3F1C081E090910905913009F080E06A
:10F7F00023E045E152E2DCC0D23019F580910905E1
:10F80000823031F080914201882309F4D4C00FC0C6
:10F810008091E3028823B1F31092E3028EEA95E629
:10F820000E94755C80910805882361F3CCC081E05B
:10F8300090910905923009F080E023E04EE052E219
:10F84000B7C0D33019F580910905833031F080912C
:10F850004201882309F4AFC00FC08091E3028823DE
:10F86000B1F31092E30283E799E60E94755C809100
:10F870000805882361F3A7C081E0909109059330C2
:10F8800009F080E023E045E052E292C0D43019F55F
:10F8900080910905843031F080914201882309F478
:10F8A0008AC00FC08091E3028823B1F31092E30273
:10F8B0000E9467930E94F0C380910805882361F33A
:10F8C00082C081E090910905943009F080E020E247
:10F8D00046EF51E26DC0D53019F5809109058530AC
:10F8E00031F080914201882309F465C00FC08091F6
:10F8F000E3028823B1F31092E3020E9462B60E94F1
:10F90000F0C380910805882361F35DC081E0909188
:10F910000905953009F080E020E246ED51E248C04B
:10F92000D63019F580910905863031F08091420179
:10F93000882309F440C00FC08091E3028823B1F30B
:10F940001092E3020E9453B50E9428588091080546
:10F95000882361F338C081E090910905963009F061
:10F9600080E020E245EC51E223C0D73021F58091C0
:10F970000905873029F0809142018823E1F00FC00A
:10F980008091E3028823B9F31092E30286EE9CE7AC
:10F990000E94755C80910805882369F314C081E09A
:10F9A00090910905973009F080E023E044EE51E2A0
:10F9B0006C2F0E945858CF5FDF5FC53009F0D5CE5D
:10F9C00088E080930705DF91CF9108951F93CF932F
:10F9D000DF9361E081E00E94895C10910A05C0E03C
:10F9E0008C2F810F01F580910905882331F08091DA
:10F9F0004201882309F448C00DC08091E3028823A6
:10FA0000B1F31092E3020E94646380910805882399
:10FA100071F341C081E090910905911180E024E0EB
:10FA20004DEB51E22EC0813079F58091090581308E
:10FA300029F080914201882339F11AC08091E302B4
:10FA40008823B9F31092E3020E9453B50E94679392
:10FA5000D82F882319F080E00E9495B18D2F0E9445
:10FA6000F0C30E94646380910805882311F313C0DA
:10FA700081E090910905913009F080E020E24BEAA5
:10FA800051E26C2F0E945858CF5FC53009F0A8CFC3
:10FA900082E080930705DF91CF911F910895AF9287
:10FAA000BF92CF92DF92EF92FF920F931F93CF936B
:10FAB000DF93F82E61E081E00E94895CD0910A0515
:10FAC000C0E08F2D90E0880F991F9C012659364F7A
:10FAD0006901FC01E259F64F5F019C012E58364F37
:10FAE0007901D11120C080910905882331F08091DE
:10FAF0004201882309F4D7C00DC08091E302882316
:10FB0000B1F31092E3020E94646380910805882398
:10FB100071F3D0C081E090910905911180E024E05B
:10FB20004CE453E2BDC0D13081F5809109058130AC
:10FB300031F080914201882309F4B5C016C080914C
:10FB4000E3028823B1F31092E30200E010E02FEF0C
:10FB500030E040E050E0B70182E493E20E947DDEB5
:10FB600080910805882329F3A5C011E0809109053B
:10FB7000813009F010E0F701808191810E945547A2
:10FB800000E09C0148E353E263C0D23081F58091EC
:10FB90000905823031F080914201882309F483C045
:10FBA00016C08091E3028823B1F31092E30200E0D3
:10FBB00010E024E031E045E050E0B50181E393E25C
:10FBC0000E947DDE80910805882329F373C011E02F
:10FBD00080910905823009F010E0F5018081918162
:10FBE0000E94554700E09C014AE253E231C0D33005
:10FBF000A1F580910905833031F08091420188237D
:10FC000009F451C016C08091E3028823B1F3109229
:10FC1000E30200E010E02EE630E045E050E0B601FF
:10FC200086E293E20E947DDE80910805882329F315
:10FC300041C011E080910905833009F010E0F60120
:10FC4000808191810E94554700E09C0142E253E28D
:10FC50006C2F812F0E9447DD26C0D43021F5809182
:10FC60000905843029F0809142018823E1F00FC01A
:10FC70008091E3028823B9F31092E3020E94679314
:10FC80000E94F0C380910805882369F313C081E0C6
:10FC900090910905943009F080E020E243E153E2BD
:10FCA0006C2F0E945858CF5FDF5FC53009F019CF25
:10FCB000C0930705DF91CF911F910F91FF90EF90B7
:10FCC000DF90CF90BF90AF90089590917C03E92F83
:10FCD000F0E0E858FC4F80839F5F943018F49093D5
:10FCE0007C0302C010927C038091FF048F5F80939D
:10FCF000FF0408958091001390910113891759F022
:10FD0000E92FF0E0E058FD4E80819F5F9F77909350
:10FD1000011390E008958FEF9FEF0895CF93FC01BA
:10FD200080818B33A9F08091FF04843088F4C62F42
:10FD3000BF0180917C0320E6829FC001112482587C
:10FD40009C4F0E9496ED8C2F0E94657E81E001C041
:10FD500080E0CF9108952F923F924F925F926F92E1
:10FD60007F928F929F92AF92BF92CF92DF92EF924B
:10FD7000FF920F931F93CF93DF9300D000D000D05A
:10FD8000CDB7DEB78C010E941840F801C680D7803D
:10FD9000E084F184C114D104E104F10409F05CC2EF
:10FDA0002485222309F4C6C232852150248721E00C
:10FDB000230F22874585241301C01286F80124E011
:10FDC000329FE00DF11D1124C684D784E088F188AC
:10FDD000F801C282D382E482F582DC01CB018C0D72
:10FDE0009D1DA11DB11D86839783A087B187848146
:10FDF0009581892B09F49EC2FFB7FD83F894F80121
:10FE0000228033800481158180910E018B3121F095
:10FE10008F3F09F01EC205C0E4EBF8E124912E8368
:10FE20009FC08BE180930E01E4EBF8E1E491EF3F9A
:10FE300009F40FC2E13009F44AC0FCF4E1118FC0AB
:10FE400014BC15BC84B5826084BD85B5816085BD58
:10FE5000EFE6F8E1E491F0E0EE0FFF1FE05CF74E13
:10FE6000859194919093880980938709EFE8F8E150
:10FE7000E491E09386091E8276C0E23009F44BC01B
:10FE8000E33009F06CC010929000109291008091C4
:10FE900091008860809391008091910081608093AF
:10FEA0009100EFE6F8E1E491F0E0EE0FFF1FE05C77
:10FEB000F74E859194919093820980938109EFE8A0
:10FEC000F8E1E491E0938009E3E0EE834CC0109206
:10FED0008000109281008091810088608093810071
:10FEE00080918100816080938100EFE6F8E1E491E8
:10FEF000F0E0EE0FFF1FE05CF74E85919491909338
:10FF0000850980938409EFE8F8E1E491E09383099F
:10FF100081E08E8328C01092B0001092B1008091D1
:10FF2000B00082608093B0008091B10081608093C6
:10FF3000B100EFE6F8E1E491F0E0EE0FFF1FE05CC6
:10FF4000F74E8591949190933F0380933E03EFE8A1
:10FF5000F8E1E491E093400392E09E8304C0EE83D5
:10FF6000FE81F7FD76C12101612C712C61E08BE1EE
:10FF70000E94303F4801A12CB12C8E818D7F09F069
:10FF8000BDC060E072E18AE790E0A50194010E94A3
:10FF900011ED29833A834B835C8369017A0121E067
:10FFA000C21AD108E108F1088FEFC816D104E104A4
:10FFB000F10409F008F44DC060E472E48FE090E0D1
:10FFC000A50194010E9411ED69017A0191E0C91A1D
:10FFD000D108E108F108EE81E23001F5FFEFCF161C
:10FFE000D104E104F10409F008F4A2C160E970ED64
:10FFF00083E090E0A50194010E9411ED69017A016E
:020000021000EC
:1000000081E0C81AD108E108F1089FEFC916D104B0
:10001000E104F10409F0E0F583E069C0EFEFCE16EA
:10002000D104E104F104B9F0B0F068E478EE81E0C5
:1000300090E0A50194010E9411ED69017A01F1E0BF
:10004000CF1AD108E108F1082E81222309F415C145
:1000500066C181E001C082E02E812223A1F047C069
:1000600089819A81AB81BC812AE0B595A795979546
:1000700087952A95D1F76C017D01E1E0CE1AD10870
:10008000E108F10885E095B5987F892B85BD7FC093
:1000900068E478EE81E090E0A50194010E9411ED02
:1000A00069017A01F1E0CF1AD108E108F1082FEFD8
:1000B000C216D104E104F10409F008F4DCC064E2E2
:1000C00074EF80E090E0A50194010E9411ED6901B8
:1000D0007A0181E0C81AD108E108F1089FEFC9163A
:1000E000D104E104F10411F008F0E9C085E0909139
:1000F000B100987F892B8093B10049C060E072E124
:100100008AE790E0A50194010E9411ED69017A014E
:1001100081E0C81AD108E108F108C114D10491E0C6
:10012000E906F10488F068E478EE81E090E0A5014A
:1001300094010E9411ED69017A01E1E0CE1AD10823
:10014000E108F10883E001C081E0FE81F13071F443
:1001500090918100987F892B8093810045284628C3
:100160004728C9F42FEF3FEFA90140C02E8123306B
:1001700071F490919100987F892B8093910045288C
:100180004628472841F42FEF3FEFA90151C04528E9
:100190004628472869F09801220F331FD1010E9499
:1001A000CCE928EE33E040E050E00E949FE903C034
:1001B0002FEF3FEFA9018E818130C1F08CF48111C6
:1001C00048C0C7BC2093910930939209409393098A
:1001D0005093940980916E00826080936E0039C0C4
:1001E0009E819230A9F0933019F133C0D0928900EA
:1001F000C092880020938D0930938E0940938F0917
:100200005093900980916F00826080936F0021C0AD
:10021000C092B300209341033093420340934303C1
:10022000509344038091700082608093700011C0ED
:10023000D0929900C09298002093890930938A093E
:1002400040938B0950938C09809171008260809358
:100250007100ED81EFBF6EC0DC01CB018C199D09EF
:10026000AE09BF09B7FD66C01498F801168217825F
:10027000108611865FC084E03ACFEFEFCE16D1042E
:10028000E104F104D1F0C8F062E17AE780E090E0A7
:10029000A50194010E9411ED69017A0181E0C81A5B
:1002A000D108E108F1089FEFC916D104E104F10477
:1002B00011F008F0D5CE84E0E6CE83E0E4CE62E132
:1002C0007AE780E090E0A50194010E9411ED6901B8
:1002D0007A01F1E0CF1AD108E108F1082FEFC21638
:1002E000D104E104F104C9F0C0F089819A81AB81A5
:1002F000BC815AE0B595A795979587955A95D1F702
:100300006C017D01E1E0CE1AD108E108F108FE811F
:10031000FF2309F4B7CE87E0EACE86E09DCE8FEFCB
:10032000C816D104E104F10409F048F684E094CE43
:1003300082E0DDCE26960FB6F894DEBF0FBECDBFAD
:10034000DF91CF911F910F91FF90EF90DF90CF90B1
:10035000BF90AF909F908F907F906F905F904F90E5
:100360003F902F900895CF93DF93EC0160E0CE0192
:100370000E948E7E811103C00E9414D3F7CFCE015C
:100380000E94C33D8823C1F3DF91CF910895DF928E
:10039000EF92FF920F931F93CF93DF93CDB7DEB70A
:1003A0006E970FB6F894DEBF0FBECDBF6091EE1111
:1003B0007091EF116115710509F14DE150E0CE0129
:1003C00001967C010E9419E51E8EF7018F010E191E
:1003D0001F09D190DD2019F09AE0D912F7CFF7016B
:1003E000E00FF11F108260E0C7010E948E7E88231B
:1003F00029F0C7010E94C33D811109C081E020910D
:10040000EE113091EF11232BA1F480E012C0DD201A
:1004100049F00F5F1F4F8091EE119091EF11080F7F
:10042000191F02C000E010E01093EF110093EE11CD
:10043000E5CF6E960FB6F894DEBF0FBECDBFDF914D
:10044000CF911F910F91FF90EF90DF90089524E7D7
:1004500033E040E753E06CE673E088E693E00C9409
:10046000E55080917E0990917F09009731F04AE034
:1004700050E060E070E00C94B7E360E070E0CB0126
:10048000089580917E0990917F09009731F04AE0AC
:1004900050E060E070E00C948CE260E070E0CB0132
:1004A00008950E94418297FD0CC00E9441826F3FD7
:1004B00071058105910509F034F40E944182862F6F
:1004C000089580E008958FEF089580917E099091BE
:1004D0007F09892B39F00E94518291E0811103C07C
:1004E00090E001C091E0892F08950F931F93CF935F
:1004F00080917E0990917F090097F1F0FC018F01B6
:10050000C1912C2F2F7D89F0C53411F0C536B9F774
:10051000F801108260E070E00E941DE1F801C083E4
:10052000562F472F382F292F0BC060E070E0CF9156
:100530001F910F910C941DE150E040E030E020E06D
:10054000652F742F832F922FCF911F910F910895B4
:1005500081548A3108F041C0A82FB0E04091771251
:10056000509178126091791270917A1204C0769548
:100570006795579547958A95D2F740FF2EC0E09131
:10058000F111F091F211A35ABD4E8C918823E9F03C
:10059000E80FF11D808190ED980F9A3098F08E321F
:1005A00011F481810CC08D3211F08B3271F4818194
:1005B00090ED980F9A3030F08E3239F4828180536A
:1005C0008A3018F49E2F8F2F02C090E080E0909325
:1005D0007E0980937F0981E0089580E008950E945C
:1005E000A882882341F081E020917E0930917F0923
:1005F000232B09F480E00895FC01238121110C9440
:100600007C35089591E0909345039091C00095FF4B
:10061000FCCF8093C60008954F925F926F927F92B5
:100620009F92AF92BF92CF92DF92EF92FF920F9381
:100630001F93CF93DF931F92CDB7DEB70E94C78180
:10064000811177C28091FF04843028F40E947A7E61
:10065000AC0197FF3BC18091B206882309F469C2BF
:100660008091FF04811102C01092FB09EE24E394F3
:100670004091520950915309609154097091550964
:1006800080914E0990914F09A0915009B091510964
:10069000481759076A077B0708F4E12C00E010E0CF
:1006A000BB24B39480E6A82E9DE8C92E94E2D92EEF
:1006B0002DE8922E8091FF04843008F03AC2E110B8
:1006C00038C28091FB09811134C28091A9089091B0
:1006D000AA08A091AB08B091AC08809352099093FE
:1006E0005309A0935409B093550941E050E0BE016D
:1006F0006F5F7F4F81EA98E00E944B38019719F4B1
:10070000898190E002C08FEF9FEFF82EEE24E394F2
:1007100040905209509053096090540970905509C7
:1007200040914E0950914F096091500970915109C3
:100730004416550666067706C8F4E12C8F3FFFEF96
:100740009F0709F46CC02AE0821709F48DC08DE080
:10075000F81609F489C093E2F91619F0EAE3FE12DB
:100760009BC08091FA09811197C073C00E94D55037
:1007700081EA98E00E947C358091BC08882359F179
:1007800081508093BC08989EC001112441E061E033
:100790008F53974F0E946A75E091BC0824E0E29F56
:1007A000F0011124E354F74F40815181628173813C
:1007B000409352095093530960935409709355091B
:1007C00081EA98E00E9437CA8091B3068823B1F08D
:1007D000B092B20613C01092B2060E94EC510E9471
:1007E000C8CF0E9445CF6D3371058105910530F06A
:1007F000D092EF11C092EE110E94C7818091B20693
:1008000081112BC0E0EAF4E284913F019FEF691A65
:10081000790A8823F1F00E940283F301F5CFE6E71D
:10082000F1E284913F012FEF621A720A882321F0CE
:100830000E940283F301F5CFE1E9F4E284913F01E4
:100840009FEF691A790A882321F00E940283F3013D
:10085000F5CFE3E2FE1208C005C023E2F21266C142
:1008600000E010E0B092FB091092FA0901151105A1
:1008700019F40E945AD10DC080917C03A89E000DEE
:10088000111D1124F801E258FC4F108280E00E94F3
:10089000657E00E010E00ECF0F35110508F00ACF9D
:1008A000FBE3FF1202C0B092FA098091FA098111AC
:1008B00001CF80917C03F801A89EE00DF11D112469
:1008C000E258FC4FF0820F5F1F4FF4CE982F20911B
:1008D0002306309124068A3019F09D3009F0F4C0C7
:1008E0001092F9092115310519F40E945AD1AACEA6
:1008F000F901E756F64F1082109224061092230653
:1009000029E939E08901F90180812F5F3F4F803269
:10091000C9F378018E3409F07CC00115110509F482
:1009200078C068E874E2C8010E9428E5DD24D39409
:10093000892B11F4D12C09C06EE470E0C801049633
:100940000E9482ED009709F08C014AE050E060E0DF
:1009500070E0C80101960E948CE260939509709343
:100960009609809397099093980900912506109114
:10097000260620912706309128060F5F1F4F2F4F24
:100980003F4F601771078207930729F0D11003C00A
:1009900085E594E22AC06AE270E0C7010E94BAEDE0
:1009A0009C01009701F1982F9E1910E0992339F0CE
:1009B0009150F701E90FF11D80811827F7CF4AE028
:1009C00050E060E070E0C90101960E948CE2012FC6
:1009D00010E020E030E0601771078207930741F0D4
:1009E00086E394E202C08CE094E20E941C7733CE4E
:1009F0008091950990919609A0919709B0919809D5
:100A00008093250690932606A0932706B093280688
:100A10000EC08091B006882351F069E472E0C801ED
:100A20000E948DED892B19F088E593E2DECF80914D
:100A30005001811124C067E470E0C7010E9482ED7B
:100A40000097E9F04AE050E060E070E001960E9413
:100A50008CE2643071058105910588F4E5E9F3E2E3
:100A600084918F010F5F1F4F882321F00E94028322
:100A7000F801F6CF60E08BE893E20E94F3586DE452
:100A800072E0C7010E948DED892B21F410921501AF
:100A90001092E50262E572E0C7010E948DED892B9C
:100AA00021F482E893E20E94EC3D67E572E0C70121
:100AB0000E948DED892B11F40E9429A761E089E93C
:100AC00099E00E948E7EBECD2F3531050CF0BACD57
:100AD0009C35C1F40E947A7E97FDB4CD2091F9092E
:100AE0002111B0CD2091230630912406A9014F5F3A
:100AF0005F4F5093240640932306F901E756F64FC3
:100B00008083A0CD9B3319F481E08093F909809113
:100B1000F909811197CDC90101969093240680931C
:100B20002306F901E756F64F40838CCD1092FA095F
:100B3000A0CE0F90DF91CF911F910F91FF90EF907A
:100B4000DF90CF90BF90AF909F907F906F905F901D
:100B50004F9008958F929F92AF92BF92EF92FF9223
:100B60001F93CF93DF93CDB7DEB7A0970FB6F8945E
:100B7000DEBF0FBECDBF611571058105910581F105
:100B800010E0842E912CA12CB12CEE24E394F12CB6
:100B9000EC0EFD1EE10EF11C17FDFA94A501940167
:100BA0000E949FE9F7016083B901CA011F5F6115C7
:100BB00071058105910549F7115020F1E1E0F0E060
:100BC000EC0FFD1FE10FF11D17FDFA9580818A30B2
:100BD00010F097E301C090E3890F0E940283ECCFED
:100BE00080E3A0960FB6F894DEBF0FBECDBFDF91B5
:100BF000CF911F91FF90EF90BF90AF909F908F90FB
:100C00000C940283A0960FB6F894DEBF0FBECDBF42
:100C1000DF91CF911F91FF90EF90BF90AF909F9089
:100C20008F900895CF92DF92EF92FF926B017C013B
:100C300097FF0BC08DE20E940283F094E094D09461
:100C4000C094C11CD11CE11CF11C4AE0C701B601D3
:100C5000FF90EF90DF90CF900C94AA858F929F9297
:100C6000AF92BF92CF92DF92EF92FF92CF936B0140
:100C70007C01B42E20E030E0A9010E94ABE587FFA3
:100C800007C08DE20E940283F7FAF094F7F8F0941F
:100C9000C0E060E070E080E09FE3CB1541F02DEC18
:100CA0003CEC4CEC5DE30E9411E6CF5FF6CF9B017C
:100CB000AC01C701B6010E94DCE96B017C010E9416
:100CC0004FEB4B015C014AE00E94AA85CC2389F1DD
:100CD000C501B4010E94B0E59B01AC01C701B6019A
:100CE0000E94DBE96B017C018EE20E94028320E01E
:100CF00030E040E251E4C701B6010E9411E64B0129
:100D00005C010E9448EB6B01770FEE08FF08C701FA
:100D1000B6010E941286C701B6010E94B2E59B018E
:100D2000AC01C501B4010E94DBE96B017C01C1503B
:100D3000F1F6CF91FF90EF90DF90CF90BF90AF9002
:100D40009F908F9008951F920F920FB60F921124CB
:100D50000BB60F922F938F939F93EF93FF93209156
:100D60000113E091001381E08E0F8F779091C60000
:100D7000821729F0F0E0E058FD4E9083E82FE093D1
:100D80000013FF91EF919F918F912F910F900BBEC8
:100D90000F900FBE0F901F901895CF93DF9361E0D7
:100DA00081E00E94895CD0910A05C0E0D11120C089
:100DB00080910905882331F080914201882309F44C
:100DC000ACC00DC08091E3028823B1F31092E3021E
:100DD0000E94646380910805882371F3A5C081E0B7
:100DE00090910905911180E024E047E056E292C01D
:100DF000D13019F580910905813031F0809142019F
:100E0000882309F48AC00FC08091E3028823B1F3DC
:100E10001092E30284EF98E80E94755C80910805C7
:100E2000882361F381C081E090910905913009F038
:100E300080E023E040E056E26DC0D23019F58091A9
:100E40000905823031F080914201882309F465C0A0
:100E50000FC08091E3028823B1F31092E30289EF7F
:100E600098E80E94755C80910805882361F35CC056
:100E700081E090910905923009F080E023E049EF8C
:100E800055E248C0D33019F580910905833031F01F
:100E900080914201882309F440C00FC08091E30291
:100EA0008823B1F31092E3028EEF98E80E94755CFC
:100EB00080910805882361F337C081E0909109058E
:100EC000933009F080E023E042EF55E223C0D430B4
:100ED00021F580910905843029F080914201882311
:100EE000E1F00FC08091E3028823B9F31092E3028E
:100EF00083E099E80E94755C80910805882369F376
:100F000013C081E090910905943009F080E023E05E
:100F100049EE55E26C2F0E945858CF5FDF5FC53015
:100F200009F044CFC0930705DF91CF9108951F9337
:100F3000CF93DF93182F7093190A6093180A61E01A
:100F400081E00E94895CD0910A05C0E091E01130F7
:100F500071F120F0123009F453C07BC0D111A5C04B
:100F60009923D9F0909109051916BCF04091CF1141
:100F70005091D0116091D1117091D2114F5F5F4F9C
:100F80006F4F7F4F4093CF115093D0116093D11189
:100F90007093D2119F5F909309058091420188233D
:100FA00009F416C121E041E062EE75E27AC0D11188
:100FB0007CC09923D9F0909109051916BCF0409195
:100FC000CF115091D0116091D1117091D2114F5F1A
:100FD0005F4F6F4F7F4F4093CF115093D01160936D
:100FE000D1117093D2119F5F9093090580914201B6
:100FF000882309F4EDC021E041E06BED75E251C0BA
:10100000D11153C09923D9F0909109051916BCF05C
:101010004091CF115091D0116091D1117091D211A6
:101020004F5F5F4F6F4F7F4F4093CF115093D01161
:101030006093D1117093D2119F5F909309058091B5
:101040004201882309F4C4C021E041E064ED75E267
:1010500028C0D1112AC09923D9F0909109051916F9
:10106000BCF04091CF115091D0116091D11170918D
:10107000D2114F5F5F4F6F4F7F4F4093CF1150930F
:10108000D0116093D1117093D2119F5F9093090595
:1010900080914201882309F49BC021E041E06BEC80
:1010A00075E28C2F0E94CAE093C0D13009F580917F
:1010B0000905813031F080914201882309F488C00C
:1010C0000DC08091E3028823B1F31092E3020E94E5
:1010D000646380910805882371F382C081E0909158
:1010E0000905913009F080E024E041EC55E26DC043
:1010F000D23019F580910905823031F0809142019A
:10110000882309F465C00FC08091E3028823B1F3FE
:101110001092E3028CE199E80E94755C80910805C9
:10112000882361F35DC081E090910905923009F058
:1011300080E023E047EB55E248C0D33019F58091B9
:101140000905833031F080914201882309F440C0C1
:101150000FC08091E3028823B1F31092E30282E290
:1011600099E80E94755C80910805882361F338C076
:1011700081E090910905933009F080E023E04EEA88
:1011800055E223C0D43021F580910905843029F03F
:10119000809142018823E1F00FC08091E30288230F
:1011A000B9F31092E30288E299E80E94755C80919D
:1011B0000805882369F314C081E0909109059430F3
:1011C00009F080E023E043EA55E26C2F0E94585872
:1011D000CF5FDF5F90E0C53009F0B9CEC09307055F
:1011E000DF91CF911F9108956BEF7AE880E00C9426
:1011F000978766EF7AE881E00C94978761EF7AE849
:1012000082E00C94978764E679E883E00C949787F2
:1012100021E02093DB026093140A7093150A8093F7
:10122000160A9093170A40E050E0BA018091180A1C
:101230009091190A0C940A5D60E070E080E291E4FC
:101240000C94088960E070E080E89FE30C940889C2
:101250006DEC7CEC8CEC9DE30C940889CF92DF92D2
:10126000EF92FF92CF93C82F0E9418406B017C0130
:1012700024EA30E74DE75FE36091140A7091150AA4
:101280008091160A9091170A0E94ABE587FD05C070
:101290004AEF50E060E070E003C040E050E0BA0187
:1012A000C40ED51EE61EF71EC092D702D092D802F9
:1012B000E092D902F092DA02C0930D01CF91FF9033
:1012C000EF90DF90CF9008958091E3021092E302B7
:1012D000882321F01092DB020C9464636091CF119B
:1012E0007091D0118091D1119091D2116115710539
:1012F0008105910571F10E94B2E52091140A3091A7
:10130000150A4091160A5091170A0E9411E69B0196
:10131000AC01609174037091750380917603909194
:1013200077030E94DCE960937403709375038093E4
:1013300076039093770383E00E942E8981E0809367
:1013400042011092CF111092D0111092D11110922F
:10135000D21180914201882349F084E793E00E94F2
:10136000D845BC018AE995E20C947B6308953F92CD
:101370004F925F926F927F928F929F92AF92BF92A5
:10138000CF92DF92EF92FF920F931F93CF93DF9351
:10139000CDB7DEB72A970FB6F894DEBF0FBECDBF2C
:1013A0009A878987362E8091E3021092E302882380
:1013B00029F01092DB020E946463FBC08091CF1180
:1013C0009091D011A091D111B091D2118D839E83B3
:1013D000AF83B887892B8A2B8B2B09F4A8C094E0A4
:1013E000699F80011124F801E859FC4F4080518029
:1013F0006280738020E030E04AE754E4C301B20128
:101400000E94DBE94B015C0120E030E04AE754E454
:10141000C301B2010E94DCE96B017C0180914101B2
:101420008823D1F1A1E03A1639F13A16A0F0B2E0E2
:101430003B1232C08090100A9090110AA090120ABC
:10144000B090130AC0903D01D0903E01E0903F0162
:10145000F090400121C08090080A9090090AA09065
:101460000A0AB0900B0AC0903501D0903601E09086
:101470003701F090380110C080900C0A90900D0A4E
:10148000A0900E0AB0900F0AC0903901D0903A0196
:10149000E0903B01F0903C016D817E818F819885C9
:1014A0000E94B2E52091140A3091150A4091160A63
:1014B0005091170A0E9411E69B01AC01C301B201D1
:1014C0000E94DCE92B013C018D819E81AF81B885B2
:1014D000B7FF18C0A5019401C301B2010E94ABE59A
:1014E00087FD08C0F801E859FC4F408251826282B2
:1014F000738217C0F801E859FC4F80829182A28262
:10150000B3820FC0A7019601C301B2010E943CEC57
:10151000181644F7F801E859FC4FC082D182E282E4
:10152000F382832D0E942E8981E0809342011092E4
:10153000CF111092D0111092D1111092D21180912E
:1015400042018823B1F1A4E03A9EC0011124FC01BC
:10155000E859FC4FDC01A450B64F2D913D914D91BF
:101560005C9160817181828193810E94DCE9698351
:101570007A838B839C832DEC3CEC4CEC5DE3609197
:10158000140A7091150A8091160A9091170A0E9408
:101590003CEC87FD05C0CE0101960E94D84504C0F1
:1015A000CE0101960E9484C0BC0189859A850E9463
:1015B0007B632A960FB6F894DEBF0FBECDBFDF91D6
:1015C000CF911F910F91FF90EF90DF90CF90BF9040
:1015D000AF909F908F907F906F905F904F903F90D3
:1015E000089562E083E995E20C94B78961E08CE8A4
:1015F00095E20C94B78960E085E895E20C94B78990
:10160000AF92BF92CF92DF92EF92FF921F93CF9350
:10161000DF9361E081E00E94895CC0910A05D0E01F
:1016200083E5E82E85E2F82E9CE1C92E95E2D92EBD
:1016300022E7A22E25E2B22EC11120C08091090519
:10164000882331F080914201882309F4B4C00DC091
:101650008091E3028823B1F31092E3020E94646355
:1016600080910805882371F339C181E090910905C3
:10167000911180E024E040E855E29AC0C13019F5AC
:1016800080910905813031F080914201882309F46D
:1016900092C00FC08091E3028823B1F31092E3025D
:1016A0008DEC96E80E94755C80910805882361F3B3
:1016B00015C181E090910905913009F080E023E0A7
:1016C00046E755E275C0C23029F5809109058230A0
:1016D00031F080914201882309F46DC011C08091DE
:1016E000E3028823B1F31092E302B092EF11A092CB
:1016F000EE110E94C78180910805882351F3EEC046
:1017000081E090910905923009F080E020E248E6FE
:1017100055E24EC0C33039F580910905833031F070
:1017200080914201882309F446C013C08091E302EE
:101730008823B1F31092E302D092EF11C092EE1120
:101740000E94C7810E945D6380910805882341F350
:10175000C5C081E090910905933009F080E020E256
:1017600047E555E225C0C43031F580910905843044
:1017700029F0809142018823F1F011C08091E302A9
:101780008823B9F31092E302F092EF11E092EE1188
:101790000E94C78180910805882359F39FC081E08A
:1017A00090910905943009F080E020E242E455E28E
:1017B0006D2F0E9458588091E4119091E51120916D
:1017C000E2113091E311232B11F4892B61F1C53023
:1017D00061F580910905853031F0809142018823BF
:1017E00009F47AC013C08091E3028823B1F3109208
:1017F000E3021092CC0C1092CB0C0E94DDCF0E9421
:101800005D6380910805882341F368C081E0909171
:101810000905953009F080E020E24DE255E26D2F98
:101820000E94585859C015E001C016E0C11324C0E9
:10183000809109058C1729F0809142018823D9F005
:101840000FC08091E3028823B9F31092E30288E38A
:101850009DE80E94755C80910805882369F33EC06D
:1018600081E0909109059C1380E023E041E255E27C
:101870006D2F0E9458581C2F81E0810FC81323C080
:10188000809109058C1729F0809142018823D9F0B5
:101890000FC08091E3028823B9F31092E30288E736
:1018A0009CE80E94755C80910805882369F316C046
:1018B00081E0909109059C1380E023E046E355E226
:1018C0006D2F0E945858DF5FCF5FD53009F0B4CE3E
:1018D0001E5F1093070502C016E0CECFDF91CF91B7
:1018E0001F91FF90EF90DF90CF90BF90AF90089541
:1018F000CF93DF9361E081E00E94895CD0910A057B
:10190000C0E0D11120C080910905882331F0809179
:101910004201882309F4A1C00DC08091E30288230D
:10192000B1F31092E3020E9464638091080588235A
:1019300071F39BC081E090910905911180E024E052
:1019400044E155E287C0D13069F5809109058130C5
:1019500031F080914201882309F47FC019C0809141
:10196000E3028823B1F31092E3024091740950918D
:10197000750960916C0970916D0980917009909161
:1019800071090E9419C180910805882311F36DC067
:1019900081E090910905913009F080E020E248E073
:1019A00055E258C0D23059F580910905823031F0A6
:1019B00080914201882309F450C017C08091E3024E
:1019C0008823B1F31092E302409174095091750994
:1019D0006FEF7FEF80917009909171090E9419C19A
:1019E00080910805882321F340C081E0909109058A
:1019F000923009F080E020E248EE54E22BC0D33070
:101A000061F580910905833029F080914201882396
:101A100021F117C08091E3028823B9F31092E30209
:101A2000409174095091750960916C0970916D092C
:101A300080E090E00E9419C180910805882329F375
:101A400014C081E090910905933009F080E020E214
:101A500048EF54E26C2F0E945858CF5FDF5FC530CB
:101A600009F04FCF84E080930705DF91CF9108956F
:101A7000CF93DF9361E081E00E94895CD0910A05F9
:101A8000C0E0D11120C080910905882331F08091F8
:101A90004201882309F4A1C00DC08091E30288238C
:101AA000B1F31092E3020E946463809108058823D9
:101AB00071F39BC081E090910905911180E024E0D1
:101AC00040EE54E287C0D13069F58091090581303C
:101AD00031F080914201882309F47FC019C08091C0
:101AE000E3028823B1F31092E3024091720950910E
:101AF000730960916A0970916B0980916E099091E8
:101B00006F090E9419C180910805882311F36DC0E7
:101B100081E090910905913009F080E020E244EDE8
:101B200054E258C0D23059F580910905823031F025
:101B300080914201882309F450C017C08091E302CC
:101B40008823B1F31092E302409172095091730916
:101B50006FEF7FEF80916E0990916F090E9419C11C
:101B600080910805882321F340C081E09091090508
:101B7000923009F080E020E244EB54E22BC0D330F5
:101B800061F580910905833029F080914201882315
:101B900021F117C08091E3028823B9F31092E30288
:101BA000409172095091730960916A0970916B09B3
:101BB00080E090E00E9419C180910805882329F3F4
:101BC00014C081E090910905933009F080E020E293
:101BD00044EC54E26C2F0E945858CF5FDF5FC53051
:101BE00009F04FCF84E080930705DF91CF910895EE
:101BF000CF93DF938F389240B1F0E6E7F1E2849122
:101C0000EF012196882321F00E940283FE01F7CF85
